:020000040800F2
:100000000000012035770008EF330008F1330008C5
:10001000F3330008F5330008F73300080000000050
:10002000000000000000000000000000F93300089C
:10003000FB33000800000000FD330008FF33000818
:100040008577000885770008013400088577000867
:1000500085770008857700080D3400081D340008F6
:10006000857700082D3400088577000835340008AE
:10007000413400084D340008857700088577000872
:10008000593400085D34000885770008857700083A
:1000900000000000857700086934000885770008B3
:1000A0008577000885770008857700088577000840
:1000B0008577000885770008857700088577000830
:1000C00085770008857700086D340008857700087B
:1000D000857700087934000885770008857700085F
:1000E0008577000885770008853400088577000843
:1000F00085770008000000000000000085770008F8
:100100008577000885770008913400088577000816
:1001100085770008857700088577000885770008CF
:1001200085770008857700088577000885770008BF
:080130008577000885770008BF
:1001400010B5054C237833B9044B13B10448AFF311
:1001500000800123237010BD48080020000000002B
:10016000A42C030808B5034B1BB103490348AFF3A4
:10017000008008BD000000004C080020A42C0308EB
:1001800014214160704714207047406A7047000096
:1001900081010008870100088B010008A101000807
:1001A00010B5044604F1100000F05CFCC4F8F8003F
:1001B0000148C4F87C0110BD90010008F8B5E6B014
:1001C00004460D4616461F460A4906A800F0CAFE18
:1001D00070996F9A05910492009733466E996D9AC3
:1001E000039102922A466C990191214600F060F831
:1001F00067B0F0BD9C010008F8B5E6B004460D46B6
:1002000016461F46094906A800F0ACFE6F996E9A83
:100210000491039200976D996C9A02910192334672
:100220002A46214600F087F867B0F0BD9C0100081F
:1002300038B500281CBF01680029184A23D1184B83
:100240001C684FF6F0710C404CF24025AC421FBFC9
:100250001B6819404CF27024A14212D1114D29683B
:1002600079B911490B68C3F30B03B3F58A6F1FBF4C
:100270000968C1F30B0140F28343994204BF012195
:10028000117028B905E0094B994204BF0121117092
:100290004068BDE8324002F073BC00BF6408002033
:1002A00000ED00E0002004E00010005C0000374892
:1002B0002DE9F04104460D46216816464A681F465E
:1002C00090478046B8F5403F2ED122680A9993683E
:1002D000204698478046B8F5403F25D12368089AC4
:1002E0000799D3F80CC02046E0478046B8F5403F58
:1002F0001AD12368069A39461F692046B8478046B6
:10030000B8F5403F10D1236829465D693246204642
:10031000A8478046B8F5403F06D123680B9A099953
:100320009D692046A847804621680A682046904774
:100330004046BDE8F0812DE9F04104460D462168B4
:1003400016464A681F4690478046B8F5403F2ED172
:1003500022680A999368204698478046B8F5403F3E
:1003600025D12368089A0799D3F80CC02046E047A6
:100370008046B8F5403F1AD12368069A39461F696E
:100380002046B8478046B8F5403F10D1236829463B
:100390005D6932462046A8478046B8F5403F06D101
:1003A00023680999DD6900222046A8478046216814
:1003B0000A68204690474046BDE8F0814FF440303F
:1003C00070470000F0B50C4685B0114600281A466B
:1003D0001CBF0568002D0B4B11D082B104B971B957
:1003E0000D9860B10F9E0E9F0A9B02900496039792
:1003F0000B980C9E009001962046A847034618468D
:1004000005B0F0BD020003002DE9F04F0646D0B064
:100410000868F56DD6F860E0726EB76EF36E00BADC
:1004200000906C46486800BA60600DF1400888682A
:1004300000BAA060C86800BAE060086900BA20612C
:10044000486900BA6061886900BAA061C86900BAE9
:10045000E061086A00BA2062486A00BA6062886A8D
:1004600000BAA062C86A00BAE062086B00BA2063F2
:10047000486B00BA6063886B00BAA063C86B00BAAF
:10048000E063402058F80C1C58F820CC58F838ACE1
:100490008CEA010158F840CC8AEA01018CEA010992
:1004A0004FEAF979401E48F8049BEBD187EA020035
:1004B00000EA0E00784010EBF5610098DFF824C4E4
:1004C00041186144C81882EABE032B404FEAF0612C
:1004D00053405918636859186144CF194FEAB5035E
:1004E00083EABE01014081EABE0111EBF765A16814
:1004F0004D196544A91883EAB0023A404FEAF16504
:100500005A405519E26855194FEAB70282EAB00716
:1005100065440F4005EBBE0E97EAB00717EBFE658A
:1005200027697D194FEAB10782EA0701654401EAAC
:100530000E01EB18514011EBF36561694D194FEA5B
:10054000BE0187EA010E65440EEA030E15EBB0000A
:100550008EEA070E0EEBF065D4F818E0754465449A
:10056000AA1881EAB30505404FEAF26E4D40AE4449
:10057000E569AE44E64477444FEAB00080EAB30E42
:100580000EEA020E8EEAB30E0EEBF765D4F820E009
:1005900075446544691880EAB2053D404FEAF16E42
:1005A0004540AE44656AAE44E6440EEBB3034FEA01
:1005B000B70787EAB20E0EEA010E8EEAB20E0EEB14
:1005C000F365D4F828E075446544281887EAB10536
:1005D0001D404FEAF06E7D40AE44E56AAE44E6440D
:1005E0000EEBB2024FEAB30383EAB10E0EEA000E3D
:1005F0008EEAB10E0EEBF265D4F830E07544654436
:10060000EF1983EAB00515404FEAF76E5D40AE443E
:10061000656BAE44E6440EEBB1014FEAB20282EAEA
:10062000B00E0EEA070E8EEAB00E0EEBF165D4F8AE
:1006300038E075446544EB1882EAB7050D404FEA8F
:10064000F36E5540AE44E56BAE44E6440EEBB000AD
:100650004FEAB10181EAB70E0EEA030E8EEAB70E39
:100660000EEBF065D4F840E07544654481EAB30EC2
:10067000AA180EEA000E4FEAF2658EEA010E7544E2
:10068000DDF844E04FEAB000754480EAB30E6544FB
:100690000EEA020E15EBB7078EEAB30E0EEBF76506
:1006A000DDF848E04FEAB202754480EA020E654484
:1006B0000EEA070E69188EEA000E0EEBF165DDF802
:1006C0004CE07544654405EBB3034FEAB70E1427BD
:1006D0000DF1500CDFF810528EEA010B82EA0B0B81
:1006E0000BEBF36A5CF804BBDA44AA44504483EA97
:1006F000B10B4FEAF06A8EEA0B0BDA445CF804BBEC
:10070000DA44AA44524480EAB30B4FEAF26A8BEA15
:10071000B10BDA445CF804BBDA444FEAB000AA44F7
:1007200080EA020BD6448BEAB30B0BEBFE6A5CF853
:1007300004BBDA444FEAB202AA4482EA0E0B0AEB87
:10074000B10180EA0B0B0BEBF16A5CF804BBDA44F5
:100750007F1DAA44282F0AEBB3034FEABE0EBBD37A
:100760003C2F61D3502F4DD204EB870CC7F15407B7
:100770005E4CA7FB04A504465D4FA8088EEA010A5B
:1007800082EA0A0A5CF804BB0AEBF3655D447D1952
:100790002C1983EAB10A4FEAF4658EEA0A0A554435
:1007A0005CF804AB5CF804BB55447D19AA1884EAD4
:1007B000B30A4FEAF2658AEAB10A55445D444FEA4A
:1007C000B4047D1984EA020AAE448AEAB30A0AEB49
:1007D000FE655CF804AB55444FEAB2027D1982EA2B
:1007E0000E0A15EBB10184EA0A0A5CF804BB0AEBB5
:1007F000F1655D447D1915EBB303401E4FEABE0E53
:10080000BCD12046F46D1B19F365336EC9183166EF
:10081000716E71447166B36ED218B266F16E401893
:10082000F06650B0BDE8F08F4EEA010B0EEA010A07
:100830000BEA020B4BEA0A0A0AEBF36554F827A00D
:10084000DFF8B0C0554443EAB10B654403EAB10A8E
:100850000BEA0E0B28184BEA0A0A7F1C0AEBF0651C
:1008600054F827A0554440EAB30B654400EAB30AA4
:100870000BEAB10BAA184BEA0A0A7F1C0AEBF265D5
:1008800054F827A055444FEAB00040EA020B6544F3
:1008900000EA020A0BEAB30BAE444BEA0A0A7F1CD9
:1008A0000AEBFE6554F827A055444FEAB20242EA2B
:1008B0000E0B654402EA0E0A0BEA000B15EBB101C0
:1008C0004BEA0A0A7F1C0AEBF16554F827A055444D
:1008D0007F1C65443C2F05EBB3034FEABE0EA3D348
:1008E00040E700BF9979825AA1EBD96ECDCCCCCC30
:1008F000D6C162CADCBC1B8F00B581B00168074A53
:10090000914200D110B9064801B000BD7C212EF003
:1009100078FF4FF4003001B000BD00BF040A0008AA
:10092000030002002DE9F0410B4A92E8F85188B02B
:10093000694681E8F8510268084B9A4200D118B91B
:10094000074808B0BDE8F0811422083000F04FFBE2
:1009500008B0BDE8F08100BFE4090008040A0008FF
:1009600003000200152904D20268044B9A4200D108
:1009700008B903487047083000F048BB040A000873
:100980000300020010B481B013460268074CA24273
:1009900000D118B901B010BC0548704701B000F192
:1009A000240210BC083000F035BB00BF040A000868
:1009B0000300020010B481B013460268074CA24243
:1009C00000D118B901B010BC054870470A4601B003
:1009D00000F1240110BC083000F070BB040A0008CC
:1009E000030002000123456789ABCDEFFEDCBA9816
:1009F00076543210F0E1D2C3000000000000000085
:100A000000000000F9080008250900086509000831
:100A100085090008B509000809040008810F0008CD
:100A2000CD0F0008890F0008F0B5A3B004460B48AD
:100A300002900D4616461F46094B0822402104A885
:100A400000F0D1FA28980190009733462A462146B3
:100A500002A800F01BF823B0F0BD00BF040A000894
:100A6000180A000810B5040008BF002408D0054883
:100A7000054B20600822402104F1080000F0B3FA81
:100A8000204610BD040A0008180A00082DE9F041AC
:100A900004460E46216817464A681D469047804620
:100AA000B8F5003F19D12268069993682046984707
:100AB0008046B8F5003F10D123683146DE683A46DB
:100AC0002046B0478046B8F5003F06D12368079A14
:100AD00029461D692046A847804621680A682046A5
:100AE00090474046BDE8F08110B500F033FA4FF46E
:100AF000403400280EBF034C4FF4C0712EF081FE2D
:100B0000204610BD0200030010B5044600F022FA92
:100B100008B9054810BD0021A160D0F87C211168FA
:100B200088474FF4403010BD0200030070B5044602
:100B30000D4600F00FFA064E40B1D0F87C01416836
:100B40008847A84224BF65604FF44036304670BDE8
:100B5000020003002DE9FF4715000C4600D02CB120
:100B6000064600F0F7F95FEA000801D16448C3E0E7
:100B7000D8F8F80001684A689047B0F5003F17D1EF
:100B8000D8F87C118A68404690478146B9F1810FB8
:100B900080F09E80A94508F1FC0A17D2D8F8F80029
:100BA0000368D3F80CC02A462146E047B0F5003F61
:100BB00040F08E80D8F8F8000368D3F810C06A4679
:100BC0005146E047B0F5003F76D10AE0002004E04E
:100BD000215C0AF800100098401C00900098A84280
:100BE000F6D34FF0000C4749474A484B01AC0098F8
:100BF000844558D2D3E9007001ADC5E90070107882
:100C000000281ABF042086464FF0000E085854F8FA
:100C10000E5028443E4D05600127D0F800E0876063
:100C2000019D4F681AF80C007D408EEA050585F09D
:100C3000040E65680F687D4085F0FC05754485F0FD
:100C4000A30568400AF80C000CF1010CCFE7D3E9CA
:100C5000004501A8C0E9004510782E4D002814BFBA
:100C60004FF0040E4FF0000E01A8744651F80EE04C
:100C70000459A6440127CEF80050DEF80040CEF813
:100C800008704D68019F40687D406C400D68684069
:100C900084F0040480F0FC00041984F057040AF87E
:100CA0000C400CF1010CCC45D1D3D8F8F800016808
:100CB0004A689047B0F5003F0AD1D8F8F8000368B9
:100CC000D3F80C804A465146C047B0F5003F01D0EA
:100CD000114811E0002006E05AF8201081F06A3136
:100CE0004AF82010401CB0EB990FF5D3B06840F0E3
:100CF0000100B0604FF4403004B0BDE8F08700BFA1
:100D000002000300EC6D0308640800202C0F0008AB
:100D1000ADBE4ED70DBE75A10100030038B50C461F
:100D2000017A1546CA0702D500F014F908B9084837
:100D300032BDD0F8F80003682146DC682A46A04797
:100D4000B0F5003F01D0034832BD4FF4403032BD12
:100D500002000300010003002DE9F84191B00546AF
:100D60000E461746402101A82EF04BFD297AC807F0
:100D700004D5284600F0EEF8040002D1DFF8A48084
:100D80004BE0D4F8F800DFF8A0800368D3F810C077
:100D90006A4601A9E047B0F5003F3ED1D4F8F8001B
:100DA00001684A689047B0F5003F36D1D4F87C110D
:100DB0008A6820469047D4F8F830024618461B68E7
:100DC000D3F80CC004F1FC01E047B0F5003F24D19A
:100DD000D4F87C0141688847D4F8F83002461846B8
:100DE0001B68D3F80CC001A9E047B0F5003F14D14F
:100DF000D4F8F8000268696893689847B0F5003F36
:100E00000BD1D4F8F80003681C693A463146A04774
:100E1000B0F5003F08BF4FF44038404612B0BDE87F
:100E2000F08100BF02000300010003002DE9F8413A
:100E3000A5B0074688461646402115A82EF0E1FCCD
:100E400000220492402105A82EF0DBFC387AC1076D
:100E50005ED5384600F07EF8050059D0D5F8F80088
:100E60002D4C0368D3F810C06A4605A9E047B0F5D9
:100E7000003F3CD1D5F8F80001684A689047B0F5CA
:100E8000003F34D1D5F87C118A6828469047D5F8C0
:100E9000F830024618461B68D3F80CC005F1FC0177
:100EA000E047B0F5003F22D1D5F87C014168884782
:100EB000D5F8F830024618461B68D3F80CC005A9CF
:100EC000E047B0F5003F12D1D5F8F8000268796824
:100ED00093689847B0F5003F09D1D5F8F80003684A
:100EE0001D6904AA15A9A847B0F5003F01D0204606
:100EF0000FE00A4B0A490B4A0396029101924046C1
:100F00001C68049B009415AA796800F0E5F900E0DC
:100F1000054826B0BDE8F08101000300F46D030828
:100F2000936E030026C703000200030004B0010112
:100F300000170145E90A0008090B00082D0B0008FD
:100F4000BD030008550B00081D0D0008590D0008D1
:100F50002D0E00080168024A914218BF0020704718
:100F6000340F000810B5040008BF002404D0034863
:100F70002060204609688847204610BD340F0008CD
:100F800020225C302EF039BCF0B58468A308002222
:100F900004F0030407E000F15C0555F8226035BA5F
:100FA00041F82250521C9A42F5D300220BE000F186
:100FB0005C0502EB830755F82360D500C5F11805E1
:100FC000EE40CE55521CA242F1D3F0BD30B5C468FC
:100FD00003690022E31AD5188C5C0544521C082AC8
:100FE0002C77F8D330BD0360C1600261704738B51B
:100FF000044615460022626023685A689047002024
:101000006061A061A5604FF4003032BD81604FF493
:10101000003070472DE9F84304462079D4F80C805D
:10102000450748BF244845D466691D46A8F101001C
:1010300000EAD60306EBC506B6EBC50F666102D221
:10104000A669761CA6611746A66906EB5576A661C9
:101050000E46E918884225D2A8EB03094A463146D4
:10106000F8182EF0CAFB2268136839460FE0424692
:1010700038462EF0C2FB23681A683946204690474E
:1010800007E0311811F00300F1D1226813682046FF
:101090009847484600EB0809A9F10101A942F0D39D
:1010A000002300E000202A1A3118F8182EF0A5FBC2
:1010B0004FF40030BDE8F283040002002DE9FC4F3C
:1010C000024685B0D0681369DFF86CC1DFF86C8127
:1010D000A0EB030A506840F004005060002703A80A
:1010E00002900DF10C0ED8E9003403A8544DC0E96C
:1010F00000342878534D00280CBF00230423994660
:101100005CF803305EF80940234401261D601C682A
:101110009E60DCF80430039DDCF80090DEF804608B
:101120005D406540484C654089EA0606474C66408C
:101130007519474C6540D8E9006B03AC0028C4E939
:10114000006B0EBF002404200424029E5CF8000003
:10115000345920183F4C04600126046886600398C7
:10116000029E43406340384C7068634089EA000047
:10117000364C6040034438484340280018BF0120E3
:101180005B1E9B41042F2CBFC0B2D80F02F1140389
:1011900053F8200007F00303C3F10303DB00D8403A
:1011A0000DF807007F1C082F9DD315460C466A6971
:1011B000AB69E868D20842EA4372401E00EA0207BF
:1011C000002302409B420AD8524508D28020E055B5
:1011D0007F1C574516D2AAEB0701E01910E08020CA
:1011E000E05500E0E355E8687F1C8742FAD32A689F
:1011F000136828469847BAF1000F03D0514620469D
:101200002EF0FFFA2A68069E059F936869462846D5
:1012100098472A68D2F8009021462846C8472B688C
:10122000DA683946284690470EB1A86830604FF416
:10123000003007B0BDE8F08FEC6D03085C120008C9
:10124000640800205FC5109304850012FC68017AD1
:10125000C0F524FF24AF33D426AF698B04B001015D
:1012600000170145F8B501240094002300240DE087
:10127000009D065D0F5D7E40F643761CF60F86F0FE
:10128000010635400095641C009DEB189442EFD395
:101290001846F2BDF8B5002301240094002A11E09D
:1012A000009C85188F1815F8016C17F8015C6E40CA
:1012B000F643761CF60F86F0010634400094009C3D
:1012C000E318521EECD11846F2BD0000651200086A
:1012D00095120008010000002DE9F84F1D46DDF8C9
:1012E00028900B9F0D9C4FF0FF3300930E469246C3
:1012F000D9F800B0804632465146D847834664B399
:10130000D9F8043032465146404698476FEA0B02FE
:10131000521C42EA0B0200996FEAD2735B1C19401F
:10132000C2430091521C024300996FEAD2735B1CC6
:101330001940009186F05531484087EA000181F05C
:101340005531216080F05531C943491C0843009A4A
:101350006FEAD070401C82430092D9F8080001283F
:1013600009D17540E943491C0D4300986FEAD572D5
:10137000521C90430AE0F11C85EA9102D243521CB0
:10138000154300986FEAD5735B1C984386F0AA3624
:10139000009086EA0B0686F0AA33F243DB430C98F2
:1013A000C2F3C0725B1C42EAD3720099D243521C52
:1013B00091430091774000998843009987F0AA37BC
:1013C0000F403843BDE8F28F00000000000000002D
:1013D00001F0FF01102A2BDB10F0070F08D010F8E6
:1013E000013B013A8B422DD010F0070F42B3F6D1EA
:1013F000F0B441EA012141EA014122F007047FF003
:1014000000070023F0E80256083C85EA010586EA59
:10141000010685FA47F5A3FA87F586FA47F6A5FA95
:1014200087F68EB9EED1F0BC01F0FF0102F00702A1
:1014300032B110F8013B013A83EA010313B1F8D14C
:101440000020704701387047002D06BF354603382D
:10145000073815F0010F07D1013015F4807F02BF66
:10146000013015F4C03F0130F0BC0138704700BFB7
:10147000034613F8012B002AFBD1181A01387047D4
:1014800081F0004102E000BF83F0004330B54FEA35
:1014900041044FEA430594EA050F08BF90EA020FA2
:1014A0001FBF54EA000C55EA020C7FEA645C7FEA35
:1014B000655C00F0E2804FEA5454D4EB5555B8BF58
:1014C0006D420CDD2C4480EA020281EA030382EAC9
:1014D000000083EA010180EA020281EA0303362D5B
:1014E00088BF30BD11F0004F4FEA01314FF4801C2E
:1014F0004CEA113102D0404261EB410113F0004F40
:101500004FEA03334CEA133302D0524263EB4303F6
:1015100094EA050F00F0A780A4F10104D5F1200E94
:101520000DDB02FA0EFC22FA05F2801841F10001EF
:1015300003FA0EF2801843FA05F359410EE0A5F1C3
:1015400020050EF1200E012A03FA0EFC28BF4CF0F4
:10155000020C43FA05F3C01851EBE37101F00045AA
:1015600007D54FF0000EDCF1000C7EEB00006EEBB7
:101570000101B1F5801F1BD3B1F5001F0CD3490841
:101580005FEA30004FEA3C0C04F101044FEA445298
:1015900012F5800F80F09A80BCF1004F08BF5FEA1F
:1015A000500C50F1000041EB045141EA050130BDFF
:1015B0005FEA4C0C404141EB0101013C28BFB1F511
:1015C000801FE9D291F0000F04BF01460020B1FA5C
:1015D00081F308BF2033A3F10B03B3F120020CDA2F
:1015E0000C3208DD02F1140CC2F10C0201FA0CF00D
:1015F00021FA02F10CE002F11402D8BFC2F1200C72
:1016000001FA02F120FA0CFCDCBF41EA0C01904027
:10161000E41AA2BF01EB0451294330BD6FEA040470
:101620001F3C1CDA0C340EDC04F11404C4F120025B
:1016300020FA04F001FA02F340EA030021FA04F36D
:1016400045EA030130BDC4F10C04C4F1200220FAC4
:1016500002F001FA04F340EA0300294630BD21FA02
:1016600004F0294630BD94F0000F83F4801306BFC8
:1016700081F480110134013D4EE77FEA645C18BFBC
:101680007FEA655C29D094EA050F08BF90EA020F53
:1016900005D054EA000C04BF1946104630BD91EA4B
:1016A000030F1EBF0021002030BD5FEA545C05D14E
:1016B0004000494128BF41F0004130BD14F580048D
:1016C0003CBF01F5801130BD01F0004545F0FE4101
:1016D00041F470014FF0000030BD7FEA645C1ABF36
:1016E000194610467FEA655C1CBF0B46024650EA6D
:1016F000013406BF52EA033591EA030F41F4002199
:1017000030BD00BF90F0000F04BF0021704730B51E
:101710004FF4806404F132044FF000054FF00001F3
:1017200050E700BF90F0000F04BF0021704730B5B4
:101730004FF4806404F1320410F0004548BF404289
:101740004FF000013EE700BF42004FEAE2014FEADE
:1017500031014FEA02701FBF12F07F4393F07F4FB9
:1017600081F06051704732F07F4208BF704793F0BC
:101770007F4F04BF41F40021704730B54FF46074CF
:1017800001F0004521F000411CE700BF50EA0102D2
:1017900008BF704730B54FF000050AE050EA01027B
:1017A00008BF704730B511F0004502D5404261EBEB
:1017B00041014FF4806404F132045FEA915C3FF42C
:1017C000D8AE4FF003025FEADC0C18BF03325FEAC9
:1017D000DC0C18BF033202EBDC02C2F1200300FA7A
:1017E00003FC20FA02F001FA03FE40EA0E0021FA9F
:1017F00002F11444BDE600BF70B54FF0FF0C4CF48D
:10180000E06C1CEA11541DBF1CEA135594EA0C0F3E
:1018100095EA0C0F00F0DEF82C4481EA030621EA79
:101820004C5123EA4C5350EA013518BF52EA0335B4
:1018300041F4801143F4801338D0A0FB02CE4FF066
:101840000005E1FB02E506F00042E0FB03E54FF096
:101850000006E1FB03569CF0000F18BF4EF0010E8E
:10186000A4F1FF04B6F5007F64F5407404D25FEA8A
:101870004E0E6D4146EB060642EAC62141EA55513D
:101880004FEAC52040EA5E504FEACE2EB4F1FD0C7F
:1018900088BFBCF5E06F1ED8BEF1004F08BF5FEAFD
:1018A000500E50F1000041EB045170BD06F00046AF
:1018B00046EA010140EA020081EA0301B4EB5C045C
:1018C000C2BFD4EB0C0541EA045170BD41F4801154
:1018D0004FF0000E013C00F3AB8014F1360FDEBF79
:1018E000002001F0004170BDC4F10004203C35DA55
:1018F0000C341BDC04F11404C4F1200500FA05F3D8
:1019000020FA04F001FA05F240EA020001F0004278
:1019100021F0004110EBD37021FA04F642EB0601EE
:101920005EEA430E08BF20EAD37070BDC4F10C0418
:10193000C4F1200500FA04F320FA05F001FA04F2DC
:1019400040EA020001F0004110EBD37041F10001C8
:101950005EEA430E08BF20EAD37070BDC4F12005D3
:1019600000FA05F24EEA020E20FA04F301FA05F23B
:1019700043EA020321FA04F001F0004121FA04F2E3
:1019800020EA020000EBD3705EEA430E08BF20EAB3
:10199000D37070BD94F0000F0FD101F000464000ED
:1019A00041EB010111F4801F08BF013CF7D041EA6F
:1019B000060195F0000F18BF704703F00046520073
:1019C00043EB030313F4801F08BF013DF7D043EA44
:1019D0000603704794EA0C0F0CEA135518BF95EAFA
:1019E0000C0F0CD050EA410618BF52EA4306D1D181
:1019F00081EA030101F000414FF0000070BD50EAA0
:101A0000410606BF1046194652EA430619D094EA29
:101A10000C0F02D150EA013613D195EA0C0F05D113
:101A200052EA03361CBF104619460AD181EA030167
:101A300001F0004141F0FE4141F470014FF000001F
:101A400070BD41F0FE4141F4780170BD70B54FF0BA
:101A5000FF0C4CF4E06C1CEA11541DBF1CEA13553A
:101A600094EA0C0F95EA0C0F00F0A7F8A4EB05041C
:101A700081EA030E52EA03354FEA013100F0888013
:101A80004FEA03334FF0805545EA131343EA1263DC
:101A90004FEA022245EA111545EA10654FEA002691
:101AA0000EF000419D4208BF964244F1FD0404F54A
:101AB000407402D25B084FEA3202B61A65EB0305A6
:101AC0005B084FEA32024FF480104FF4002CB6EB63
:101AD000020E75EB030E22BFB61A754640EA0C00E3
:101AE0005B084FEA3202B6EB020E75EB030E22BF23
:101AF000B61A754640EA5C005B084FEA3202B6EB64
:101B0000020E75EB030E22BFB61A754640EA9C0022
:101B10005B084FEA3202B6EB020E75EB030E22BFF2
:101B2000B61A754640EADC0055EA060E18D04FEAB0
:101B3000051545EA16754FEA06164FEAC30343EA50
:101B400052734FEAC2025FEA1C1CC0D111F4801F1D
:101B50000BD141EA00014FF000004FF0004CB6E716
:101B600011F4801F04BF01430020B4F1FD0C88BFB5
:101B7000BCF5E06F3FF6AFAEB5EB030C04BFB6EBC0
:101B8000020C5FEA500C50F1000041EB045170BDB3
:101B90000EF0004E4EEA113114EB5C04C2BFD4EBE0
:101BA0000C0541EA045170BD41F480114FF0000E64
:101BB000013C90E645EA060E8DE60CEA135594EAE0
:101BC0000C0F08BF95EA0C0F3FF43BAF94EA0C0FE3
:101BD0000AD150EA01347FF434AF95EA0C0F7FF458
:101BE00025AF104619462CE795EA0C0F06D152EAAC
:101BF00003353FF4FDAE1046194622E750EA410690
:101C000018BF52EA43067FF4C5AE50EA41047FF4A0
:101C10000DAF52EA43057FF4EBAE12E74FF0FF3C05
:101C200006E000BF4FF0010C02E000BF4FF0010CD6
:101C30004DF804CD4FEA410C7FEA6C5C4FEA430C4F
:101C400018BF7FEA6C5C1BD001B050EA410C0CBF9E
:101C500052EA430C91EA030F02BF90EA020F002000
:101C6000704710F1000F91EA030F58BF994208BF67
:101C700090422CBFD8176FEAE37040F00100704724
:101C80004FEA410C7FEA6C5C02D150EA013C07D17B
:101C90004FEA430C7FEA6C5CD6D152EA033CD3D0C6
:101CA0005DF8040B704700BF8446104662468C46C0
:101CB0001946634600E000BF01B5FFF7B7FF0028F3
:101CC00048BF10F1000F01BD4DF808EDFFF7F4FF1C
:101CD0000CBF012000205DF808FB00BF4DF808EDA7
:101CE000FFF7EAFF34BF012000205DF808FB00BFCA
:101CF0004DF808EDFFF7E0FF94BF012000205DF8EC
:101D000008FB00BF4DF808EDFFF7CEFF94BF0120A0
:101D100000205DF808FB00BF4DF808EDFFF7C4FF99
:101D200034BF012000205DF808FB00BF4FEA410CE2
:101D30007FEA6C5C02D150EA013C0AD14FEA430CC5
:101D40007FEA6C5C02D152EA033C02D14FF0000002
:101D500070474FF0010070474FEA410212F5001240
:101D600015D211D56FF47873B3EB625212D94FEAE2
:101D7000C12343F0004343EA505311F0004F23FACC
:101D800002F018BF404270474FF00000704750EA21
:101D9000013005D111F0004008BF6FF000407047DE
:101DA0004FF00000704700BF4FEA4102B2F1E0433C
:101DB00024BFB3F5001CDCF1FE5C0DD901F0004C32
:101DC0004FEAC0024CEA5070B2F1004F40EB830082
:101DD00008BF20F00100704711F0804F21D113F1AE
:101DE0003872BCBF01F00040704741F480114FEAE7
:101DF0005252C2F11802C2F1200C10FA0CF320FA70
:101E000002F018BF40F001004FEAC1234FEAD3238C
:101E100003FA0CFC40EA0C0023FA02F34FEA4303F6
:101E2000CCE77FEA625307D150EA01331EBF4FF07F
:101E3000FE4040F44000704701F0004040F0FE409A
:101E400040F40000704700BF80F0004002E000BF97
:101E500081F0004142001FBF5FEA410392EA030F95
:101E60007FEA226C7FEA236C6AD04FEA1262D2EBDF
:101E70001363C1BFD218414048404140B8BF5B42E4
:101E8000192B88BF704710F0004F40F4000020F07D
:101E90007F4018BF404211F0004F41F4000121F093
:101EA0007F4118BF494292EA030F3FD0A2F10102DD
:101EB00041FA03FC10EB0C00C3F1200301FA03F11B
:101EC00000F0004302D5494260EB4000B0F5000F3E
:101ED00013D3B0F1807F06D340084FEA310102F1FD
:101EE0000102FE2A51D2B1F1004F40EBC25008BFAF
:101EF00020F0010040EA03007047490040EB000079
:101F0000013A28BFB0F5000FEDD2B0FA80FCACF179
:101F1000080CB2EB0C0200FA0CF0AABF00EBC250A6
:101F200052421843BCBFD0401843704792F0000F94
:101F300081F4000106BF80F400000132013BB5E7E7
:101F40004FEA41037FEA226C18BF7FEA236C21D05D
:101F500092EA030F04D092F0000F08BF08467047C2
:101F600090EA010F1CBF0020704712F07F4F04D190
:101F7000400028BF40F00040704712F100723CBFA3
:101F800000F50000704700F0004343F0FE4040F4CD
:101F9000000070477FEA226216BF08467FEA23638B
:101FA0000146420206BF5FEA412390EA010F40F476
:101FB000800070474FF0000304E000BF10F00043C2
:101FC00048BF40425FEA000C08BF704743F09643A9
:101FD00001464FF000001CE050EA010208BF7047C4
:101FE0004FF000030AE000BF50EA010208BF70474B
:101FF00011F0004302D5404261EB41015FEA010C60
:1020000002BF84460146002043F0B64308BFA3F157
:102010008053A3F50003BCFA8CF2083AA3EBC25339
:1020200010DB01FA02FC634400FA02FCC2F1200258
:10203000BCF1004F20FA02F243EB020008BF20F08F
:102040000100704702F1200201FA02FCC2F12002F5
:1020500050EA4C0021FA02F243EB020008BF20EAEA
:10206000DC7070474FF0FF0C1CEAD0521EBF1CEA18
:10207000D15392EA0C0F93EA0C0F6FD01A4480EA06
:10208000010C400218BF5FEA41211ED04FF00063EF
:1020900043EA501043EA5111A0FB01310CF000401B
:1020A000B1F5000F3EBF490041EAD3715B0040EA41
:1020B000010062F17F02FD2A1DD8B3F1004F40EB11
:1020C000C25008BF20F00100704790F0000F0CF0E4
:1020D000004C08BF49024CEA502040EA51207F3AA8
:1020E000C2BFD2F1FF0340EAC250704740F4000083
:1020F0004FF00003013A5DDC12F1190FDCBF00F074
:1021000000407047C2F10002410021FA02F1C2F121
:10211000200200FA02FC5FEA310040F1000053EABD
:102120004C0308BF20EADC70704792F0000F00F00B
:10213000004C02BF400010F4000F013AF9D040EA11
:102140000C0093F0000F01F0004C02BF490011F4A5
:10215000000F013BF9D041EA0C018FE70CEAD153A3
:1021600092EA0C0F18BF93EA0C0F0AD030F0004C23
:1021700018BF31F0004CD8D180EA010000F00040D7
:10218000704790F0000F17BF90F0004F084691F095
:10219000000F91F0004F14D092EA0C0F01D14202CF
:1021A0000FD193EA0C0F03D14B0218BF084608D198
:1021B00080EA010000F0004040F0FE4040F40000E2
:1021C000704740F0FE4040F4400070474FF0FF0C75
:1021D0001CEAD0521EBF1CEAD15392EA0C0F93EABC
:1021E0000C0F69D0A2EB030280EA010C49024FEA0E
:1021F000402037D04FF0805343EA111143EA1013C7
:102200000CF000408B4238BF5B0042F17D024FF47E
:10221000000C8B4224BF5B1A40EA0C00B3EB510F59
:1022200024BFA3EB510340EA5C00B3EB910F24BF42
:10223000A3EB910340EA9C00B3EBD10F24BFA3EBC7
:10224000D10340EADC001B0118BF5FEA1C1CE0D18F
:10225000FD2A3FF650AF8B4240EBC25008BF20F042
:10226000010070470CF0004C4CEA50207F32C2BF96
:10227000D2F1FF0340EAC250704740F400004FF033
:102280000003013A37E792F0000F00F0004C02BF64
:10229000400010F4000F013AF9D040EA0C0093F02E
:1022A000000F01F0004C02BF490011F4000F013B88
:1022B000F9D041EA0C0195E70CEAD15392EA0C0FF0
:1022C00008D142027FF47DAF93EA0C0F7FF470AF28
:1022D000084676E793EA0C0F04D14B023FF44CAF6B
:1022E00008466EE730F0004C18BF31F0004CCAD100
:1022F00030F000427FF45CAF31F000437FF43CAF3C
:102300005FE700BF4FF0FF3C06E000BF4FF0010C5D
:1023100002E000BF4FF0010C4DF804CD4FEA40023F
:102320004FEA41037FEA226C18BF7FEA236C11D089
:1023300001B052EA530C18BF90EA010F58BFB2EB3C
:10234000030088BFC81738BF6FEAE17018BF40F0BC
:10235000010070477FEA226C02D15FEA402C05D170
:102360007FEA236CE4D15FEA412CE1D05DF8040BF5
:10237000704700BF844608466146FFE70FB5FFF788
:10238000C9FF002848BF10F1000F0FBD4DF808ED40
:10239000FFF7F4FF0CBF012000205DF808FB00BF31
:1023A0004DF808EDFFF7EAFF34BF012000205DF88B
:1023B00008FB00BF4DF808EDFFF7E0FF94BF0120D8
:1023C00000205DF808FB00BF4DF808EDFFF7D2FFD5
:1023D00094BF012000205DF808FB00BF4DF808ED18
:1023E000FFF7C8FF34BF012000205DF808FB00BFE5
:1023F0004FEA40024FEA41037FEA226C02D15FEAD2
:10240000402C08D17FEA236C02D15FEA412C02D133
:102410004FF0000070474FF0010070474FEA400254
:10242000B2F1FE4F0FD34FF09E03B3EB12620DD902
:102430004FEA002343F0004310F0004F23FA02F06C
:1024400018BF404270474FF00000704712F1610F13
:1024500001D1420205D110F0004008BF6FF00040EA
:1024600070474FF00000704742000ED2B2F1FE4FAD
:102470000BD34FF09E03B3EB126209D44FEA002353
:1024800043F0004323FA02F070474FF0000070471A
:1024900012F1610F01D1420202D14FF0FF307047BB
:1024A0004FF00000704700BF53B94AB9002908BF78
:1024B00000281CBF4FF0FF314FF0FF3000F06AB929
:1024C000ADF1080C6DE904CE00F006F8DDF804E08B
:1024D000DDE9022304B070472DE9F047089D0C4662
:1024E000002B4ED194468C458646B2FA82F262D9D0
:1024F0004AB1C2F12003914020FA03F30CFA02FC26
:10250000194300FA02FE4FEA1C471FFA8CF6B1FB92
:10251000F7F44FEA1E4307FB141143EA014304FB9F
:1025200006F199420AD91CEB030304F1FF3080F055
:102530001281994240F20F81023C6344591A1FFAFA
:102540008EF3B1FBF7F007FB101143EA014300FBE8
:1025500006F69E420AD91CEB030300F1FF3180F01E
:10256000FC809E4240F2F980634402389B1B40EAA3
:10257000044000211DB1D3400022C5E90032BDE86E
:10258000F0878B4205D90DB1C5E90001002108464D
:10259000F5E7B3FA83F1002946D1A34202D3904272
:1025A000C0F0F080861A64EB03030120002DE6D012
:1025B000C5E90063E3E7002A40F09080A1EB0C043A
:1025C0004FEA1C481FFA8CF70121B4FBF8F64FEADA
:1025D0001E4308FB164443EA044307FB06F09842F7
:1025E00008D91CEB030306F1FF3402D2984200F233
:1025F000CD8026461C1A1FFA8EF3B4FBF8F008FBB8
:10260000104443EA044300FB07F79F4208D91CEB40
:10261000030300F1FF3402D29F4200F2B080204653
:10262000DB1B40EA0640A5E7C1F120068B4022FAF9
:1026300006F71F4320FA06FC04FA01F343EA0C03F1
:10264000F44000FA01F8380C4FEA1349B4FBF0FEED
:102650001FFA87FC00FB1E4449EA04440EFB0CF9F8
:10266000A14502FA01F20AD93C190EF1FF3A80F0B5
:102670008480A14540F28180AEF1020E3C44A4EB7F
:1026800009041FFA83F9B4FBF0F300FB134449EA91
:10269000044403FB0CFCA44507D93C1903F1FF30AB
:1026A00067D2A44565D9023B3C4443EA0E40A0FBF7
:1026B0000293A4EB0C049C42CE469C4651D34ED0D0
:1026C00055B1B8EB0E0364EB0C0404FA06F6CB40EC
:1026D0001E43CC40C5E90064002150E7C2F120034D
:1026E00020FA03F10CFA02FC24FA03F394400C43A1
:1026F0004FEA1C4800FA02FE1FFA8CF7B3FBF8F011
:1027000008FB1031230C43EA014300FB07F1994217
:1027100008D91CEB030300F1FF362CD299422AD9C9
:10272000023863445B1AA4B2B3FBF8F108FB11331F
:1027300044EA034401FB07F3A34208D91CEB040459
:1027400001F1FF3613D2A34211D902396444E41ACD
:1027500041EA004139E70446F0E6084606E7C84585
:10276000AED2B9EB020E63EB070C0138A8E7314695
:10277000EDE7034699E73046D4E7D6467FE7634462
:1027800002384DE70646234608460FE7023E6344FB
:1027900030E700BF704700BF00487047001BB74BD1
:1027A00070B50C4601F0EAF9104E05460821304696
:1027B00006F0E4F8012804D001F0E0F9431BA3423D
:1027C00007D30821094806F0D9F8431E584258415A
:1027D00070BD72B60821304606F0D0F8012800D04E
:1027E00030BF62B6BFF36F8FE0E700BF0004004860
:1027F00008B5002210214FF0904006F0C5F80548BA
:102800000022202106F0C0F8BDE80840022001F0B7
:10281000BDB900BF0004004810B50C4C01221021C6
:10282000204606F0B1F8052001F0B0F9204601225B
:10283000202106F0A9F84FF090400122102106F067
:10284000A3F8BDE81040022001F0A0B90004004840
:1028500070B54FF090400C46164610210022144DE2
:1028600006F092F800232B701248B3B2224621469C
:1028700007F07EFAD8B901F081F941F287360446B3
:102880002B783BB1BDE87040012210214FF0904001
:1028900006F07AB801F072F9031BB342F2D872B6AF
:1028A0002B7803B930BF62B6BFF36F8FE8E770BD16
:1028B00065080020C8090020014B01221A707047EA
:1028C0006508002000487047F86D030813B5114BE8
:1028D0000446186800909B88ADF804300120FFF78B
:1028E0009BFF062269460120FFF7B2FF0120FFF798
:1028F0007FFF9DF80430112B08D19DF80520122A86
:1029000004D101202370627002B010BD00231A466A
:102910001846F7E7C02C03080CB4F0B5ADB032ABE5
:1029200006AF53F8042B059305460E46384696210C
:102930002CF0B6FE9528C1BF42F62E63ADF8AA3042
:102940002E23ADF8AC3000F037F83C24042D4FF4C2
:102950007A7E1449B0FBFEFCB0FBF1F14EF6602329
:10296000B0FBF3F3B3FBF4F204FB1232BCFBF4F361
:1029700004FB13C30EFB1C049ABF0B48405D3F20B1
:10298000CDE90040CDE9026708482CF009FE084B6C
:102990001B6898682CF02EFD2DB0BDE8F04002B009
:1029A000704700BF80EE3600566E0308346E030891
:1029B0007006002001F0EAB801F0E0B81348144AAC
:1029C00008B54FF00043C0E9002304224261012210
:1029D0000023C2614FF480510722C0E90233C0E9ED
:1029E0000933C0E90C1203610383837680F8203039
:1029F00080F82C30826380F83C30C36404F016FF0A
:102A000018B1BDE8084000F099BB08BD6808002077
:102A1000002401400268084B9A4282B00AD14FF06C
:102A2000B0431A6E42F400721A661B6E03F4007310
:102A30000193019B02B07047002401400268054BDE
:102A40009A4201BF4FF0B042136E23F40073136635
:102A5000704700BF0024014030B585B00024054612
:102A6000CDE901440394FFF7A9FF144805F072FA79
:102A700008B100F063FB1148039401A9CDE90154AA
:102A800005F032F808B100F059FB0C4805F08CF95C
:102A900008B100F053FB4FF0FF31084804F0C6FFC7
:102AA000064805F039FA054805F01AF804460348C7
:102AB00005F0DCF9204605B030BD00BF68080020F5
:102AC000014B024A1A607047680800200024014048
:102AD00008B50948FFF7C0FF68B1084BB3F8AA3042
:102AE0004FF6FF72934216BF40F6E442044B534345
:102AF000B3FBF0F398B208BD002000B40075FF1FCF
:102B0000D8084C0013B50023ADF80630FFF7E0FFFE
:102B100004461948FFF7A0FF184BB3F8C820B3F8D4
:102B2000A8108A4204FB00F018D040F6E443B0FB42
:102B3000F3F364205B1A4343521A93FBF2F31E3300
:102B40001BB2ADF80630BDF806305BB21B02ADF823
:102B50000630BDF8060000B202B010BD4FF47A7224
:102B600040F6FF73B0FBF3F35343A3F53923A3F50A
:102B70000C6340F6C412E0E7001000B00075FF1FC0
:102B80004FF0B04382B09A6A22F480529A629A6CF3
:102B900042F480529A649B6C03F480530193019B2E
:102BA000002002B070474FF0B04307B59A6C42F076
:102BB00004029A649A6C02F004020192019A9A6CDF
:102BC00042F001029A649B6C002203F0010311465B
:102BD00000930B20009B05F05BFA0B2005F08AFAAE
:102BE000002211460C2005F053FA0C2005F082FA61
:102BF000002211460D2005F04BFA0D2005F07AFA5F
:102C0000002202210F2005F043FA0F2005F072FA8E
:102C100000221146102005F03BFA102005F06AFA58
:102C200000221146112005F033FA112003B05DF89F
:102C300004EB05F05FBA000008B505F09FFC10B189
:102C40006FF0040008BD064B9A6942F040429A6159
:102C50004CF2FA321A6105F0A3FC0028F2D0EFE73B
:102C600000400058F0B585B000230D46009306469D
:102C7000A8B3FFF7E1FF044670BB05F07FFC88BBFB
:102C80001A481B4A02230193D0F8E01506F1784355
:102C900002EA8121B3FBF1F701FB1733DB0A029350
:102CA000D0F8E00505F178410139314402EA80228B
:102CB000B1FBF2F002FB1011C3EBD12301336946E3
:102CC00001A8039305F0ECFC20B1022814BF6FF0BB
:102CD0000104012405F064FC204605B0F0BD6FF04E
:102CE0000504F9E76FF00404F6E700BF0070FF1F6A
:102CF00000FCFF03014B186000207047CC08002047
:102D00002DE9F04FB0F1006F89B006460F469046AE
:102D1000C0F0C080DFF89091644DD9F8E03505EA45
:102D2000832303F10063013B984200F2B380002942
:102D300000F0B38040EA02035B0740F0AE80FFF78B
:102D40007BFF044690BB05F019FC002840F0A880EA
:102D5000D9F8E015009705EA812106F17842B2FB27
:102D6000F1F301FB132208F17843013B3344B3FB39
:102D7000F1F001FB1033DB0A01334FEAD22AA3EB57
:102D8000D222012A039388BFC6F30A050AF58037C9
:102D9000C6F108038CBFC5F500654546FF02B34682
:102DA0000693039B9A4505D305F0FAFB204609B02C
:102DB000BDE8F08FA6F10803069A1A4495421CD884
:102DC000009B04950193CDF814B04FF00009059BCA
:102DD00009EB0301049B99453DD3009BAB442B4475
:102DE000A8EB0505B5F5006F009328BF4FF400650B
:102DF0000AF1010A07F50067D3E753F8081F5A687C
:102E0000B2F1FF3F08BFB1F1FF3FD5D0284B1868A2
:102E100010B96FF00504C7E727B14FF400623946D7
:102E200012F040FEDFF888900099D9F80030CBF31B
:102E30000A001844AAB212F035FE4FF40061384679
:102E4000FFF710FF00BBD9F8003001934FF4006387
:102E500005970493B9E7019B07914B440293012026
:102E6000D3E9002305F0D6FB88B90799019BD1E986
:102E7000000259F80310029B5B689A4208BF88421F
:102E800005D109F10809A2E76FF001048CE76FF0A2
:102E9000030489E74FF0FF3488E76FF0050485E706
:102EA0006FF0040482E700BF0070FF1F00FCFF0307
:102EB000CC080020B1F1006F70B510D30B4BD3F8E4
:102EC000E0650B4B03EA862303F10063013B994263
:102ED00005D838B192B212F0E5FD002070BD4FF078
:102EE000FF30FBE76FF00500F8E700BF0070FF1F41
:102EF00000FCFF03B0F1006F10B40DD3084BD3F802
:102F0000E045084B03EA842303F10063013B984248
:102F100002D810BCFFF7A6BE4FF0FF3010BC7047C0
:102F20000070FF1F00FCFF034FF0B04382B0DA6C6B
:102F30000243DA64DB6C03400193019B02B07047EB
:102F40002DE9F04186B01422002101A82CF0C6FB27
:102F50000220464EFFF7E8FF0420FFF7E5FF0120BF
:102F6000FFF7E2FF04213046002205F00DFD0022AC
:102F700010214FF0904005F007FD042300240125A7
:102F800002270DEB03013046CDE901354FF0100863
:102F9000CDE9034705F0D2FB01A93046CDE9018513
:102FA000CDE9037405F0CAFB202301A93046CDE921
:102FB0000135CDE9037405F0C1FB01A94FF0904044
:102FC000CDE90185CDE9034405F0B8FB08224FF4B3
:102FD000881301A93046CDE901234FF00308CDE95C
:102FE000034705F0ABFB4FF4441301A94FF09040A9
:102FF000CDE90183CDE9035705F0A0FB4FF4405321
:1030000001A93046CDE90135CDE9034805F096FB2D
:103010004FF404134021CDE901131548039501A98C
:1030200005F08CFB22460F21062005F031F8062022
:1030300005F060F822460F21072005F029F8072047
:1030400005F058F822462146092005F021F809200C
:1030500005F050F822462146092005F019F809200C
:1030600005F048F806B0BDE8F08100BF0004004854
:103070000008004800B59BB04822002108A82CF0A9
:103080002DFB1822002102A82CF028FB05F096FC4D
:103090004FF0B0420120D2F8903023F01803C2F86C
:1030A0009030D2F8003423F4C06343F40073C2F8C4
:1030B0000034D2F8003403F4C0630193019B24234D
:1030C000089381230B930023CDE91003B02208A8B5
:1030D000CDE9122305F0EAFD08B172B6FEE74F23F1
:1030E000CDE90230CDE90400CDE90600022102A8B5
:1030F00006F076F808B172B6FEE71BB05DF804FB87
:1031000008B504F041FBFFF7B5FFFFF719FFFFF724
:103110004AFD00F0D9FF00F06BFE00F089F8064888
:103120000122042105F030FC02F06CFC00F006FCEA
:1031300002F06FFCFCE700BF0004004872B6FEE737
:1031400000B58DB02C22002101A82CF0C7FA174839
:10315000174B03601F2383604FF080420023C0E9B8
:103160000433C0E9072383614FF48073436206F0A0
:10317000DDFA08B1FFF7E2FF0C4806F003FC08B1E6
:10318000FFF7DCFF4FF00053002207930748089237
:103190004FF4807301A9029206920B9306F026FB6E
:1031A00008B1FFF7CBFF0DB05DF804FBD00800209D
:1031B0000028004010B5044690B03822002102A833
:1031C0002CF08CFA2268194B9A422CD14FF48033A0
:1031D000029302A84FF480730F9306F025F908B10B
:1031E000FFF7ACFF4FF0B0430220D3F8902042F439
:1031F0000042C3F890209A6D42F480629A659B6DFC
:10320000002203F4806311460193019B04F040FF08
:10321000022004F06FFF00222A20114604F038FF3C
:103220002A2004F067FF10B010BD00BF0028004046
:103230001148124A08B54FF48273C0E900230023F5
:103240004FF4E062C0E902324FF400712822C0E975
:1032500006120722C0E90433C0E90833C0E90B2392
:1032600083620823436306F0FDFC18B1BDE8084003
:10327000FFF764BF08BD00BFC8090020003001404F
:10328000F0B5054689B01422002103A82CF026FAD7
:103290002A68374B9A4269D14FF0B04302261A6E22
:1032A00042F480521A661A6E02F480520292029A16
:1032B000DA6C42F00102DA64DA6C02F00102019287
:1032C000019ADA6C42F00202DA64DB6C03F002036A
:1032D00000930524009B0327D02303A94FF09040BF
:1032E000CDE90336CDE9067405F028FA2023CDE9AF
:1032F00003364FF09040002603A90794CDE90567F7
:103300001C4C05F01BFA1C4826620723C4E9000385
:1033100080232046C4E90266C4E90436C4E906668F
:1033200004F048FF08B1FFF709FF144AAC65A56235
:10333000134C0823C4E900231021002380222046D7
:10334000C4E90213C4E90423C4E90633236204F088
:1033500031FF08B1FFF7F2FE002222206C65114612
:10336000A56204F095FE222004F0C4FE09B0F0BD71
:1033700000300140680900201C000240300002407B
:10338000080900207047000008B504F013FA044B48
:103390000120C3F88800BDE8084005F067BB00BF06
:1033A0000004005808B504F00CFA00F09DFFFFF788
:1033B000C7FDFFF7F8FB00F01BFDBDE80840FFF775
:1033C00037BF08B504F0FDF9FFF7BAFDFFF7EBFBD7
:1033D000BDE80840FFF72CBF08B504F0EBF9BDE8E5
:1033E00008400121002005F0F1BA70477047FEE760
:1033F000FEE7FEE7FEE7FEE770477047704770475D
:10340000014806F0E5BA00BFD0080020024B0120B9
:10341000187005F0C7BA00BF1A1F0020024B012226
:1034200002201A7005F0BEBA191F0020082005F00E
:10343000B9BA0000014805F033B800BFD41300202A
:10344000014805F02DB800BF68090020014805F0CB
:1034500027B800BF0809002070470000014805F0A8
:103460001FB800BF8814002070470000014806F014
:103470006DBE00BFC8090020014807F0EBBF00BFC8
:10348000E8140020014806F0D7B800BFD00800209B
:10349000014807F0ECB800BFC01300202DE9F0434D
:1034A00089B080460020109E0790894615461F4629
:1034B000FCF7BEFEF0B9104CCDE90090CDE9020456
:1034C00007AB0E480593142304933A464346294616
:1034D0000068FCF777FF2346324604F1140153F8E5
:1034E000044B42F8044B8B42F9D1079B337509B06A
:1034F000BDE8F0830120FAE7420A0020E86D0308E6
:103500007FB5124C00253C2302A86375CDE9025516
:10351000257500F0DDFA042303AA009412210C485B
:10352000FFF7BCFF0B49142220462CF0C7F80646D3
:10353000B0FA80F040096075074B00902A46294692
:10354000022012F0A9F9304604B070BD2C0A002008
:10355000926E0308DE210020746E0308034A0448BB
:1035600040F21B53002107F0A5BD00BF560A002002
:1035700034140020312BF0B52DD81825102415FB5C
:103580000343194D00244FF0800C4CFA04F6A3F1CC
:103590001007314205EB470714BF4FF0240E4FF0E0
:1035A000140EA7F806E0A3F10807304205EB470721
:1035B00014BF4FF0240E4FF0140E0134324205EBCD
:1035C0004306A7F806E00CBF14272427082CF78031
:1035D00003F10103D9D1054B1B781BB9BDE8F040BD
:1035E000FFF7BCBFF0BD00BF560A0020841F0020BB
:1035F00010B500240022E3B2114610460134FFF753
:10360000B9FF322CF6D1BDE81040FFF7A7BF00008C
:1036100070B504460D46FFF7EBFF0F4B04EB440477
:1036200000261C44142000F0B1FAA27861782078BA
:1036300012FB05F211FB05F110FB05F0F3B2D2B25B
:10364000C9B2C0B20136FFF795FF322EEAD1BDE80C
:1036500070400A2000F09ABA080000202DE9F041DD
:1036600006460F462048904600214FF416622CF083
:1036700035F81E4A10254FF0800C2B4600244CFADA
:1036800004F1A3F110000F4202EB400014BF4FF011
:10369000240E4FF0140EA0F806E0A3F108000E422D
:1036A00002EB400014BF4FF0240E4FF0140E013413
:1036B00018EA010F02EB4301A0F806E00CBF14204A
:1036C0002420082CC88003F10103D8D11835B5F5A2
:1036D000986FD2D1064B1B781BB9BDE8F041FFF7BC
:1036E0003DBFBDE8F08100BF5C0A0020560A002003
:1036F000841F002000F00F000B4607281ED8DFE8CB
:1037000000F004070A0F1316191B0022114600E0EF
:103710000022104602E0002211461846FFF79EBF25
:103720000A4600210020F9E700220846F6E70A468B
:103730000021EEE70A46F5E70A46E7E77047000092
:10374000024B1878024B1978FFF7D4BF060000200F
:103750000000002070B468480378DBB20B2B12D84D
:10376000DFE813F00C00230027002D00340059007F
:103770008E00A300B300C200C200C2005F4B1B78E2
:10378000DBB25F4A13700378012B04D05D4B1B78CA
:10379000002B00F0AE805A4A002313705A4A13706F
:1037A0005A4A137070BCFFF723BF554B00221A70A2
:1037B000E9E7574A1278012A08BF0123E1E7554B90
:1037C0001A78002A7CD14E4B0122F0E7514A524B25
:1037D000117861B951490978012908D11C78012C67
:1037E000E1B204D1464B1970474B1970CBE7127800
:1037F000012A05D0494A127812B11A78002AC2D19A
:103800003F49414A02240C7014701B78002BBAD136
:1038100023230B70B6E73F4C394A25783E493A4B93
:1038200095B93E4D2D78012D0ED10E78012EF5B2B1
:103830000AD115701D703A4C2478052C1ED8DFE88B
:1038400004F01D1B19101B1B2478012C05D0334CD0
:10385000247814B10C78002CEDD1022414701C7063
:10386000E9E704241C701470097800298BD1232106
:103870001170BAE70224F5E72324F3E70124F1E706
:10388000244B1A7832B9224A1278012AD1B201D1D6
:103890001B4BAAE71B78012B04D01D4B1B78002B78
:1038A0007FF471AF164B022281E71A4B1A781AB9CE
:1038B0001C4A1278002A86D01B78012BF2D0194BB3
:1038C0001B78012B7FF45FAFECE7124B1A7822B91B
:1038D000154A1278042A3FF476AF1B78012BE1D009
:1038E000114B1B78052BEDE70F4B1A78042AF8D102
:1038F00069E770BC704700BF06010020040000208B
:1039000007000020841F0020060000200100002086
:10391000DD2100200B1F0020090100200A010020EA
:10392000921500200A1F0020091F0020024803688A
:103930000021596307F038BC34140020002270B510
:103940000F4B1146022011F0A7FF01240A2529463A
:1039500020461435FFF7CEFEEDB2322000F016F906
:103960006E2DF4D10134E4B2FFF742FE082CEDD104
:103970000022BDE87040034B1146022011F08CBFBD
:10398000A46E0308D76E0308054808B50823036032
:1039900006F08AFC18B1BDE80840FFF7CFBB08BDB0
:1039A000C01300204FF0B04307B55A6E42F0010239
:1039B0005A665B6E002203F0010301931146322028
:1039C000019B04F065FB322003B05DF804EB04F0CA
:1039D00091BB00000CB407B5054A05AB102101935B
:1039E00012F02CFC03B05DF804EB02B0704700BF8E
:1039F0000D6F030830B585B0044602A80D4612F0DD
:103A0000B5F9BDF90C30064A00931021029B2046FF
:103A1000FFF7E0FF2046FDF72BFD288005B030BD05
:103A20000D6F03084FF0B04210B5936823F40043C4
:103A3000936012F0B7FA104B01241C7000F0ACF840
:103A400011F0C0FE0D4811F0D7FE0D4B4FF40042AF
:103A50001A61022011F0D6FEFFF732F800F002F9E9
:103A600011F0CAFF2146204611F0E6FF214620460C
:103A7000BDE8104011F0CABFCC130020F539000892
:103A80000040005811F0EEBF08B5FFF721F840F6EE
:103A9000B83398420CD8B0F5E16F0BD3FE23A0F5F4
:103AA000E16058434FF49663B0FBF3F0C0B208BD39
:103AB000FE20FCE70020FAE77FB5684600F0B6F884
:103AC0000198FEF7ABFC00B207B05DF804FB000004
:103AD000194A38B5D2F88035591C044619D103F07B
:103AE00077FE054603F080FE054403F077FE2B0EBB
:103AF000E3712B0CA3712B0A6371030EE370C0F307
:103B00000742C0F307232571C0B2A2706370207012
:103B100038BD190AC3718171190C1B0E41710371F3
:103B2000D2F88435C370D2F88405C0F30722C0F3FD
:103B30000743000EE9E700BF0070FF1F38B5094BCF
:103B4000D3F8803503600133054609D103F040FE08
:103B5000044603F043FE444003F046FE44402C601C
:103B600038BD00BF0070FF1F0121022011F04EBFC1
:103B70000021022011F04ABF00207047024B187844
:103B800008B100F0DDB97047CC13002082B001907D
:103B9000019802B000F070BAF0B5224A224CD2F877
:103BA000903043F4804389B0C2F8903003F022FE95
:103BB00003F028FE03F02EFE012304930323069353
:103BC00000254FF0B04305950795DA6C42F00202EC
:103BD000DA64DA6C02F002020292029ADA6C42F0C3
:103BE0000202DA64DB6C03F0020301934FF48057A6
:103BF00003A92046019B03974FF4005604F09EFD55
:103C000003A92046039604F099FD2A46394620462A
:103C100004F0BAFE2A463146204604F0B5FE09B04B
:103C2000F0BD00BF000800580004004810B504466D
:103C3000FEF768FF074BA36040F30F20FEF7BEF9C5
:103C4000054B064A2360064B6060C4E9032300204D
:103C500010BD00BF0000484200007A440D093E003C
:103C6000AB030500002070470120704708B52BF01A
:103C700097FD162303604FF0FF3008BD08B52BF009
:103C80008FFD16230360FEE770B50D4614460E4601
:103C9000731B9C4201DC204670BDAFF3008006F828
:103CA000010BF5E730B5104600234FF06042834228
:103CB00000DB30BDD2F8804EE50707D5D2F8004EC4
:103CC000E40703D5CC5C156815B114700133EEE739
:103CD00000BFF8E74FF0FF3070474FF400534B60E0
:103CE0000020704701207047002070470B4A116880
:103CF00010B5034609B90A491160106809490A4C10
:103D00000344091B8B4206D92BF04AFD0C230360A8
:103D10004FF0FF3010BD1360FCE700BFD013002050
:103D200020420020000001200008000037B5184B99
:103D300002689A42054628D14FF0B043154C1A6EDE
:103D400042F400621A661B6E134A03F40063019387
:103D5000019B1723C4E90023102100238020C4E91C
:103D600002134FF48073C4E904034FF4806C2023E2
:103D7000C4E906C320464FF40053236204F01AFA44
:103D800008B1FFF7DBF96C62A56203B030BD00BF7C
:103D9000002C0140D41300200800024010B5044656
:103DA00086B01422002101A82BF098FC22680F4B4A
:103DB0009A4218D14FF0B04301A9DA6C42F00102E7
:103DC000DA64DB6C03F0010300930222009B4FF4E2
:103DD0008073CDE901324FF090400123CDE90332E9
:103DE000059304F0ABFC06B010BD00BF002C0140F1
:103DF00010B510229CB0002400210DEB02002BF026
:103E00006DFC1C22214608A8CDE9014403942BF047
:103E100065FC342221460FA82BF060FC2B482C4B6C
:103E20008460C0E900343B23C0E90334C0E90544A1
:103E300006F086FE08B1FFF781F94FF4805323485E
:103E4000049304A906F09AFF08B1FFF777F91F4819
:103E500006F0A6FE08B1FFF771F900241B48039491
:103E600001A9CDE9014407F0A1F908B1FFF766F90E
:103E7000602316480E94002208A9CDE90834CDE944
:103E80000A44CDE90C4406F0F3FE08B1FFF756F9F9
:103E900000234FF40052CDE914230C4813934FF044
:103EA00000720FA9CDE90F33CDE91133CDE91633F7
:103EB000CDE91823CDE91A3307F0A4F908B1FFF7CB
:103EC0003DF90248FFF76AFF1CB010BD3414002012
:103ED000002C0140014B1868704700BF801400207F
:103EE0000320704708B501464FF47A720023800220
:103EF000890DFEF7D9FA08BD4FF47A73A0FB0303CE
:103F0000800A40EA83507047034B98689A68904251
:103F1000FBD1C043704700BF0028004008B5FFF741
:103F2000F3FF014B186008BD8014002008B5FFF7AF
:103F3000EBFF024B1B68C01A08BD00BF80140020B5
:103F4000024B187808B1FFF7DFBF704784140020D8
:103F500010B5074B074C0122DA654FF480712046FB
:103F600005F030FB4FF0FF332363002010BD00BF8E
:103F700000280040D008002002460021014805F03A
:103F800038BD00BFD008002002460121014805F0DD
:103F900030BD00BFD008002010B58CB02C2200210D
:103FA000044601A82BF09AFBFFF7D2FF0C4B0D48FB
:103FB0001B681C440023089306934FF00053E4430E
:103FC000079301224FF4807301A902940B9305F02B
:103FD0000DFC08B1FFF7B2F800200CB010BD00BF17
:103FE00080140020D008002038B50546FFF78CFF6C
:103FF00002210446074805F003FDC4F309024FF40B
:104000007A71A2FB0121920AA30A2A8043EA805016
:1040100038BD00BFD00800200148002105F0F0BCE9
:10402000D00800200148012105F0EABCD00800209A
:10403000F8B50F4D2E78CEB90E4C4FF0FF372763F1
:10404000FFF77EF8FFF784FF4FF48071204605F0FC
:10405000B9FA2046276305F077FC32462046022154
:1040600005F0C7FCFFF75AFF01232B700020F8BDB5
:1040700084140020D0080020014610B54FF47A7255
:1040800000238002890DFEF70FFA0146FFF73CFF7F
:104090000446FFF739FF031B8B4200D310BD00BF5E
:1040A000F7E712F087B8000010B5064C0221204651
:1040B00005F0A6FC0221421C2046BDE8104005F098
:1040C00098BC00BFD00800201648174A08B54FF426
:1040D000E133C0E9002300230C22C0E90233C0E928
:1040E0000523C0E90733C0E90933036107F097FFEF
:1040F00008B1FFF723F80B48002108F008F908B1D0
:10410000FFF71CF80748002108F021F908B1FFF774
:1041100015F8044808F0DBF818B1BDE80840FFF7CF
:104120000DB808BDE81400200044004070B596B0FA
:1041300006461422002103A82BF0D0FA38220021D1
:1041400008A82BF0CBFA3268274B9A424AD10223B7
:10415000089308A84FF440230A9305F065F908B1C5
:10416000FEF7ECFF4FF0B04300259A6D1F4C42F470
:1041700000329A659A6D02F400320292029ADA6C69
:1041800042F00102DA64DB6C03F001030193019B4E
:104190000C220223CDE9032303A907234FF090400B
:1041A0000793CDE9055504F0C9FA11492562142396
:1041B000C4E900131023C4E9023520468023C4E972
:1041C0000435C4E9065503F0F5FF08B1FEF7B6FF64
:1041D0002520F46700220221A66203F059FF252062
:1041E00003F088FF16B070BD004400408814002022
:1041F0008000024002680C4B9A4210B5044612D16E
:104200004FF0B0420C21936D23F4003393654FF0CF
:10421000904004F03FFBE06F04F03EF8BDE8104032
:10422000252003F075BF10BD0044004008B50A46C4
:104230000146024807F072F8002008BDE81400208B
:1042400013B5114B114C18604FF40013009302ABDF
:1042500013E90600204607F0DEFF2368DA69D10380
:10426000FCD4DA695202FCD59A68084842F480020C
:104270009A6008F016F806490448012207F084FF06
:10428000002002B010BD00BF7C150020E814002003
:104290008415002008B5074B1860FEF784FCFFF773
:1042A00013FF054AD2F8803043F00063C2F8803033
:1042B000002008BD801500200008005808B54FF008
:1042C000B04308489A6B42F400329A639A6B22F426
:1042D00000329A63FFF78EFF112003F019FF0020D0
:1042E00008BD00BFE814002008B5074807F097FE96
:1042F00008B1FEF723FF054803F05CFF18B1BDE8E5
:104300000840FEF71BBF08BDE814002088140020F9
:104310000268044B9A4203D1034B00201B681847E4
:10432000704700BF004400408015002002680B4B1E
:104330009A4210B504460FD1094B1B682BB1D0F837
:10434000902012B907480121984720460549BDE849
:104350001040012207F018BF10BD00BF004400400C
:104360007C150020841500202DE9F04F9DB0FEF74C
:10437000A9FA14F0C7FB024640B90146644B02207B
:1043800011F08AFA01201DB0BDE8F08F012014F071
:1043900061FC13F05DF90446039040B90246014602
:1043A0005C4B022011F078FA14F020FCEAE75A4D39
:1043B000296813F09DFD6968204613F0B3FD297A42
:1043C000204613F0E3FD697A204613F013FE696975
:1043D000204613F09FFEE868FEF746F881B22046BB
:1043E00013F022FE2969204613F0EAFDA97A20463F
:1043F00013F0B2FD0221204613F064FE1021204686
:1044000013F0A2FE039813F0ABF90246049040B9F2
:104410000146424B022011F03FFA03A813F078F94D
:10442000C2E703A813F074F9049813F001FD0246E3
:1044300040B901463A4B022011F02EFA04A813F0BD
:10444000ADFAB1E7374EDFF8E0A0DFF8E0B00023C7
:1044500033604FF00208049805AB0A2208A913F054
:10446000D9FA054628BB02460146314B022011F01D
:1044700013FA30682C49FDF7F5FD4FF07C51FDF73C
:10448000F1FD3060049813F003FD044604A813F016
:1044900085FA14F0ABFB002C3FF474AF002D3FF411
:1044A00071AF0022234B1146032011F0F5F90020D3
:1044B00069E731680998FDF7CDFCBDF818903060C8
:1044C00000221D4BCDF800901146022011F0E4F9B6
:1044D00008AC0027BBB2994504F1080405D8B8F12F
:1044E000010FC6D04FF00108B5E754F8040C51464F
:1044F000FDF7B8FDFDF7B8FF019034F8083C0093D4
:1045000000225B461146022011F0C6F90137E1E7AF
:10451000686F0308806F030820000020B56F030850
:10452000DC6F03081C1F002000007A443F70030862
:1045300005700308567003082E70030830B5044652
:1045400085B0084614491546FDF78CFDFDF766FF5A
:10455000CCB1114902902846FDF784FDFDF75EFFBE
:104560000E4901902846FDF773FC0D49FDF72EFE1C
:10457000FDF77AFF002200900A4B1146032011F04C
:104580008BF905B030BD0090074B22462146032031
:1045900011F082F9F5E700BF00007A44CDCC4C3F22
:1045A000CDCCCC3E6F7003089C7003082DE9F04F12
:1045B000ADF2344D4FF4007200210CA82BF08EF8B0
:1045C0004FF4007200218CA8B34E2BF087F8002521
:1045D00037464FF000082C46B9682046FDF73AFCF4
:1045E000796804462846FDF735FC08F10408B8F55B
:1045F000007F054607F11007EED14FF070512046BD
:10460000FDF730FD4FF0705104462846FDF72AFDB6
:104610000025DFF8848207464FF00009AA46D8F843
:1046200008002146FDF714FC0146FDF71BFD01467D
:104630005046FDF70FFC39468246D8F80400FDF7D6
:1046400007FC0146FDF70EFD01462846FDF702FC7A
:1046500009F10409B9F5007F054608F11008DED11B
:104660004FF070515046FDF7FDFC4FF070510A902D
:104670002846FDF7F7FC82460A98FDF765F8874B58
:1046800000222CF0A1FFCDE904015046FDF75CF8B3
:10469000824B00222CF098FFFDF786FB0DF13009CC
:1046A0000546C84600234FF0000BB168B069069379
:1046B000FDF7CEFBFDF7B2FE0028B8BF4042FDF784
:1046C0007DFC48F8040B01465846FDF7C3FB069BEA
:1046D0000433B3F5FE7F834606F11006E5D1704939
:1046E000FDF774FD0DF13008064600234FF0000B76
:1046F000314658F8040B0693FDF7AAFB0146FDF777
:10470000B1FC069B01461846FDF7A4FB0BF1010B1B
:104710001FFA8BFBBBF17F0F0346E9D16049FDF720
:1047200055FDFDF711F85D4B00222CF04DFFCDE952
:1047300006010DF50C78C346002200234846D9F83F
:10474000001040680B930892FDF782FBFDF766FEB0
:104750000028B8BF4042FDF731FC089A4BF8040B23
:1047600001461046FDF776FB0B9B01339BB27E2B77
:1047700009F104090246E1D14A49FDF727FD4FF04E
:10478000000B81460023494658F8040B0893FDF7B7
:104790005FFB0146FDF766FC089B01461846FDF7E6
:1047A00059FB0BF1010B1FFA8BFBBBF17E0F03468C
:1047B000E9D13C49FDF70AFDFCF7C6FF374B002263
:1047C0002CF002FFCDE9080137492846FDF74AFCE5
:1047D000FDF724FE344902905046FDF743FCFDF7F7
:1047E0001DFE314901903846FDF73CFCFDF716FEF1
:1047F00000222E4B00901146022011F04DF82C4A59
:1048000013889BB2FA2B00F2D580108880B2FDF796
:10481000D5FB2946FDF7D8FD264F08B105233B708F
:10482000254B1A78254B1B889BB29A4280F08D80CD
:10483000234B1A78234B1B889BB29A4206D22249FB
:104840002046FDF7CBFD08B101233B701F4FDFF879
:1048500080A03B880A9A01339BB23B803B889BB285
:104860000A2B04BF00233B803B884FF01C0B9BB2FC
:104870000BFB03F3DDE904014AF803403B889BB2DC
:104880000BFB03A35A603B889BB20BFB03A8FDF70D
:104890008BFA3B881EE000BFAC1600200000E03F12
:1048A0000000FE420000FC4200007A44B27003089F
:1048B0003C00002092150020A70300208A1500204C
:1048C000A603002088150020CDCC4C3FAC1E002054
:1048D00094150020C8F808009BB20BFB03A34FF00F
:1048E0008641DD603D883046FDF7BCFBADB20BFB79
:1048F00005A528613D88DDE90601FDF755FA4FF071
:104900008641FDF7AFFBADB23B880BFB05A59BB223
:104910006861334D0BFB03AA2A788AF81820DDE979
:104920000801FDF741FA4FF08641FDF79BFBFDF7CB
:104930009BFD2C4BC0B218802B78012B05D1002297
:10494000294B1146022010F0A7FF284F244D3B7839
:10495000DFF89C80012B24D1DFF89890264EB9F81F
:104960000030B9F800204FF01C0A9BB292B20AFB4B
:1049700003F30AFB0262F0589168FDF76BFA2146D7
:10498000FDF72CFDC0B102232B702B78022BD8B27F
:1049900004D10022194B114610F07EFF2B78DBB2B8
:1049A0003B702B78DBB23B70C8F800400DF2344D01
:1049B000BDE8F08F12482CE7B9F80030D8F8009025
:1049C0009BB20AFB03662046B168FDF743FA4946ED
:1049D000FDF704FD10B103232B70E2E72870E0E738
:1049E0009215002086150020F8700308901500200D
:1049F0008C150020AC1E0020941500203D7103088A
:104A000000007A432DE9F04F9FB0FDF75BFF14F0F3
:104A100079F8024640B90146A84B032010F03CFF4C
:104A200001201FB0BDE8F08F012014F013F911F040
:104A300027FD04460D9040B902460146A04B0320D5
:104A400010F02AFF14F0D2F8EAE79E4F3B78012BD2
:104A5000DDB252D0022D6FD0002D39D1042112F0D9
:104A6000D5F80121204611F0FFFF9749204612F0AA
:104A70002FF89649204612F011F89549204611F07A
:104A8000BFFF9449204611F0D5FF0221204612F0C5
:104A9000F1F89149204612F0D3F8214606A812F009
:104AA00031F88E4A19928E4A1A924FF07C530022A6
:104AB00018A9204618931B921C921D9312F04EF8D1
:104AC0002946204612F06EF80321204612F084F8A1
:104AD0000D9800243C7011F069FD02460E900028EC
:104AE0006DD1804B0146032010F0D6FE0DA811F0C9
:104AF00035FD0EA811F0E8FDA4E77B4E294611F024
:104B0000B3FF7149204611F0E3FFB168204611F070
:104B100077FFF168204611F08DFF716A204611F091
:104B2000BDFFF16C204612F08BF8704B002211464D
:104B3000012010F0B1FECBE76B4D012111F094FF85
:104B4000E969204611F0C4FF696A204611F0A6FF0A
:104B5000A968204611F054FFE968204611F06AFF69
:104B6000A86CFDF781FC81B2204612F083F8E96C55
:104B7000204612F065F8214606A811F0C3FF2B6B02
:104B800018936B6B1993AB6B1A93EB6B1B932B6C9A
:104B90001C9318A96B6C1D93204611F0DFFFA86AC7
:104BA000FDF762FCC1B2204611F0FCFF286AFDF758
:104BB0005BFCC1B2204612F077F84D4BB6E711F01E
:104BC00019FE38B900224B4B1146032010F064FE49
:104BD000002026E71422214613A82AF07FFD002694
:104BE000DFF8EC80DFF81091DFF810A121253746BF
:104BF0000E980FA911F056FE0246002840F08A8058
:104C000001463F4B032010F047FEDFF8F8800E9876
:104C100011F010FEB8F8003000229BB2114600934C
:104C20000320394B10F038FE0D9D0121284611F06C
:104C30001BFF0421284611F0E9FF2349284611F003
:104C400047FF2249284611F029FF2149284611F043
:104C5000D7FE2049284611F0EDFE0221284612F029
:104C600009F81D49284611F0EBFF294606A811F066
:104C700049FF1A4A1992254A1B924FF07C534FF074
:104C80007E5218A928461C9218931A931D9311F06E
:104C900065FF0021284611F085FF0321284611F009
:104CA0009BFF0D990EA811F039FD0246002840F037
:104CB00084800146164B022016E700BF686F030888
:104CC00082710308181F0020000082429A99993FC0
:104CD000CDCC4C3F000020406666263F00002041BE
:104CE0000AD7233C04720308B01E0020A2710308F7
:104CF000D27103081F720308CDCCCC3EA403002060
:104D00003D720308AE1E002066720308CDCC4C3EF7
:104D10009B720308119A10999DF83C00FFF70EFC56
:104D20009DF83C30FBB1DDF844B038465946FDF7FC
:104D300091F8109907463046FDF78CF84146064633
:104D40005846FDF785F84946FDF740FAFDF78CFB1C
:104D50001EAB80B203EB4000013430F82C3C013331
:104D6000E4B220F82C3C9AF80030012B1ED1DFF879
:104D70002CB28B4ABBF8003011999BB202EB0313A3
:104D80009960BBF800309BB202EB0312109B53609A
:104D9000BBF800309BB25A1C92B2802BABF80020BB
:104DA00004D1FFF703FC0023ABF800300F20FDF720
:104DB00001FE013D7FF41CAF27E70E9811F01AFDAC
:104DC00000283FF4FFAE0DA811F0C8FBDFF8D4B106
:104DD0004FF021090E980FA911F064FD0546002837
:104DE00040F08680024601466F4B032010F054FDD0
:104DF000B8F80030DFF8B4919BB20022009311465E
:104E00006B4B032010F048FD012C94BF00230123BD
:104E100089F80030674B1B782BB999F80030012BCB
:104E200001D100F0D3FD99F80030DFF88CB10022F9
:104E3000CDE900431146614B032010F02DFD0DF12B
:104E40004C084FF0000A38F8022B3AB1CDE900A225
:104E500000225B461146012010F01EFD0AF1010AF6
:104E6000BAF10A0FEFD156493846FDF7FBF807466D
:104E70002046FDF7A3F8804601463846FDF7A6F91F
:104E80004F4907463046FDF7EDF84146FDF79EF9DC
:104E90004C4B1F604C4B002118608046FDF776FAA2
:104EA0000646A8B94223404699F80090CDE903434D
:104EB000FDF7B4FA02903846FDF7B0FA5FFA89F9C7
:104EC000CDE90090414B32463146032010F0E4FC1E
:104ED0000E9811F0AFFC04460EA811F0F5FB13F08C
:104EE00085FE002C3FF49CAD85F00100C0B298E532
:104EF000119A10999DF83C00FFF720FB9DF849306E
:104F0000002B43D19DF83C30FBB1DDF844A038467E
:104F10005146FCF79FFF109907463046FCF79AFF71
:104F20002B4906465046FCF793FF5946FDF74EF9CC
:104F3000FDF79AFA1EAB80B203EB4000013430F863
:104F40002C3C0133E4B220F82C3C224B1B78012B83
:104F50001CD1B8F80030124A11999BB202EB03132E
:104F60009960B8F800309BB202EB0312109B5360BB
:104F7000B8F800309BB25A1C92B2802BA8F80020DF
:104F800004D1FFF713FB0023A8F800300F20FDF732
:104F900011FDB9F101097FF41DAF29E7AE1E002014
:104FA000AC160020CDCCCC3E3D7203080B1F002078
:104FB000BB720308081F00201A730308E672030877
:104FC00000007A44041F0020001F00203A730308E9
:104FD000CDCC4C3FA40300202DE9F043ADB0142309
:104FE0000DF10E0204A9ADF80E3014F013F80446CA
:104FF00048B902460146194B032010F04DFC2046EB
:105000002DB0BDE8F0830022154B164FDFF8588015
:10501000DFF858901146032010F03EFC0025BDF843
:105020000E30AAB29342EAD9AAB22CAB03EBC20269
:10503000032012F89C6C52F8A03C002E14BF3A4694
:105040004246CDE9003200224B46114610F024FCC6
:10505000002E05F1010508BF3446E0E7947303080C
:10506000B77303088A7303088F730308DB7303089D
:1050700030B5102289B00025294604460DEB020008
:1050800003952AF02BFB15F06FFB2A46A34B0090EB
:105090002946032010F000FCFDF714FC13F032FD4C
:1050A0008DF80C0013F0D8FD431B18BF012301211C
:1050B0008DF80D30029013F0EDFD029813F08CFF87
:1050C000029813F001FE0298FFF786FF002840F0D7
:1050D000008102A813F0D0FD13F088FD029813F0B0
:1050E0000FFE029813F028FE0298FFF775FF0028C4
:1050F00040F0F38002A813F0BFFD13F077FD029893
:1051000013F036FE0022864B1146032010F0C4FB3C
:10511000029813F049FE0298FFF75EFF002840F066
:10512000E08002A813F0A8FD13F060FD029813F0D0
:1051300057FE002211467B4B032010F0ADFB0022EE
:10514000794B1146032010F0A7FB029813F0D4FE10
:105150000298FFF741FF002840F0C78002A813F033
:105160008BFD13F043FD029813F0E2FE002211467E
:105170006E4B032010F090FB00226D4B1146032074
:1051800010F08AFB029813F0EFFE0298FFF724FF5D
:10519000002840F0AE8002A813F06EFD13F026FD4B
:1051A000029813F0FDFE00221146624B032010F01E
:1051B00073FB0022604B1146032010F06DFB029838
:1051C00013F02AFE0298FFF707FF002840F09580B1
:1051D00002A813F051FD13F009FD029813F038FEF8
:1051E00000221146554B032010F056FB0022544B71
:1051F0001146032010F050FB029813F045FE029870
:10520000FFF7EAFE00287CD102A813F035FD13F069
:10521000EDFC029813F054FE00221146494B032086
:1052200010F03AFB0022404B1146032010F034FBF3
:10523000029813F061FE0298FFF7CEFE002864D1B9
:1052400002A813F019FD13F0D1FC029813F070FEC0
:1052500000221146354B032010F01EFB0022344B78
:105260001146032010F018FB029813F07DFE0298FF
:10527000FFF7B2FE00284CD102A813F0FDFC13F09A
:10528000B5FC029813F08CFE00221146294B032036
:1052900010F002FB002211462B4B032010F0FCFA09
:1052A00001238DF8173003AB03CB00222060186870
:1052B00061600C23A060114600930320234B10F083
:1052C000EBFA02A813F0D8FC13F090FC002009B010
:1052D00030BD01238DF80E3000E701238DF80F302B
:1052E0000DE701238DF8103020E701238DF81130F0
:1052F00039E701238DF8123052E701238DF813307E
:105300006BE701238DF8143083E701238DF8153006
:105310009BE701238DF81630B3E700BFF173030854
:105320001A7403084D7403087E740308AD740308EF
:10533000DA7403080F7503084275030875750308CE
:10534000A6750308D67503080476030831760308AA
:1053500002480122102103F017BB00BF00040048DF
:1053600002480022102103F00FBB00BF00040048D8
:1053700013B5134C23785BB9E37C03F0FF023BB910
:10538000104B1146022002B0BDE8104010F084BA64
:10539000FEF7B6F800380C4B18BF0120400018701B
:1053A0001A78022A02BF00222270E2741B7800934E
:1053B0000022064B1146032010F06EFA02B010BD19
:1053C000DE21002050760308841F00206C7603083D
:1053D00038B5184C23785BBBE37C03F0FF023BBB82
:1053E000154D2B68012B0CD92B68042B09D81146BD
:1053F000124B022010F050FA114A0421012000F053
:10540000DBFF2B68042B13D900220E4B1146022020
:1054100010F042FAFEF774F800380B4B18BF012069
:10542000400018701B78022B02BF00232370E37426
:1054300038BD00BFDE210020801F002083760308D6
:10544000A8760308AD760308841F002010B5124C1F
:10545000237863B101214FF0904003F08FFA0F4B96
:105460000022187022701B780D4ADBB213700D4CAD
:10547000237863B102214FF0904003F07FFA0A4B8A
:105480000022187022701B78084ADBB21370BDE846
:105490001040FEF75FB900BF1A1F00200A0100206C
:1054A00008010020191F0020090100200701002029
:1054B00010B5164B1A78022A26D91B78082B23D848
:1054C000FFF7A0FA1248134A037811785B1A1249C1
:1054D00018BF01230B7003781048DBB21370104B18
:1054E000104A1C780378E31A18BF012313700E4B7F
:1054F00004701B7823B100230B700C490B701370E0
:10550000BDE81040FEF726B910BD00BF060100201F
:105510000B1F0020081F00200C1F002090150020EA
:105520009215002091150020841F00200D1F0020DF
:1055300008B501214FF0904003F020FA064B0128F6
:1055400016BF022218701A701878044B1978BDE83B
:105550000840FEF75DB800BF0600002000000020F4
:1055600038B5324D324C287BFCF724FD3149FCF72D
:1055700079FDA060687BFCF71DFD2E49FCF772FDEC
:10558000E060A87BFCF716FD2A49FCF76BFD606222
:10559000E87BFCF70FFD2849FCF764FD274BE0642E
:1055A0002361287CFCF706FD6060687CFCF702FD47
:1055B000A061A87CFCF7FEFCE061E87CFCF7FAFC4B
:1055C0002062287DFCF7F6FCA062687DFCF7F6FC03
:1055D0001849FCF747FD2063A87DFCF7EBFC6063EE
:1055E000E87DFCF7EBFC1449FCF73CFDA063287E4A
:1055F000FCF7E0FCE063687EFCF7E0FC0D49FCF79B
:1056000031FD2064A87EFCF7D9FC0A49FCF72AFD8D
:105610006064E87EFCF7CEFCA064287FFCF7CAFC3F
:10562000074BE06202221A7038BD00BF5803002009
:10563000B01E0020CDCCCC3D0AD7233CCDCCCC3EF7
:10564000181F002038B5114D114C287BFCF7B6FC13
:105650001049FCF707FDA060687BFCF7AFFC0D4923
:10566000FCF700FDE060A87BFCF7A8FC0949FCF70B
:10567000F9FC6062E87BFCF7A1FC0749FCF7F2FC4F
:10568000064BE06401221A7038BD00BF58030020A9
:10569000B01E0020CDCCCC3D0AD7233C181F0020E3
:1056A00073B52F4D2F4E2B7803702F4B1B78437003
:1056B000044601214FF0904003F060F93378A07068
:1056C000E37002214FF0904003F058F9274B20710E
:1056D0001B7863713378012B3ED1254B1868FCF79A
:1056E000C3FE244BE0801868FCF7BEFE80B2224B5C
:1056F000A0831B78191F4A424A41A2771F4A92F899
:105700002B1084F82B10D26AE262012B84F8283027
:105710000FD11B4B009300221A4B1146022010F0B0
:10572000BBF8194B1B8884F82930184B1B8884F868
:105730002A30174B1B7853B1164B1B683BB1164BE5
:105740001B78012B01BF154A232313702B70144BB8
:1057500001221A7002B070BD0020E080C7E700BFD0
:10576000060000200B1F0020060100200A1F002059
:10577000041F0020001F002092150020201F002081
:1057800052000020E07603088A15002086150020CC
:10579000A5030020141F0020DB21002007000020AB
:1057A0007C1F0020024B01220021032010F074B85E
:1057B0000E77030808B50122074B0021032010F0E3
:1057C0006BF8FFF7C5FDFFF7CBFE044A002313700B
:1057D000034A137008BD00BF54770308181F002048
:1057E000D921002010B5144B01220021022010F015
:1057F00053F8124B1A78124BD2B25A70002401227D
:1058000063211A7083F8331083F834209C63DC63BF
:105810001C645C649C64DC641C655C6583F82B40E0
:10582000DC625C629C77FFF793FDFFF7BBFFFFF73D
:10583000C1FF044B1C7010BD8A77030806010020CD
:10584000201F0020D92100201FB5114B11491C68D1
:1058500058681A7A5B7ACDE90223FCF703FCFCF75F
:1058600003FE0C4901902046FCF7FCFBFCF7FCFD15
:105870000022094B00901146032010F00DF8FEF7AE
:1058800073FD642004B0BDE81040FEF77FB900BF8F
:105890002000002000007A44C17703082DE9F04180
:1058A00086B00D460446FFF753FD01F06DFFFDF78E
:1058B00047FB9620FEF76AF9154F00264FF00508C2
:1058C000AE420FD14FF47A70FEF760F901AB03CB13
:1058D0001B8823810F4B2060002261601A7006B084
:1058E000BDE8F081FEF72AF887F80080FDF728FF71
:1058F0004FF47A70FEF74AF901A8FFF7B9FB41F2BD
:105900008830FEF743F90136FFF79EFFD8E700BF66
:1059100006000020D921002030B585B004460025BE
:1059200003A8ADF80C50FCF7D1FF70B19DF80C3016
:105930009DF80D20237062702946CDE900320320C6
:10594000034B2A460FF0A8FF012005B030BD00BF71
:10595000F6770308022801D8FFF7FABC704702283F
:1059600001D8FFF7FDBC7047022803D80248102178
:1059700003F00FB8704700BF0004004807B5684641
:1059800010F01AFA054B1B7803F0FF021BB9044B09
:1059900000999963DA6303B05DF804FB030000200B
:1059A000201F002007B5684610F006FA054B1B784B
:1059B00003F0FF021BB9044B009919645A6403B049
:1059C0005DF804FB02000020201F002007B5684698
:1059D00010F0F2F90849009B0A689A1A022A08D9BD
:1059E000064A1278012A01BF054A00209364D06458
:1059F0000B6003B05DF804FB101F00200B1F00209C
:105A0000201F002008B5FEF70DF8BDE8084000F0A3
:105A100027BF4FF0FF3010F089B87047014B0122CB
:105A20001A707047E81F0020014BD870704700BF04
:105A300018010020014B1874704700BF18010020A6
:105A400007B5064B00221B5C00931146044B022055
:105A50000FF022FF03B05DF804FB00BF35780308A8
:105A60001B7803080021012010F028B813B5104A54
:105A7000104C42F21073002818BF03460E482360F2
:105A8000136010F0F7FA21680B4810F07BFB0A480E
:105A900010F03EFB23684FF47A72B3FBF2F300225E
:105AA00000931146054B02200FF0F6FE02B010BD28
:105AB0009C030020140100204021002039780308B5
:105AC00013B50D4C206023680BB90C4B23600C48B8
:105AD00010F0D0FA21680A4810F054FB084810F082
:105AE00017FB236800930022064B114602200FF09B
:105AF000D3FE02B010BD00BF9C030020A0860100B1
:105B0000881F00206578030813B50F4C20602368B8
:105B100013B942F2107323600C4810F0ABFA2168FD
:105B20000A4810F02FFB094810F0F2FA23684FF4EE
:105B30007A72B3FBF2F3002200931146044B01206A
:105B40000FF0AAFE02B010BDA0030020A01F00208D
:105B5000A178030837B5044600283DD090F90650D7
:105B6000002D51D12C4810F085FAFDF741FD2B4B4B
:105B700001221A70FDF7F2FC2A462946284B022022
:105B80000FF08AFEE379012B0CBF264B264B2A46E9
:105B900029460220254D0FF07FFEE3792B70244B20
:105BA0001868FFF78DFF2978224A234B012908BF87
:105BB0001346002200931146204B01200FF06CFE8B
:105BC00094F90530019394F90430009300221C4BA2
:105BD000114603200FF060FE1A4810F099FA4FF4B6
:105BE000FA60FDF7D3FF184B0122002102201A7042
:105BF0000FF064FF4FF4FA60FDF7C8FF134803B0DD
:105C0000BDE8304010F084BA0022114B114602204A
:105C10000FF042FED4E700BFEC1F0020060000207A
:105C2000E3780308F878030815790308DA210020DF
:105C30009C030020DA780308DE7803083279030831
:105C40006A790308D01F0020D8210020A01F00205F
:105C5000517903080A460149FDF72CB900F0030801
:105C600070B5164810F006FA06F0D2FF044650B19F
:105C70000022134B114602200FF00EFEBDE87040CB
:105C8000104810F045BA104D104B02460146022054
:105C90000FF002FE01260E4B2E70224621460220F6
:105CA0000FF0FAFD0B4806F047FE2878314606F063
:105CB0009BFB024810F02CFAE0E700BF40210020D7
:105CC00093790308282100207C010020B179030882
:105CD000C57903081801002070B5A2B0FDF7D4FE05
:105CE000054606F07BFC0646002846D1824C0BA8F0
:105CF000FFF7D6FC13232370804B1A7802F0FF01C4
:105D0000002A3CD01E70142323707D4B62681B78E0
:105D100063F07F03137028B2636800EB400000EB70
:105D20004010FE220225B0FBF2F05870754B1B7834
:105D3000012B88BF00256570734C237823B907F0C9
:105D400089F908B901232370704C637A33B106F0E6
:105D500031FC012802D1204610F08CF96C4B6648CA
:105D6000D978002206F050FC0146002840F0AF80B0
:105D70000122684B10460FF08FFD22B070BD664BBC
:105D80001A7802F0FF05002AD0D019705C4B6268C7
:105D90001B78624E63F07F03137063689DF82C10CC
:105DA000597062689DF82D3093703278042A45D17D
:105DB00062689DF82E00D07062689DF82F00107107
:105DC00062689DF8300050710625554A03EB830345
:105DD00003EB830313440193524A01F00F0303EBD7
:105DE000830302EB43030022009311464E4B012034
:105DF0000FF052FD3378052B55D19DF854300893A0
:105E0000149B07939DF84A300693BDF848300593DC
:105E1000BDF8323004939DF8313003939DF8303053
:105E200002939DF82F30019300229DF82E300093AD
:105E300011463E4B01200FF02FFD77E73278052AFF
:105E40002FD162689DF82E00D07062689DF82F00F7
:105E5000107162689DF83000507162689DF83100E1
:105E60009071BDF832206068120AC2716268BDF894
:105E700032001072BDF84800000A5072BDF84800A8
:105E800090729DF84A00D0729DF8540010739DF8EE
:105E9000570050731698000A90731698D073102507
:105EA00093E7032591E73378042B7FF43FAF9DF808
:105EB000303002939DF82F30019300229DF82E3050
:105EC000009311461A4B01200FF0E6FC2EE7063135
:105ED0007FF453AF06F068FB00283FF44EAF012279
:105EE0004FF47A730021B0FBF3F0124B0090104690
:105EF0000FF0D2FC41E700BF0C010020D8210020A8
:105F000034200020841F0020E81F0020EC1F002008
:105F100018010020877B03087C1F00200601002059
:105F20007D010020F4020020E47903080C7A0308C4
:105F3000197B0308967B030813B568460FF03CFFF6
:105F40001A4B009A19781A4B11B9996B511AD963E7
:105F50001849DC6B0878844281BF012083F82B004C
:105F6000D86BD8621448007810B9186C101A5864AD
:105F70005C6C0878844281BF012083F82B00586C48
:105F8000D8620E480078012802BF986C121ADA64B1
:105F9000D86C0A78904205D9012283F83220DA6C55
:105FA00092B21A86064B1B7802B010BD0300002087
:105FB000201F0020A5030020020000200B1F00204E
:105FC0009215002000B503468DB000282CD04078F3
:105FD00002280AD003282AD0164B0022114602209C
:105FE0000DB05DF804EB0FF057BC1A7F0B92DA7E10
:105FF0000A929A7E09925A7E08921A7E0792DA7D58
:1060000006929A7D05925A680492DA68039293F98F
:1060100014200292B3F9122001921B7C00930022FB
:10602000054B11460FF038FC0DB05DF804FB034B37
:10603000D3E700BFB47B0308CB7B03083D7C030898
:1060400001284FF000020CBF024B034B1146022007
:106050000FF022BC5C7C03086E7C03081FB504466D
:10606000002831D00378002B2ED01D4810F050F8B6
:10607000002211461B4B02200FF00EFC94F9183041
:10608000039394F90A300293237C0193E36800930D
:1060900000221146144B03200FF0FEFB0022134B8D
:1060A000114603200FF0F8FB237A012B0ED1617A01
:1060B0000F4A104B002918BF1346002200931146C7
:1060C0000D4B03200FF0E8FB04B010BD00220B4B7A
:1060D0001146032004B0BDE810400FF0DDBB00BF47
:1060E0001C200020877C0308B87C0308E97C030897
:1060F000837C0308827C0308F67C0308077D030881
:1061000008B5104B0122002102201A700FF0D6FCB6
:106110000D480FF0FDFF0D4B1B788BB10C4B1A781F
:1061200072B9DB7C63B90B4B1A68042A9EBF1A68EC
:1061300001321A600021BDE8084010200FF0BEBCFB
:1061400008BD00BFD8210020881F0020DA210020D0
:10615000DE210020801F002013B50E4C00214020BE
:106160000FF0ACFC2378009300220B4B1146022069
:106170000FF092FB094B1B7853B12378012B07D109
:1061800000210220217002B0BDE810400FF096BC43
:1061900002B010BD0C1F0020157D0308DA2100207D
:1061A000044B1B78022B03D1002108200FF086BC82
:1061B000704700BF7C010020044B1B78012B03D0EB
:1061C000002180200FF07ABC704700BF060100203C
:1061D00008B506F026FD80B906F0ECF901280CD1CF
:1061E000BFF34F8F0549064BCA6802F4E0621343C0
:1061F000CB60BFF34F8F00BFFDE708BD00ED00E0AF
:106200000400FA0538B504460D4607484FF400610E
:10621000FCF770FE30B92A4621460348BDE83840F5
:10622000FCF76EBD38BD00BF00F0030810B506F0E6
:10623000A3FD10F1080F07D1064B0022BDE8104066
:10624000114602200FF028BB013001D1024BF4E7C8
:1062500010BD00BF3D7D0308537D030838B5104CC9
:10626000237822781809D2B20CD10E4D2A782378DF
:106270009A4206D020781E21FDF73CFA2378DBB243
:106280002B7038BD084C23781E2133B1FDF732FA4C
:10629000237883F001032370F3E702F00F00F5E7A2
:1062A00006000020DC210020980300207047000039
:1062B000022873B5044635D0402865D001282FD177
:1062C000334E337863B34FF4E170FDF75FFC214642
:1062D0004FF0904002F052FB2E4B214618704FF0C9
:1062E000904002F04BFB214605464FF0904002F0F3
:1062F00045FB294A294B002808BF134600221146B6
:10630000CDE900530220264B0FF0C6FAFFF736FB0B
:10631000FFF79CF8002102200FF0D0FB0023337020
:1063200002B070BD1F4B1B78002BF9D04FF4E17009
:10633000FDF72CFC21464FF0904002F01FFB1A4B5A
:10634000214618704FF0904002F018FB2146054698
:106350004FF0904002F012FB144A154B002808BF82
:10636000134600221146CDE900532046114B0FF091
:1063700093FAFFF717FBFFF769F80021204602B0F8
:10638000BDE870400FF09ABB00210420F7E700BF82
:106390001A1F0020030000206B7D0308777D03088F
:1063A0009D7D0308191F002002000020837D030843
:1063B000907D0308C37D030873B505460C46164659
:1063C00006F00CF90346002832D002B070BD4A68CE
:1063D000F05CD0540133DAB2A242F8D31E4B0D70F8
:1063E0001A781B78012A88BF00244C700022CDE95E
:1063F00000341A4C1A4B114601200FF04DFA637A03
:1064000033B106F0D7F8012802D120460FF032FE52
:10641000144B1548D978002206F0F6F8014648B921
:10642000124B0122032002B0BDE870400FF034BAD5
:106430000D49D0E70631C8D106F0B6F80028C4D01F
:106440004FF47A730122B0FBF3F000210090084B67
:1064500003200FF021FAB8E7841F0020EC1F002072
:10646000E87D0308180100200C010020877B030849
:10647000967B0308044B1B7823B9044A05210120AD
:10648000FFF79ABF704700BF841F0020197E0308E2
:1064900010B5002490B03C22214601A8009429F0B8
:1064A0001DF9454B2022DA7219788DF800105978C1
:1064B0008DF8011099788DF80210D9788DF80310B5
:1064C00019798DF8041059798DF8051099798DF89E
:1064D0000610D9798DF80710197A8DF80810597AB5
:1064E0008DF80910997A8DF80A108DF80B20214645
:1064F0000DF10B0258180131007B02F8010F14292D
:10650000F8D193F820208DF8202093F821208DF8E1
:10651000212093F822208DF8222093F823208DF853
:10652000232093F824208DF8242093F825208DF83B
:10653000252093F826208DF8262093F827208DF823
:10654000272093F828208DF8282093F829208DF80B
:10655000292093F82A208DF82A2093F82B2093F8ED
:1065600028108DF82B20154A19BB93F8291001F03B
:10657000FF00F1B9107093F82C206AB193F83F2016
:1065800052B10DF12B0100229818013290F82C0025
:1065900001F8010F142AF7D109484FF40061FCF704
:1065A000A9FC20B9064840226946FCF7A9FB10B0B7
:1065B00010BD01211170DEE758030020A403002064
:1065C00000F8030810B5002204461146054B0220CE
:1065D0000FF062F920460449BDE8104040220FF058
:1065E00061BA00BF1F7E030800F8030838B5454CA8
:1065F000207963794D2BC0B26AD1C0EB00108000C6
:10660000A379E2790A2838BF0A204D2ADBB267D184
:10661000C3EB03139B004FF47A7202FB03F594F86B
:106620002C30002B64D194F83F30002B60D142F223
:106630001070FFF71BFA344B1868FFF741FA237A02
:1066400032493348DBB20B70324B01221A70637A45
:10665000DBB2037094F827302F48DBB203700B785D
:106660002E49052B2E4B18BF00221A7094F82830A3
:106670002C4A03EB83035B00DBB2137094F82930E0
:10668000294A03EB83035B00DBB2137094F82A30D2
:10669000264A0133DBB2DB01138094F82B30244A05
:1066A00003EB83035B00DBB213700023E21892F864
:1066B0002C20D2B2CA540133142BF7D1A378012B6A
:1066C0001FD1E37A202B1CD1BDE83840FFF78AB8F0
:1066D0006379482B0ABF4FF46163637958438FE7AE
:1066E000E279482A0ABF4FF46162E279534392E7A4
:1066F0004FF47A735843FFF7E3F92846FFF704FA9B
:106700009DE738BD580300209C03002006010020AF
:10671000841F00200600002005000020DE2100204C
:10672000A4030020A7030020A60300203C000020B3
:10673000A503002010B590B000213C2201A80091D3
:1067400028F0CCFF4022434968460FF0ABF99DF892
:1067500000203AB99DF80100072803D19DF80210E6
:1067600001290FD000223C4B114602200FF094F873
:10677000FFF78EFE4FF47A70FDF708FAFFF736FF49
:1067800010B010BD354B1A70587099709DF80310F9
:10679000D9709DF8041019719DF8051059719DF874
:1067A000061099719DF80710D9719DF8081019729B
:1067B0009DF8091059729DF80A1099729DF80B10F6
:1067C00001F03F01D9720DF10B019818013211F857
:1067D000014F0473142AF8D19DF8202083F820205B
:1067E0009DF8212083F821209DF8222083F8222083
:1067F0009DF8232083F823209DF8242083F824206B
:106800009DF8252083F825209DF8262083F8262052
:106810009DF8272083F8262083F827209DF828203C
:1068200083F828209DF8292083F829209DF82A2024
:1068300083F82A209DF82B2083F82B200DF12B01C3
:1068400000229818013211F8014F80F82C40142AC8
:10685000F7D193E700F80308337E030858030020BC
:10686000F0B506238BB0052600240125CDE90536B9
:1068700018220723CDE9033221466D4B02942246AC
:106880000327CDE90055022009940FF005F8694B64
:10689000029422462146CDE9005702200EF0FCFF6B
:1068A000CDE901640226644B00962246214630461B
:1068B0000EF0F2FF614B009522462146CDE90174AE
:1068C00030460EF0E9FF09A9204606F08FF9099B32
:1068D000C3F307220292C3F307421B0E01920093F7
:1068E0002246574B214630460EF0D6FF09A92846CE
:1068F00006F07CF9099BDAB20392C3F307220292F5
:10690000C3F307421B0E0192009322464D4B2146D2
:1069100030460EF0C1FF4C4B4C48009422464FF4D9
:10692000FA710FF049FB4A4B4A48009422464FF453
:10693000FA710FF041FB484B484800942A464FF447
:10694000FA710FF039FB464B464800942A464FF443
:10695000FA710FF031FB444B444800942A4642F24E
:1069600010710FF029FB2046FCF7C4F908B1FCF7C1
:10697000E5FB3F4B009400224FF4FA613D480FF0D5
:106980001BFB3D4A002101200FF054F93B4A002136
:1069900002200FF04FF93A4A002104200FF04AF983
:1069A000384A002108200FF045F90021012006F0A7
:1069B0009FF8354B1C7000F041FE3449344806F016
:1069C000CBF8344805F0B8FF24480FF0A1FB324B58
:1069D0000021187805F008FDFFF7ACFE2F4A0021D2
:1069E00010200FF027F92E4A002120200FF022F965
:1069F0002C4A002140200FF01DF92B4A0021802055
:106A00000FF018F9294B2A4819682A4B00940122E3
:106A10000FF0D2FA284B29481968294B009401221B
:106A20000FF0CAFA25480FF073FB0BB0F0BD00BFA2
:106A3000737E0308B37E0308D47E0308F57E030843
:106A4000167F0308377F03081B5A00081C2000200C
:106A5000AD62000804200020B9610008EC1F00208E
:106A60005D620008D01F0020395F0008B81F0020B9
:106A7000A1610008282100203DC70008D95C00085A
:106A80002D620008615C0008E81F0020000003017F
:106A900030010020180100207C010020D1530008A3
:106AA0004D540008B154000831550008A0030020DF
:106AB000A01F0020596100089C030020881F0020AF
:106AC0000161000873B50D4D00262E60FEF7BCFE77
:106AD000C820FDF75BF828683146FBF757FC0446F1
:106AE0000028F3D12868FBF799FC054B009022465B
:106AF000214601200EF0D0FE02B070BD1C1F002008
:106B00005B7F030830B50024A5B07C22214605A890
:106B1000049428F0E3FD53238DF81030012540F252
:106B20000713ADF81230ADF800408DF81450FCF7A3
:106B3000ABFFFE23B0FBF3F000EB400000EB401096
:106B40003A4B8DF815002246214603200EF0A4FE94
:106B50006846FEF7E1FE9DF800309DF801201343E2
:106B600014D158238DF81630072480220021304894
:106B700028F0B4FD224604A92D4828F045FE2C4AF1
:106B800021460120FFF718FC25B030BD0E23294611
:106B900001A8CDE901448DF81630ADF80C40FEF7A0
:106BA0007DFE01AB03CB234C1B88CDF81B10ADF849
:106BB0001F30CDF81700FEF747FE2068FBF754FCA6
:106BC0000A254FF47A7380B2B0FBF3F0B0FBF5F313
:106BD00005FB130030308DF821002068FBF744FCE2
:106BE000642380B2B0FBF3F0B0FBF5F305FB1300B8
:106BF00030308DF822002068FBF736FC80B2B0FB05
:106C0000F5F0B0FBF5F305FB130030308DF82300F1
:106C10002068FBF729FC80B2B0FBF5F305FB1300FD
:106C200030308DF8240015249FE700BF8E7F0308C5
:106C3000582100201C1F00202DE9F047044698B081
:106C4000C1480D46802200210EF036FF2378592BD3
:106C500040F06982052D5ED86378443B162B5AD8E4
:106C6000DFE813F0AB0159009B015900A301590063
:106C7000590059005900BD005900860159005900BA
:106C80005900060259005900E700590059005900FF
:106C90001700A678482E17D1AC4A14210120FFF71F
:106CA0008BFB41F28830FCF771FF0022A84B1146A4
:106CB00003200EF0F1FD40F6B830FCF767FF18B086
:106CC000BDE8F047FFF784BA532E0DD1FFF71AFF46
:106CD00041F28830FCF75AFF9B4A1521012018B079
:106CE000BDE8F047FFF768BB432E17D1002408A882
:106CF0008DF8204005F098FD934A4C23137007232C
:106D000093709DF82030547001204133D07013717E
:106D10000521FFF751FB18B0BDE8F087442EFAD1EA
:106D2000894C8C4DA670592323705A236370FFF74A
:106D3000C9FE2868FBF772FB0022874B00901146C2
:106D400003200EF0A9FD7F220021601C28F0C6FC64
:106D5000072326700126A370E6702671FCF794FEC7
:106D6000FE23B0FBF3F000EB4000042300EB4010E7
:106D70006071A3712868FBF777FB0A274FF47A73D9
:106D800080B2B0FBF3F0B0FBF7F307FB1300303039
:106D9000E0712868FBF768FB642380B2B0FBF3F076
:106DA000B0FBF7F307FB1300303020722868FBF7C5
:106DB0005BFB80B2B0FBF7F0B0FBF7F307FB13000F
:106DC000303060722868FBF74FFB80B2B0FBF7F3FE
:106DD00007FB13003030A07222460B217EE7A37818
:106DE000303BDBB2092B96D85C4C5D4A237023788C
:106DF000DBB25372544A592313704D2353702378D6
:106E00000321303301209370FFF7D6FA23780093E3
:106E10000022544B114601200EF03EFDFFF738FBD7
:106E20002378002B3FF477AF18B0BDE8F047FCF7AC
:106E3000DFBBA578482D48D1434C56232370072348
:106E4000A37018236371062300250126A37106A8E9
:106E50000523E3716570E67026710EF087FF0698D2
:106E600008A912380FF00AF80D9B03F26C73059312
:106E70000C9B334404930B9B0393089B0293099B45
:106E800001930A9B00932A46374B294602200EF0B5
:106E900003FD0D9B25726C3363720C9B3344A3720C
:106EA0000B9BE3720A9B2373099B63732246089B27
:106EB000A3730F213046FFF77FFA2C4B00942A462C
:106EC000114602200EF0E8FC25E7432D7FF423AFA6
:106ED00000213C2209A81C4C089128F0FFFB08A8BF
:106EE000FFF770FB9DF8203063709DF82130A37090
:106EF0009DF82230E3709DF8233023719DF82430F3
:106F000063719DF82530A3719DF82630E3719DF8DB
:106F10002730257023729DF82B509DF8283063721E
:106F20009DF82930A3722A469DF82A30E3720BA9F6
:106F300004F10D00257328F067FC05F10D012246D0
:106F4000C9B20120E5E600BF58210020A77F030851
:106F5000BC7F03081C1F0020DE7F0308841F002065
:106F600058030020018003082A8003085480030886
:106F7000A07839280CD83038C0B2FEF7EBFC8E4A26
:106F80002378137063785370A37893700321A5E678
:106F900018B0BDE8F047FFF76DBAA0783928F7D8E8
:106FA0003038C0B2FEF7DBFCE9E7A0783928EFD82B
:106FB0003038C0B2FEF7D8FCE1E7A378303BDAB254
:106FC000092AE5D8E578303DEAB2092AE0D82179E6
:106FD000A1F14802D2B20B2ADAD8784840FA02F27C
:106FE000D007D5D40A224D2902FB03553BD13C23BF
:106FF0005D43734B4FF47A7068431860714B1860AF
:10700000FEF75EFD6C4A2378137063785370A378A3
:107010009370E378D3700521237913710120FFF772
:10702000CBF9694B002607221E705A7001229A7014
:10703000DA70A178303901EB8100E178303901EB69
:107040004001C9B2197122795A71604A1278D2B2DC
:107050001A725F4A1278D2B25A72FFF719FA5D4B70
:10706000009532462CE74829C3D14FF46163BFE74E
:10707000A278303AD3B2092B8AD8E378303BD9B220
:10708000092985D82079A0F14801C9B20B293FF61A
:107090007FAF4A4D45FA01F1C9073FF579AF0A21A3
:1070A0004D2801FB023339D13C2253434FF47A720D
:1070B0005343494A13601068FEF726FD3E4A237881
:1070C000137063785370A3789370E378D3700521BD
:1070D000237913710120FFF76FF93B4B00221A70DF
:1070E00007225A7001229A70DA70A278303A02EBC5
:1070F0008201E278303A02EB4102D2B29A712279EF
:10710000DA71324A1278D2B21A72314A1278D2B295
:107110005A7218B0BDE8F047FFF7BAB94828C5D190
:107120004FF46162C1E7502B40F0B381022D7FF62E
:10713000F2AD6178A1F13003012B3FF6ECADA378FD
:10714000312B7FF4E8AD052D4ED1E378302B40F0A4
:10715000C1801E4D214E00232B702B7803F0FF02BF
:1071600053B92379303BDBB2337033780093114647
:107170001B4B02200EF090FB15491A4A00230B709E
:107180003378DBB213702B780F4ADBB213720B78B3
:10719000DBB25372FFF77CF9074B22781A706278E2
:1071A0005A70A2789A70E278DA7022791A71FCF734
:1071B000D1FA0521004A91E558210020DEF7FFFFB2
:1071C000140100209C030020580300200601002029
:1071D000841F00207E800308A003002004000020FC
:1071E000B580030806000020082D67D1E378462B00
:1071F00040F0F8802179A1F13000C0B2092800F2F6
:1072000046816279A2F13003092B00F24081A67910
:10721000A6F13003092B00F23A81E379A3F130059E
:10722000092D00F2348101EB81014900B74D203175
:1072300002EB8202C9B2520029702032B449D2B2A4
:107240002F3E0A70F6B2B34A03EB8303F6015B00EC
:1072500016802033B04ADBB21370B04A82F828009F
:107260006379303BDBB282F82930A3792F3BDBB264
:1072700082F82A30E379303BDBB282F82B302B786E
:107280002BB90B7803F0FF020BB9A54B1A70FFF76F
:10729000FFF8A44B22781A7062785A70A2789A701C
:1072A000E278DA7022791A7162795A71A2799A7148
:1072B000E279DA71FCF74EFA08217BE7042D3CD124
:1072C000E278A2F13003DBB2092B11D9A2F141031C
:1072D000192B0AD9FFF7CEF80022934B1146012053
:1072E00018B0BDE8F0470EF0D7BAA2F13703DBB211
:1072F0008E4803708B4B20785970312199708B49DF
:107300001870DA700B78854ADBB213720B78052B94
:10731000834B0CBF012100211970854B1B78DBB218
:107320005372FFF7B5F8FCF715FA4FF4FA60FCF763
:107330002DFCFEF74DFF04213CE71D2D4FD9A61C67
:107340000025DFF8D891DFF8ECA13746A84617F8FA
:10735000012F303AD2B2092A3ED809EB05030320A7
:107360001A731B7BCDE902533B780022CDE9005311
:10737000114653460EF090FA01351E2DE7D1B8F1B3
:10738000000FA7D1FEF7ECF8664B50221A700022CE
:107390005A7007229A700122DA7003F8042F203401
:1073A00016F8012F03F8012FB442F9D15B4B0022EC
:1073B0001A7007225A7001229A70DA705B4A1278AA
:1073C000D2B21A725A4A1278D2B25A721E22DA72A3
:1073D000FFF75EF82321EDE64FF00108CCE7072D1B
:1073E0007FF678AF00254D4FDFF8488102342E46F6
:1073F00014F8012F303AD2B2092A46D8791903205D
:107400000A730B7BCDE9025323780022CDE90053A8
:10741000114643460EF040FA0135082DE8D1002E02
:107420007FF458AFFEF70EF93E4B3C4C50221A70D9
:1074300007229A701A460121002502F8041F5D7088
:10744000D97061190135097B082D01F1300102F86D
:10745000011FF6D10022114600930120364B0EF099
:107460001BFA00232370072363700123A370E370CA
:107470002E4B1B78DBB223722D4B1B78DBB2637271
:10748000E572FFF705F80D2194E60126C4E7002117
:1074900090E6412B7FF43FAC6378432B7FF43BAC09
:1074A000162D7FF438AC254D621C002312F8011F05
:1074B000E9540133142BF9D1FDF75AFF204B5B7DC2
:1074C000012B1ED115490023EA5CC8180133D2B242
:1074D000142B80F82C20F7D1154B00221A701B7842
:1074E000DBB24B72FEF7D4FF0E4A631E153413F85D
:1074F000011F02F8011BA342F9D10A4A1621FFF726
:10750000EDBB0B4B02221A70EEE700BFA703002071
:10751000A60300203C000020A50300205803002003
:10752000A403002058210020148103080601002034
:10753000841F0020D1800308F9800308DE21002089
:107540002C0A002070B5054688B00C46002951D0A1
:1075500033480EF0DDFD26789EB3002D5ED06868BE
:107560002E7870B3032E0BD0132E45D0022E28D1C7
:107570006978012925D00B0623D4FFF75DFB20E0B5
:107580006B78012B07D10078012802D0022800D0A7
:1075900008B905F003F900250DF11F008DF81F5003
:1075A00005F042F91F4A4C231370072393709DF88E
:1075B0001F305570012041330521D0701371FEF743
:1075C000FBFE237C052B15D894F90A20059294F92B
:1075D00009200492144A52F82330039394F9083096
:1075E000CDE901630022E368009311460F4B0320AD
:1075F0000EF052F908B070BD6B78012BE1D1027822
:107600000B4B02F001021A702AB90A4B11460320F3
:107610000EF042F9D5E7084B0022F7E72E46D0E7F7
:107620000420002058210020A08103084C81030879
:10763000342000203981030843810308034B0022D2
:10764000C3E902220122C3E900227047F42100208D
:1076500000487047F42100204FF0B04382B0DA6C4C
:107660000243DA64DB6C03400193019B02B0704774
:107670002DE9F04186B000240220154D0594FFF756
:10768000EBFF0420FFF7E8FF124F03944FF48076DE
:1076900001230DEB0001CDE9016328460323049388
:1076A0004FF4005801F04AF801A93846CDF804809B
:1076B00001F044F822464146384601F065F9284673
:1076C0002246314601F060F9204606B0BDE8F0815F
:1076D0000004004800080048032810B50ED801280F
:1076E00010D868B902460B484FF4807101F04CF98C
:1076F000002209484FF4005101F046F9002010BD66
:107700000122F0E7002203484FF4807101F03CF9B8
:107710000122EEE7000400480008004802207047FC
:107720000020704701207047002814BF16200F204A
:10773000704700000D48854600F025F80C480D49BB
:107740000D4A002302E0D458C4500433C4188C42BC
:10775000F9D30A4A0A4C002301E013600432A24222
:10776000FBD328F023F8FBF7CBFCFEE70000012059
:10777000000000204808002060E8030848080020B6
:1077800020420020FEE7704710B5032000F06EFC99
:1077900001F07CFA064B18600F20FCF7EDF9044667
:1077A00018B9FBF723FE204610BD0124FBE700BFFC
:1077B000A80300204FF0E022136923F002031361B5
:1077C00070474FF0E022136943F0020313617047E2
:1077D000014BD3F8900570470070FF1F014BD3F8A1
:1077E000940570470070FF1F014BD3F89805704750
:1077F0000070FF1F024A536843F001035360704753
:10780000002004E0024A536843F0020353607047CB
:10781000002004E0024A536843F0040353607047B9
:10782000002004E08068C0F380007047F7B50023B3
:1078300001930446002800F0E980856D25B9FBF727
:10784000E9F8E56584F8545023689A68D00040F15F
:10785000A1809A68D10000F1B480A26D42F01002BC
:10786000A265E26D42F00102E26501251846FFF7CC
:10787000D9FFA26D02F01002024340F0C980A26D50
:10788000206922F4817242F00202A2659A68D2074E
:107890005DD4226BA67E94F82CC0003A18BF01225A
:1078A0001703D4E902120A43217E42EA8132617E43
:1078B00042EAC13242EA4632002842EA4C02B4BFF0
:1078C00020F000414FF400113A430A4394F820108D
:1078D000012903D1002E76D142F48032616A21B1B0
:1078E000A66A01F4E07131430A43D968E66C21F4D9
:1078F000FE3121F4FF711143D96094F83C20616896
:10790000012A01F0404C4CEA060609D1D4E91027BF
:107910003A433243A66C324342EA0C0242F001067B
:107920001F693E4A3A4032431A6121F00042B2F1E7
:10793000804F0CD0B1F1004F09D0394ED6F808274E
:1079400001F4701122F470120A43C6F808275A692C
:10795000666BA16B22F0070232435A615A6922F02A
:10796000700242EA01125A61002835D19A6A62F027
:107970000F029A625B6903F007039E423CD1002329
:10798000E365A36D23F0030343F00103A3652846D9
:1079900003B0F0BD9A68234922F0104222F017028A
:1079A00042F080529A60204A1268B2FBF1F2013232
:1079B00052000192019A002A3FF44BAF019A013A1A
:1079C000F7E7002552E7A16D41F02001A165E16DC7
:1079D00041F00101E16581E7B0F5001FCAD19A6A63
:1079E000E269013A92006FF00F0102F01C0201FA05
:1079F00002F2216E0A43BCE7A36D23F0120343F0A9
:107A00001003A365E36D43F00103E3650125BEE7C1
:107A1000A36D43F01003A365F8E700BF02FCFF1F4E
:107A200000200140400D0300A8030020F8B545697F
:107A3000082D04460E460AD00368DB68D80705D532
:107A4000A36D43F02003A3650120F8BD0425FCF7D6
:107A500095F8074623681A682A4220D0A26D42F49E
:107A60000072A265DA6812F4406F14D1A27E92B956
:107A70001A6812070FD51846FFF7D4FE20BB5A68C4
:107A800022F00C025A60A26D22F4807222F00102F0
:107A900042F00102A265227EFAB10020D5E7711CF6
:107AA000D9D0FCF76BF8C01BB04201D8002ED1D161
:107AB00023681B682B40CDD1A26D84F8543042F06E
:107AC0000402A2650320C0E7A26D42F02002A26575
:107AD000E26D42F00102E265DDE70C221A60DCE7AC
:107AE0000368186C70470000F7B50023019390F805
:107AF0005430012B044600F0C08005680269012360
:107B000080F854302846FFF78DFE002840F0AF8003
:107B1000D1E90030022822F004027ED0B2F1004FF9
:107B2000C3F3110E35D1AA6A42EA0E02AA628A682C
:107B3000686902EA032222F07C4222F0FF0220EA76
:107B400003210A43002B6A611DDA4D4A4D4DD2F8DC
:107B50000817AB4201F0E07043D10D0213D4D2F804
:107B6000083723F0E073034343F40003C2F80837F7
:107B7000454B1A68454BB2FBF3F20C2302FB03336F
:107B80000193019B53BB0020002384F8543003B0C1
:107B9000F0BD226E00F01F074FF00F0C0CFA07FC2F
:107BA0006FEA0C0622EA0C0CBEF1000F11D1C3F3F0
:107BB0008462BA4042EA0C0222668008E26901301F
:107BC0009042B4D8A86AC3F38362BA4006403243F5
:107BD000ACE793FAA3F2B2FA82F2EAE7019B013B27
:107BE000CEE72B4DAB420BD1C901CCD4D2F808372C
:107BF00023F0E073034343F08073C2F80837C2E711
:107C0000244DAB42BFD14B02BDD4D2F8083723F08C
:107C1000E073034343F48003EFE7B2F1004F01BF89
:107C2000AA6AC3F311018A43AA62002BABDA154892
:107C300013498342D1F8082709D1D1F8083702F057
:107C4000A07223F0E0731A43C1F808279BE710489D
:107C5000834204D1D1F8083702F44002F1E70D481D
:107C6000834290D1D1F8083702F0C072E9E7A26DE3
:107C700042F02002A265184686E7022087E700BF8F
:107C800000200140001000B0A8030020400D0300B8
:107C9000004000B8002000B4026838B50446104621
:107CA000FFF7C0FD08B9002038BD9368990707D4D5
:107CB000936823F0004323F0170343F0100393600D
:107CC000FBF75CFF054623689B685B07EBD5FBF77A
:107CD00055FF401B0228F6D923689B685A07F2D546
:107CE000A36D43F01003A365E36D43F00103E36567
:107CF0000120D9E773B50023026801939368DD077B
:107D0000044602D5002002B070BD9168214B194293
:107D100009D0A36D43F01003A365E36D43F00103A5
:107D2000E3650120EFE7936823F0004323F0170396
:107D300043F001039360184BD3F8083718021CD4A2
:107D4000637E012BDED0FBF719FF144E0546226837
:107D50001368DB07D6D49368D9075FBF93683340B5
:107D600043F001039360FBF709FF401B0228EED9A3
:107D700023681B68DA07EAD4CBE7094B094A1B687A
:107D8000B3FBF2F301330193019B002BD8D0019B8D
:107D9000013BF8E71700008000200140E8FFFF7F6B
:107DA000A8030020400D030038B504460068FFF723
:107DB00039FD054620BB94F85430012B20D0012317
:107DC00084F854302046FFF795FFB0B9A36D2268C0
:107DD00023F4706323F0010343F48073A3651C2331
:107DE000E065136084F85400936823F0004323F0A7
:107DF000170343F00403936038BD84F85450FBE745
:107E00000220F9E7026838B5936891680446C8070C
:107E100001D4002038BD9907FBD4936803F0050313
:107E2000012B19D1936823F0004323F0170343F08B
:107E30000203936003231360FBF7A0FE054623684B
:107E40009B68DB07E5D5FBF799FE401B0228F6D9B6
:107E500023689B68DA07F2D5A36D43F01003A3658E
:107E6000E36D43F00103E3650120D3E770B50446F9
:107E700000284BD0836D43F002038365FFF70CFFAE
:107E8000054668B92046FFF7BDFF054608B901233E
:107E9000A3652268936823F0104323F017039360CF
:107EA00023685A6822F4677222F003025A6040F293
:107EB0009F321A60D968164A0A40DA601A6922F0BD
:107EC00040421A615A6922F007025A611A6A02F0A6
:107ED000F0221A625A6A02F0F0225A62DA6A02F05A
:107EE000F022DA629A6A0B4A00269E62D2F80837BC
:107EF00023F0FE73C2F808372046FAF79FFDE665C7
:107F00002666A66584F85460284670BD0125FBE707
:107F100000023E830020014010B590F85430012B40
:107F2000044615D0012380F85430FFF7B5FE58B948
:107F30002046FFF767FF38B9A36D23F4807323F061
:107F4000010343F00103A365002384F8543010BDFE
:107F50000220FCE7F7B50023019390F85430012B81
:107F600004467FD0012380F85430FFF74BFF23688D
:107F70009A6812F00102054607D0A36D43F0100382
:107F8000A365002384F854302DE0A16D364F21F411
:107F9000817141F00201A165DE68D96826F4FF46CF
:107FA00026F07C0621F40041360421F00301360C52
:107FB000D96008209968394041F00041996099687A
:107FC000002913DA0199013101910199B1F52E3F90
:107FD000F5D3A36D23F0120343F01003A365002330
:107FE00084F854300125284603B0F0BDD3F8B4100E
:107FF000013801F07F010A44DCD199681A48014038
:1080000041F001019960D3F8B41021F07F0141EAF9
:10801000D202C3F8B4209A68024042F002029A6089
:10802000FBF7ACFD074623689A68D20708D4DA68E4
:108030003243DA60A36D23F0030343F001039FE7AB
:10804000FBF79CFDC01B0228EDD923689B68D9076C
:10805000E9D5A36D43F01003A365E36D43F001037D
:10806000E365BFE70225BEE7E8FFFF7F0749CA686F
:1080700022F4E0620302120403F4E063120C1343DF
:1080800043F0BF6343F40033CB60704700ED00E082
:10809000164B30B5DC68C4F30224C4F10703251D78
:1080A000042B28BF0423062D4FF0FF358CBF033C63
:1080B000002405FA03F321EA0303A54022EA05029E
:1080C000A340002843EA0203ACBF00F16040084A25
:1080D0004FEA0313B8BF00F00F00DBB2AABF00F5F0
:1080E0006140135480F8003330BD00BF00ED00E064
:1080F00014ED00E0002807DB044A4109012300F0E9
:108100001F00834042F82130704700BF00E100E0CB
:1081100000280CDB4309064900F01F002033012230
:10812000824041F82320BFF34F8FBFF36F8F70471A
:1081300000E100E070B5D0E913456560446D14B10D
:10814000D0E916456560D0E9105404F01C060124FE
:10815000B4406C60046863608368102B0BBFA2603E
:10816000A160E160E26070BD0268416CD3B210B5FD
:10817000083B1424B3FBF4F30B4CA24288BF0B4A18
:1081800021F0030199BF01F1804202F50232521839
:1081900007338264064AC26403F01F03012202FA15
:1081A00003F3036510BD00BF070402401C08024032
:1081B0008008024038B500285CD002682E4B9A42F5
:1081C0004FF014014AD82D4B1344B3FBF1F32C4963
:1081D0009B00C0E91013022380F82530136805695D
:1081E00023F4FF4323F070031360D0E902432343D9
:1081F0002B43456911682B4385692B43C5692B4384
:10820000056A2B430B431360FFF7AEFFB4F5804FB5
:1082100004BF002343604368816C03F07F020A605F
:10822000D0E91314013B032B4C601ED8154B1649A3
:10823000816513449B000121013A01FA02F20021F9
:108240004365C2651960114B5A6400230122C36360
:1082500080F8243080F82520184638BD0C4B134494
:10826000B3FBF1F30B499B00B3E70023C0E91533DF
:10827000C365EAE70120F0E707040240F8FFFDBF0D
:10828000000002403F820010400902400009024005
:10829000F8FBFDBF0004024038B5002841D0026859
:1082A000136823F0010313601F4B9A424FF014012F
:1082B00030D81E4B1344B3FBF1F31D499B00C0E9BA
:1082C0001013012403F01C0304FA03F300251560C6
:1082D0004B60FFF749FF836C41681D60D0E91332A2
:1082E0005A604A1E032A06D8124B0B449B00944046
:1082F0001D60114B5C640023C363C0E91533C0E902
:108300000B33C0E90D33C36580F8253080F8243085
:10831000184638BD094B1344B3FBF1F308499B00E1
:10832000CDE70120F5E700BF07040240F8FFFDBFDD
:10833000000002403F82001000090240F8FBFDBF30
:108340000004024070B590F82450012D04463BD043
:1083500090F825600125AE4280F824504FF00006C9
:108360002CD1022580F825500568C6632E6826F0BA
:1083700001062E60FFF7DEFE036BBBB12B6843F0F6
:108380000E032B60A36C1A68D20342BF1A6842F432
:1083900080721A60636D1BB11A6842F480721A60B1
:1083A0002B6843F001032B60002070BD2B6823F085
:1083B00004032B602B6843F00A03E2E78023C363C6
:1083C00080F824602846F0E70220EEE7034640B13B
:1083D00090F82520022A06D00422C263002280F8E9
:1083E0002420012070470268806C116821F00E0182
:1083F0001160016821F480710160116821F00101B0
:108400001160D3E9100202F01C0101228A4042608F
:10841000D3E9132151605A6D32B1116821F4807192
:108420001160D3E9162151600122002083F8252034
:1084300083F82400704708B590F82530022B03D04C
:108440000423C363012008BD03681A6822F00E02EA
:108450001A601A6822F001021A60826C136823F411
:1084600080731360D0E9101303F01C0201239340C2
:108470004B60D0E913325A60436D33B11A6822F46D
:1084800080721A60D0E916325A60012380F82530D4
:10849000002380F82430836B03B198470020D2E793
:1084A00070B4426C046C036826681D6802F01C02FC
:1084B0000421914031420FD015F0040F0CD01A68FE
:1084C00092065EBF1A6822F004021A60036B6160B4
:1084D000002B33D070BC184702219140314217D095
:1084E00015F0020F14D01A68940606D41A6822F008
:1084F0000A021A60012280F82520114A93428CBF9B
:10850000104B114B5960002380F82430C36ADFE719
:1085100008219140314211D029070FD5196821F067
:108520000E011960012303FA02F26260C36380F84E
:108530002530002380F82430436BC9E770BC7047B6
:108540008000024000040240000002400A4A5369D1
:1085500043F4802330B55361EFF3108472B60023E7
:10856000CD58C5500433B3F5807FF9D11369DB03CF
:10857000FCD484F3108830BD00400058064B5A6983
:10858000002ABFBF054A9A6002F188329A60BABFDA
:108590005869C00F0020704700400058230167450C
:1085A000044B5A6942F000425A615869C043C00FF7
:1085B000704700BF0040005870B50546FBF7DEFA73
:1085C000124E04463369D90313D43369DA0744BF22
:1085D000012232614CF2FA32134011D10B4E306954
:1085E00010F480200BD0FBF7C9FA001BA842F6D389
:1085F00004E0FBF7C3FA001BA842E3D3032070BDDD
:10860000024A1361024A01205360F8E70040005813
:10861000042200202DE9F041184D98462B78012BBB
:1086200006460C46174626D001232B704FF47A706D
:1086300000236B60FFF7C0FFA0B9012E16D1104ACE
:10864000536943F0010353612760BFF36F8FC4F890
:1086500004804FF47A70FFF7AFFF094A536923EAA9
:108660000603536100232B70BDE8F0813946204694
:10867000FFF76CFFEDE70220F6E700BF04220020C1
:1086800000400058054A536923F47E7343EAC00052
:1086900040F4803040F002005061704700400058C4
:1086A0002DE9F041234F3B78012B054688463FD00A
:1086B00001233B704FF47A7000237B60FFF77CFF4F
:1086C000044688B92B68042B13D11B4A536943F421
:1086D000803343F0040353614FF47A70FFF76CFF6B
:1086E0000446154B1A681B6800233B702046BDE802
:1086F000F0814FF0FF33C8F800306E68D5E90132E1
:108700001344B3420AD93046FFF7BCFF4FF47A70E6
:10871000FFF752FF50B1C8F800600446064A53699B
:1087200023F47E7323F002035361DAE70136E5E7B1
:108730000224DBE704220020004000582DE9F04F1E
:10874000524C00234FF00F090A6832FA03F501D1A9
:10875000BDE8F08F012505FA03F818EA020200F0DF
:108760008E804E68032706F003054FEA430E07FA92
:108770000EFC6F1E012F6FEA0C0C32D8876807EAD7
:108780000C0ACF6807FA0EF747EA0A0787604768BE
:1087900027EA0808C6F300179F4047EA0807476022
:1087A000C76807EA0C088F6807FA0EF747EA080758
:1087B000022DC76017D14FEAD30800EB880803F0F9
:1087C000070AD8F820704FEA8A0A09FA0AFB27EA52
:1087D0000B0B0F6907FA0AF747EA0B07C8F8207076
:1087E00001E0032DDCD1076805FA0EF507EA0C0756
:1087F0003D4316F4403F056041D023F0030707F1E5
:10880000804707F5803703F0030CBD684FEA8C0CF6
:108810004FF0070E0EFA0CFEB0F1904F25EA0E0E47
:108820002FD01B4DA8422ED005F58065A84214BF5D
:108830000725022505FA0CF545EA0E05BD602568F9
:10884000D74316F4801F0CBF3D4015432560656873
:1088500016F4001F0CBF3D4015436560D4F88050EE
:1088600016F4803F0CBF3D401543C4F88050D4F847
:108870008450B60354BF3D401543C4F884500133BF
:1088800062E70025D6E70125D4E700BF00080058BD
:1088900000040048374A2DE9F04F00234FF0010A49
:1088A0004FF0070B4FF00F0931FA03F401D1BDE887
:1088B000F08F0AFA03FC1CEA010654D023F00304EB
:1088C00004F1804404F5803403F00307A568BF0079
:1088D0000BFA07F8B0F1904F08EA050E45D0264D87
:1088E000A84244D005F58065A8420CBF02250725A3
:1088F000BD40754517D1D2F8805025EA0605C2F86B
:108900008050D2F8845025EA0605C2F884501568D4
:1089100025EA06051560556825EA06055560A5682F
:1089200025EA0805A560056803265C0006FA04F43C
:1089300023FA06F6254300EB8606056003F00705DB
:10894000376AAD0009FA05F527EA05073762856839
:1089500025EA04058560456825EA0C054560C5687B
:1089600025EA0404C46001339EE70025C0E7012521
:10897000BEE700BF00080058000400480369194220
:1089800014BF0120002070470AB1816170478162E5
:108990007047436901EA030221EA030141EA024107
:1089A00081617047044AD168014208B502D0D060A5
:1089B000FDF77EFC08BD00BF00080058024A13689E
:1089C00043F4807313607047000400580D4B10B5DA
:1089D0005B690C4628B99A0507D500F027F820B145
:1089E00010BD9B0501D400F019F8074A1369012C4A
:1089F00023F00403136101D130BFF1E740BF20BF72
:108A000020BFEDE70004005800ED00E0024B1868BD
:108A100000F4C060704700BF00040058024A1368A9
:108A200043F4804313607047000400580C4A1368F5
:108A300023F4804313600B4B1B6832214B430A49DC
:108A4000B3FBF1F35169890500D533B9536913F4C8
:108A5000007F14BF032000207047013BF2E700BFF6
:108A600000040058A803002040420F000B4A13687E
:108A700023F0070343F002031360094B1A6901282E
:108A800042F004021A6105D130BF1A6922F00402D3
:108A90001A61704740BF20BF20BFF6E700040058AE
:108AA00000ED00E04FF0B0431868C0F3404070475D
:108AB0004FF0B0431868C0F3400070474FF0B04229
:108AC000536823F47F4343EA0023536070474FF019
:108AD000B0431868C0F34060704700007FB54FF0A6
:108AE000B0432C4AD3F80831C0F3031003F00F034E
:108AF00052F82040284A52F82330B4FBF3F4FFF731
:108B000085FF264B054693E80700B5F5007F04ABCB
:108B100003E9070010D0224B9C4218D303F5B7039A
:108B200003F67F539C4229D903F5741303F51063B0
:108B30009C4225D802230BE01A4B9C4207D91A4BC2
:108B40009C421BD903F5370303F5D853F0E7002304
:108B500004AA02EB830353F80C4C144D2B6823F04A
:108B6000070323432B60FBF709F806462B6803F045
:108B700007039C4206D1002004B070BD0123E7E743
:108B80000024EAE7FAF7FAFF801B0228EED9032057
:108B9000F2E700BFB881030818820308C82C030855
:108BA000C0CF6A00BFEA21013F9334020040005861
:108BB0004FF0B04310B59A68D96812F00C0205D096
:108BC0000C2A4AD101F00303012B51D14FF0B041DF
:108BD0002B480B6813F0080306D00B6813F008034A
:108BE00037D1D1F8941007E00C68240756BFD1F8AC
:108BF00094300968C3F3032350F82330002A0CBFD4
:108C0000184600204FF0B0418A6802F00C020C2A8E
:108C10001ED1CA6802F00302022A2ED0032A06D10E
:108C20000B68184A13F4801F174B18BF13464FF0F8
:108C3000B042D068D168D268C0F306205843C1F36F
:108C400002130133B0FBF3F0530F0133B0FBF3F029
:108C500010BD0B68C3F30313CEE7042A05D0082A1E
:108C600006D11B6813F4801305D006480023C9E71A
:108C700000231846C6E70448C4E7024BD7E700BF05
:108C8000B88103080024F4000048E80108B5FFF7A4
:108C90008FFF4FF0B043044A9B68C3F3031352F8AD
:108CA0002330B0FBF3F008BD188203082DE9F04132
:108CB0000446002853D04FF0B0439D68DE68036837
:108CC0009B0605F00C0506F0030668D5026A1DB187
:108CD0000C2D46D1012E44D1002A40D04FF0B04394
:108CE000A16A1A68170756BFD3F894301B681B098E
:108CF00003F0F00399421FD90846FFF7EFFE002862
:108D00002DD14FF0B042136843F00803136013688D
:108D1000A16A23F0F0030B431360606AFFF7CEFEF5
:108D2000FFF7B4FFAB4B1860AB4B1868FAF724FFA2
:108D3000002834D0BDE8F0814FF0B042136843F012
:108D400008031360136823F0F0030B431360606A99
:108D5000FFF7B4FE0846FFF7C1FE0028E0D001206F
:108D6000E8E74FF0B043002A54D01A6842F00102FD
:108D70001A60FAF703FF0746FFF79AFE002842D071
:108D80004FF0B042136843F0080313601368A16A00
:108D900023F0F0030B431360606AFFF78FFE236834
:108DA000D80748D42368990700F18C8023681E07F0
:108DB00040F1FA80A3694FF0B046002B00F0E1804B
:108DC000D6F89430E16903F01002914200F0C480BB
:108DD00003F00302022AC2D0D80740F1B380D6F8CC
:108DE000943023F00103C6F89430FAF7C7FE074623
:108DF000D6F89430990740F1A580FAF7BFFEC31B5F
:108E0000112BF5D904E0FAF7B9FEC01B0228B3D93B
:108E100003208FE71A6822F001021A60FAF7AEFE0B
:108E20000746FFF745FE0028B9D0FAF7A7FEC01B9A
:108E30000228F6D9ECE7082D03D00C2D05D1032E1E
:108E400003D16368002BADD189E74FF0B043A1682F
:108E50001A6822F480120A431A606268B2F5803FF1
:108E600010D11A6842F480321A60FAF787FE07467A
:108E7000FFF718FE002895D1FAF780FEC01B642882
:108E8000F6D9C5E7B2F5041F04D11A6842F40012FE
:108E90001A60E6E7196821F480311960196821F435
:108EA00000111960002AE0D1FAF768FE0746FFF7C3
:108EB000F9FD00283FF476AFFAF760FEC01B642886
:108EC000F5D9A5E7042D236903D00C2D0ED1022E70
:108ED0000CD1002B3FF443AF4FF0B04261695368AF
:108EE00023F0FE4343EA016353605FE74FF0B0466F
:108EF000BBB1336843F480733360FAF73FFE074633
:108F000033685A0505D4FAF739FEC31B022BF7D98B
:108F10007EE77368626923F0FE4343EA026373608D
:108F200044E7336823F480733360FAF727FE07467B
:108F300033685B057FF53AAFFAF720FEC31B022BBF
:108F4000F6D965E74FF0B042E169D2F8943023F0EA
:108F500010030B43C2F894304FF0B047D7F8943069
:108F600043F00103C7F89430FAF708FE0646D7F835
:108F700094309A0718D4FAF701FE831B112BF6D907
:108F800046E7D6F8943023F00103C6F89430FAF798
:108F9000F5FD0746D6F894309B0705D5FAF7EEFDA8
:108FA000C31B112BF6D933E72368580754D50B4F51
:108FB0003B68D90514D4FFF701FDFAF7DFFD06463B
:108FC0003B68DA050CD4FAF7D9FD831B022BF7D9DD
:108FD0001EE700BFA8030020AC03002000040058D7
:108FE000E3684FF0B046002B58D023F08003052BE8
:108FF00002BFD6F8903043F00403C6F890304FF02B
:10900000B046FAF7BBFDD6F8903043F001030746AF
:10901000C6F8903041F28838D6F890309B0705D4D6
:10902000FAF7ACFDC31B4345F6D9F1E6E36823F03C
:109030000403812B1BD1FAF7A1FDD6F8903043F041
:109040008003C6F8903007464FF0B04641F28838AA
:10905000D6F89030180504D5E36A002B4AD10020D9
:1090600068E6FAF78BFDC01B4045F1D9D0E6FAF768
:1090700085FDD6F8903023F08003C6F8903007467F
:109080004FF0B04641F28838D6F890301905E3D554
:10909000FAF774FDC01B4045F6D9B9E6FAF76EFD44
:1090A000D6F8903023F080030746C6F8903041F29E
:1090B0008838D6F890301A0516D4FAF75FFDD6F83E
:1090C000903023F00103C6F8903007464FF0B048C7
:1090D00041F28836D8F890309B07BDD5FAF74EFD9F
:1090E000C31BB342F6D993E6FAF748FDC01B4045CF
:1090F000DFD98DE60C2D4ED0022B4FF0B0431A680D
:1091000022F080721A6033D1FAF738FD0546FFF776
:10911000DEFC38BBD4E90C314FF0B0420B43D068D1
:109120002D4901400B43E16B0B43216C0B43616CF8
:109130000B43A16B43EA0123D360136843F08073B0
:109140001360D36843F08053D360FAF717FD0446E9
:10915000FFF7BDFC002882D1FAF710FD001B0A289A
:10916000F6D955E6FAF70AFD401B0A28CFD94FE693
:10917000FAF704FD0446FFF7AAFC30B94FF0B042FD
:10918000164BD1680B40D36069E7FAF7F7FC001B78
:109190000A28F0D93CE6012B3FF4E1AD4FF0B04393
:1091A000D868236B00F003029A427FF4D8AD626B5B
:1091B00000F0700393427FF4D2ADA26B00F4FE4343
:1091C000B3EB022F7FF4CBAD636C00F06040C01AAC
:1091D00018BF0120AEE500BF8C80C111FCFFFEEE80
:1091E0002DE9F0410D46044610B90120BDE8F0819B
:1091F000684E336803F007038B4216D323689A073F
:1092000027D54FF0B047A268BB6823F0F0031343A3
:10921000BB60FAF7B3FC0646BB68DB0319D4FAF768
:10922000ADFC831B022BF7D911E0336823F0070351
:109230000B433360FAF7A2FC0746336803F00703D9
:10924000AB42DBD0FAF79AFCC01B0228F5D9032009
:10925000CCE72368580617D54FF0B0476269D7F8B6
:10926000083123F00F0343EA1213C7F80831FAF765
:1092700085FC0646D7F80831D90305D4FAF77EFCF9
:10928000831B022BF6D9E2E723685A0713D54FF068
:10929000B047E268BB6823F4E0631343BB60FAF7AE
:1092A0006DFC0646BB689B0305D4FAF767FC831B7D
:1092B000022BF7D9CBE72368180714D54FF0B04736
:1092C0002269BB6823F4605343EAC203BB60FAF728
:1092D00055FC0646BB68590305D4FAF74FFC831BBF
:1092E000022BF7D9B3E72368DA070FD4294C236898
:1092F00003F00703AB4239D8FFF7C8FC264B1860D0
:10930000264BBDE8F0411868FAF736BC6268022ABD
:109310001DD1FFF7C7FB00283FF467AF4FF0B04601
:1093200041F28838B36823F003031343B360FAF7BC
:1093300025FC0746B368626803F00C03B3EB820FA9
:10934000D4D0FAF71BFCC01B4045F3D97FE7032AB2
:1093500002D1FFF7BCFBDEE712B9FFF7A9FBDAE7A2
:109360004FF0B0431B685B05D8D43EE7236823F079
:1093700007032B432360FAF701FC0646236803F03A
:109380000703AB42B8D0FAF7F9FB801B0228F5D9E6
:109390005DE700BF00400058A8030020AC03002098
:1093A00008B5FFF773FC4FF0B043044A9B68C3F362
:1093B000022352F82330D84008BD00BFF8810308CB
:1093C00008B5FFF763FC4FF0B043044A9B68C3F352
:1093D000C22352F82330D84008BD00BFF8810308EB
:1093E0004FF0B043D3F89000C0F3400070474FF007
:1093F000B0410209D1F8883002F47F22000123EA4B
:10940000020300F47F200343C1F8883070474FF017
:10941000B041020CD1F88830120423EA020343EA77
:109420000040C1F8880070470368DA0370B504464D
:1094300039D5FFF7C3FAFAF7A1FB614E0546336849
:10944000DB0532D54FF0B043616BD3F8902002F4C6
:10945000407291421DD0D3F89010D3F8902042F47E
:109460008032C3F89020D3F8902021F4407022F489
:1094700080328D07C3F89020C3F8900009D5FAF721
:109480007DFB41F288360546FFF7AAFF012840F030
:1094900090804FF0B042616BD2F8903023F440736B
:1094A0000B43C2F89030002605E0FAF767FB401B3B
:1094B0000228C4D903262568E8070AD54FF0B04131
:1094C0006268D1F8883023EA124392B21343C1F89C
:1094D0008830A9070AD54FF0B041A268D1F888308A
:1094E00023EA124392B21343C1F88830AA0609D581
:1094F0004FF0B0422169D2F8883023F440630B4327
:10950000C2F88830AB0502D5206AFFF780FF6805F6
:1095100002D5606AFFF77BFF290502D5A06AFFF735
:1095200076FF6A0602D56069FFF761FF2B0602D558
:10953000A069FFF75CFFE80502D5E069FFF757FF78
:10954000E90610D54FF0B042E168D2F8883023F434
:1095500040730B43C2F88830B1F5807F02BFD368F7
:1095600043F08073D3602A040ED54FF0B042216BD4
:10957000D2F8883023F040430B43C2F8883019B941
:10958000D36843F08073D3606B0410D54FF0B042C2
:10959000E16AD2F8883023F040530B43B1F1005F09
:1095A000C2F8883003D1D36843F48033D3603046A7
:1095B00070BDFAF7E3FA401BB0427FF665AF79E77A
:1095C0000004005830B590F82C30012B02464FF0C3
:1095D000020022D0174B82F82D00CA24012582F800
:1095E0002C505C6253245C62B1F5807F146B9969E6
:1095F00014D121F488519961596C24F0010421F0AF
:10960000004159641463DD650A4BFF215962002053
:10961000012382F82D3082F82C0030BD21F408514E
:109620009961D96C24F0020421F00041D9641463DB
:10963000D865E9E70028004070B50B4E036B756DE7
:109640001D40EA07044603D50123F365FAF729FD17
:10965000AB0704D50223F365204600F0C9F90123C6
:1096600084F82D3070BD00BF0028004038B50A4C8A
:10967000E36823F02003E360FAF780FA0546E36825
:109680009B0601D5002038BDFAF778FA401BB0F5EB
:109690007A7FF4D90320F6E700280040F8B5114D91
:1096A000EC6814F0400406461AD1EB6843F08003DE
:1096B000EB60FAF763FA23460746EC6814F04004BF
:1096C00001D1032B01D11846F8BDFAF757FAC01B98
:1096D000B0F57A7F234684BF032386F82D30ECE76C
:1096E0000023F0E70028004038B50F4CE36823F072
:1096F0008003E360A3699B06054606D4FFF7B6FF27
:1097000010B1032085F82D0038BDA36923F0200394
:10971000A361FFF7ABFF10B1032085F82D00A3690B
:1097200043F02003A361EFE70028004038B504466A
:1097300000284BD090F82D3003F0FF021BB980F8C1
:109740002C20F9F737FD0223214D84F82D30EB68EA
:10975000DB0636D4CA236B6253236B622046FFF7C5
:109760009DFF10B1FF236B6238BDAB6923F08E63A0
:1097700023F04003AB6121696368AA690B4313437B
:10978000A2691343AB61D4E9022343EA02432B618C
:10979000D4E90931EA680B4322F4F8521343EB6031
:1097A0002046FFF7A1FF0028DCD1D4E90713AA69FE
:1097B0000B4322F06042134362691343AB61FF2302
:1097C0006B62012384F82D300020CDE70120CBE728
:1097D000002800400023092803D840EA0310C0B243
:1097E00070470A380133C0B2F5E700002DE9F047B1
:1097F00090F82C30012B05464FF0020069D0012370
:1098000085F82C304E4B85F82D00DE6806F4407646
:10981000B6F5807F78D04C69087891F8019091F87E
:1098200002A091F82470002A55D19B6913F04003DF
:1098300008BFCB70FFF7CEFF80464846FFF7CAFF50
:1098400002465046FFF7C6FF81463846FFF7C2FF83
:109850000B6ACF78234343EA875343EA090343EA79
:10986000084343EA022343EA0063354ACA205062B0
:10987000532050628C6A8869B4F5807F946945D121
:1098800024F4885494610124D465B6F5807F09BF1F
:10989000CB6913640343536418BF5064284B4A6870
:1098A0001A672A6B42F001022A639A6942F48852CD
:1098B0009A61244AD2F8803043F40033C2F88030F1
:1098C0001F4BFF225A620020012385F82D3085F8B6
:1098D0002C00BDE8F087B4F1803F07D0B4F5000F4D
:1098E00004D09B6913F0400308BFCB700B6ACA78A1
:1098F0001C4344EA0A0444EA004343EA092343EAD6
:10990000825343EA0763B0E70023AEE724F4085428
:1099100094610224D465B6F5807F09BFCB69936456
:109920000343D36418BFD064054B4A685A672A6B57
:1099300042F002022A639A6942F40852B8E700BF73
:10994000002800400008005890F82C20012A034607
:109950004FF0020012D00A4A83F82D00CA2151624A
:1099600053215162916941F020019161FF215162BF
:109970000020012283F82D2083F82C00704700BFBF
:109980000028004090F82C20012A03464FF00200E6
:1099900019D00D4A83F82D00CA215162532151621A
:1099A00091690A4841F080019161D0F8801041F43A
:1099B0008021C0F88010FF2151620020012283F82D
:1099C0002D2083F82C007047002800400008005824
:1099D000064B5A6D520610B5044603D54022DA658F
:1099E000FAF762FB012384F82D3010BD00280040F7
:1099F0007047890001F1804101F531410A607047EB
:109A0000890001F1804101F531410868704700008B
:109A10002DE9F3471F46894690460446FAF7AEF80B
:109A20000A9D3D442D1AFAF7A9F8264B1E68C6F385
:109A3000CB366E43824601962268936839EA030367
:109A40000CBF01230023434501D100202EE07B1CE5
:109A5000F3D0FAF793F8A0EB0A00A84229D32368C1
:109A60005A6822F0E0025A606268B2F5827F0AD139
:109A7000A268B2F5004F02D0B2F5806F03D11A6828
:109A800022F040021A60A26AB2F5005F07D11A689C
:109A900022F400521A601A6842F400521A6001233C
:109AA00084F85D30002384F85C30032002B0BDE808
:109AB000F087019A019B002A03F1FF33019308BF4D
:109AC0001546B9E7A80300202DE9F74F9946002372
:109AD0008DF80330044688461746FAF74FF80C9D78
:109AE0004D442D1AFAF74AF82C4BD4F800B01E68F2
:109AF00023235E43360D6E438246019622689368A7
:109B000003EA0803BB4201D100203AE0B8F5C06F78
:109B100007D137B99BF80C30DBB28DF803309DF8D4
:109B20000330B9F1FF3FEAD0FAF728F8A0EB0A00BA
:109B3000A84229D323685A6822F0E0025A6062687A
:109B4000B2F5827F0AD1A268B2F5004F02D0B2F519
:109B5000806F03D11A6822F040021A60A26AB2F53F
:109B6000005F07D11A6822F400521A601A6842F4A2
:109B700000521A60012384F85D30002384F85C30C1
:109B8000032003B0BDE8F08F019A019B002A03F186
:109B9000FF33019308BF1546B0E700BFA8030020BC
:109BA00073B50B4600920D4616464FF4C051002285
:109BB0000446FFF789FF024630B1236E43F02003CD
:109BC0002366032002B070BD00962B4680212046FC
:109BD000FFF71EFF02460028EFD100962B464FF4F8
:109BE000C0612046FFF770FF0028EBD0E5E743682F
:109BF000B3F5827FF7B504460E4617460BD183684E
:109C0000B3F5004F02D0B3F5806F04D1226813681A
:109C100023F0400313600097334600228021204642
:109C2000FFF7F6FE054628B1236E43F020032366B6
:109C3000032514E06368B3F5827F10D1A368B3F500
:109C4000004F02D0B3F5806F09D100973346002250
:109C50004FF4C0612046FFF737FF0028E4D12846C3
:109C600003B0F0BDF8B5044600287ED0436A002B4F
:109C700050D14268B2F5827F00D0C36194F85D3064
:109C800003F0FF0223B984F85C202046F9F7F8FAC4
:109C90002268E068022384F85D301368B0F5E06F55
:109CA00023F0400313604FF0000337D91D46B0F591
:109CB000706F18BFA362A7686368A169A66A07F4FA
:109CC000044703F482733B43276907F002073B43D1
:109CD000676907F001073B4301F400773B43E769FD
:109CE00007F038073B43276A07F080073B4306F439
:109CF00000573B43B6F5005F136014D1236B8BBB59
:109D0000B0F5E06F0DD902232363136843F40063B9
:109D1000136008E00023C0E90433AFE74FF4805537
:109D2000C7E701232363636A676B03F0100307F03F
:109D3000080700F470603B43090C034301F0040181
:109D40000B432B43B6F5005F536004BFA38D136133
:109D5000D36923F40063D36100200123206684F8D3
:109D60005D30F8BD022BDED1CFE70120F9E700001E
:109D700070B5044690F85C00012800F0CF80012007
:109D800084F85C0094F85D0066680128C5B20AD0CA
:109D9000B6F5827F40F0C080A068002840F0BC800B
:109DA000042D40F0B980002951D0002A4FD0002B5B
:109DB0004DD094F85D00A16304281CBF052084F8F1
:109DC0005D0000202066C4E91300A06AE387B0F5B7
:109DD000005F2168A3872264A4F84430A4F84630C9
:109DE00007D1086820F400500860086840F400506B
:109DF0000860486820F4C0404860E068B0F5E06F53
:109E0000A06D29D94B6823F480534B6094F85D30E2
:109E1000434E444D042B444B18BF1D46434B18BFC3
:109E20003346C0E90B35424B436300238363B4F8E8
:109E300046300C319BB2FEF785FA0346002848D025
:109E4000236E43F010032366012384F85D30012064
:109E5000002384F85C3070BD4D6845F480554D603A
:109E6000656DAD69B5F5806F0AD113F0010F4B68D0
:109E70001ED123F480434B60E38FC3F34E03E3878B
:109E80008369B3F5806FC1D14B6823F480534B6075
:109E9000B4F8463013F0010F4B6811D123F400538E
:109EA0004B60B4F84630C3F34E03A4F84630ADE738
:109EB00043F480434B60E38FC3F34E030133DEE78B
:109EC00043F400534B60B4F84630C3F34E03013300
:109ED000EBE72268606D516841F001015160C0E913
:109EE0000B33C0E90D33E38FA16B9BB20C32FEF74D
:109EF00029FA0028A4D123681A6852065EBF1A689E
:109F000042F040021A605A6842F020025A605A68D1
:109F100042F002025A609BE7022099E702209AE78A
:109F200069A00008399F0008459F0008739F00083A
:109F3000519F00087047704708B5806AFFF7FBFF24
:109F400008BD704708B5806AFFF7FBFF08BD704782
:109F5000806A026808B5536823F003035360036EF8
:109F600043F010030366012380F85D30FFF7EFFF35
:109F700008BD7FB5064600230393846A8DF80B3035
:109F8000F9F7FCFD33681B689A06054668D4226819
:109F9000536823F020035360A36AB3F5005F13D125
:109FA00001220090642311462046FFF731FD18B1CD
:109FB000236E43F002032366E3682668B3F5E06F7F
:109FC0002ED9F3680393039BA2682368002A43D128
:109FD0006268B2F5827F3FD15A6822F003025A606C
:109FE00064212A462046FFF702FE08B1202323669B
:109FF0000023A4F846302268012384F85D3093687A
:10A00000DB0606D5236E43F0020323664FF6EF739B
:10A010009360236E23B32046FFF799FF04B070BD11
:10A02000337BDBB28DF80B309DF80B30236B022BAA
:10A03000CAD101220095642311462046FFF7E8FCAF
:10A0400018B1236E43F002032366337BDBB28DF835
:10A050000B309DF80B30B7E75A6822F00102BEE7DB
:10A060002046FFF767FFD9E77FB506460023039335
:10A07000846A8DF80B30F9F781FD33681B68990607
:10A0800005465ED42268536823F020035360A36A18
:10A09000B3F5005F1BD1E368B3F5E06F3ED1236BEE
:10A0A000012B3BD1009064234FF400724FF4C06148
:10A0B0002046FFF709FD18B1236E43F00203236623
:10A0C00023681B7BDBB28DF80B309DF80B302A46E2
:10A0D00064212046FFF764FD18B1236E43F020038E
:10A0E000236623685A6822F003025A600022E2873E
:10A0F000A4F84620012284F85D209A68D20606D58D
:10A10000226E42F0020222664FF6EF729A60236ED0
:10A11000BBB12046FFF71BFF04B070BD0095642360
:10A120004FF480624FF4C0612046FFF7CDFC18B1B8
:10A13000236E43F0020323662368DB680393039BCB
:10A14000C5E72046F8F7B8FBE6E70000036830B53E
:10A1500059689A6802F04105012D85B0044606D180
:10A160004D0604D5C36C05B0BDE8304018479507CF
:10A1700004D5080602D5236D2046F4E712F4B07F1B
:10A1800059D08D0657D550060FD594F85D00032899
:10A190004FF0000549D0206E40F004002066009585
:10A1A000D868009098680090009895060CD5206EAD
:10A1B00040F0010020660020029098680290186824
:10A1C00020F0400018600298D00508D5226E42F0B9
:10A1D00008022266002203929A680392039A226E72
:10A1E0004AB35A6822F0E0025A60012284F85D20E6
:10A1F0008A0722D05A68A06D22F003025A6040B14B
:10A20000104B8363FEF717F918B1236E43F0400338
:10A210002366606D78B10B4B8363FEF70CF950B188
:10A22000236E43F04003236605E00195DA6801924E
:10A230009B680193019B05B030BD2046FFF787FE68
:10A24000F9E700BF49A2000808B5806A0023A0F81A
:10A250004630C387FFF77BFE08BD0000034AD2F8F3
:10A26000903043F40043C2F8903070470004005827
:10A27000034AD2F8903023F40043C2F8903070477C
:10A2800000040058074B1A6822F040021A6040F49C
:10A2900041704FF4B85218605A601A6842F0400298
:10A2A0001A6070470000015837B5054600284ED0A7
:10A2B000837903F0FF046BB1032C0BD0254B4FF4D3
:10A2C00000629A612868FFF7DDFF002401232B71EB
:10A2D000AC602FE000236B712846F9F763FB1E4A40
:10A2E000D2F8903043F48053C2F89030002CE5D17E
:10A2F00002234FF0B042AB71D2F8943023F4004304
:10A30000C2F89430154B1B681C214B43DB0C6421B5
:10A310004B430193019B93B90124AC60FFF79EFF6F
:10A320000C4B9A6842F400629A604FF400629A61A2
:10A33000002CC7D00123AB71204603B030BD019B78
:10A34000013B0193D2F894305B04E3D4E6E70124A7
:10A35000F2E700BF0004005800080058A8030020DE
:10A3600037B5174D2B6802461C204343DB0C642095
:10A37000434314480193019B93B901209060114C11
:10A3800021732B681C214B43DB0C64214B4301934D
:10A39000019B6BB9012090600A4BDB6803B030BDB4
:10A3A000019B013B019383689C07E4D50020E6E70D
:10A3B000019B013B0193A368DB07E9D5ECE700BFF4
:10A3C000A80300200000015837B5184D2B6802463D
:10A3D0001C204343DB0C6420434315480193019B3D
:10A3E000A3B901209060124CFF2323732B681C2516
:10A3F0006B43DB0C64256B430193019B73B9012014
:10A4000090600B4BDB680B7003B030BD019B013BD0
:10A41000019383689C07E2D50020E4E7019B013BA0
:10A420000193A368DB07E8D5EBE700BFA803002092
:10A43000000001580E4B0F491B681822534382B08D
:10A440001B0D6422534301934B69019AC3F38003AC
:10A4500022B902238360012002B07047019A013AB9
:10A4600001924A69920701D5002BEDD10020F3E754
:10A47000A80300200004005807B50379012B0FD171
:10A480000A4B1B68182253431B0C0193FFF7F0FE85
:10A49000019B013B0193019B002BF9D1FFF7DEFEED
:10A4A00003B05DF804EBFFF7C5BF00BFA8030020B1
:10A4B000F8B51E468379012B154604460F46DAB2DD
:10A4C0002DD14379012B2AD0022342718371FFF7EA
:10A4D000D3FF0D212046FFF7CBFEFFF741FF390ADE
:10A4E0002046FFF73DFFF9B22046FFF739FF2E4423
:10A4F000B5420ED12046FFF7B1FEFFF79BFFA068E3
:10A5000001230038A3714FF0000318BF01206371CD
:10A51000F8BD15F8011B2046FFF722FFE8E70220EF
:10A52000F6E7F8B51E468379012B154604460F461B
:10A53000DAB22FD14379012B2CD04271FFF79CFF67
:10A540001D212046FFF794FEFFF70AFF390A204637
:10A55000FFF706FFF9B22046FFF702FF0021204671
:10A56000FFF7FEFE2E44B5420ED12046FFF776FEE1
:10A57000FFF760FFA06801230038A3714FF00003CC
:10A5800018BF01206371F8BD29462046FFF71CFF64
:10A590000135E8E70220F6E7F8B51F468379012B7D
:10A5A000154604460E46DAB22CD14379012B29D048
:10A5B0004271FFF761FF06F0EF03A3F184025342FB
:10A5C0005341237131462046FFF752FEFFF7C8FE84
:10A5D0002F44AF4210D1FFF741FE842E02D0204617
:10A5E000FFF728FFA06801230038A3714FF0000394
:10A5F00018BF01206371F8BD15F8011B2046FFF755
:10A60000AFFEE6E70220F6E7F8B51E468379012B98
:10A61000154604460F46DAB227D14379012B24D0E0
:10A620004271FFF729FF39462046FFF721FEFFF769
:10A6300097FE00212046FFF793FE2E44B5420ED12F
:10A640002046FFF70BFEFFF7F5FEA0680123003858
:10A65000A3714FF0000318BF01206371F8BD2946B4
:10A660002046FFF7B1FE0135E8E70220F6E737B5EF
:10A670000023ADF8043001AA022312210546FFF79A
:10A68000C3FFBDF80440022364BA01AAA4B219466C
:10A690002846FFF781FFE20702D528460AF094FF1B
:10A6A000A30702D528460AF095FF600702D5284681
:10A6B0000AF0BAFF210702D528460AF0BBFFE206DE
:10A6C00002D528460AF0BCFFA30602D528460AF0A8
:10A6D000A5FF600602D528460AF082FF210606D5AE
:10A6E00014F4807118BF012128460AF07FFFA205EB
:10A6F00002D528460AF08AFF630402D528460AF0EC
:10A70000A5FF03B030BDF8B51E468379012B154671
:10A7100004460F46DAB227D14379012B24D0427187
:10A72000FFF7AAFE0E212046FFF7A2FDFFF718FE55
:10A7300039462046FFF714FE2E44B5420ED120467E
:10A74000FFF78CFDFFF776FEA06801230038A371A8
:10A750004FF0000318BF01206371F8BD15F8011B0D
:10A760002046FFF7FDFDE8E70220F6E7F8B51E46B4
:10A770008379012B154604460F46DAB22BD1437973
:10A78000012B28D04271FFF777FE1E212046FFF7EC
:10A790006FFDFFF7E5FD39462046FFF7E1FD00219B
:10A7A0002046FFF7DDFD2E44B5420ED12046FFF7CF
:10A7B00055FDFFF73FFEA06801230038A3714FF05D
:10A7C000000318BF01206371F8BD29462046FFF73A
:10A7D000FBFD0135E8E70220F6E70000036A23F0FD
:10A7E00001030362036A70B5446882690D6822F44C
:10A7F000803222F073022A438D6823F002032B4338
:10A80000124DA84206D0124EB04203D0A6F5806683
:10A81000B04214D1CE6823F008033343A84223F09A
:10A82000040306D00B4DA84203D005F58065A8426D
:10A8300005D124F44075D1E9054634432C434460E6
:10A8400082614A684263036270BD00BF002C014010
:10A850000048014000440140036A23F4807303620E
:10A86000036A426870B5C4690D6824F4803424F02A
:10A8700073042C438D6823F4007343EA05230F4DC2
:10A88000A8420ED1CD6823F4006343EA052323F4E4
:10A890008063D1E9055622F44052354342EA05125D
:10A8A00006E0074DA842F4D005F58065A842F0D037
:10A8B00042604A68C461C263036270BD002C0140FB
:10A8C00000440140036A23F480530362026A30B5F6
:10A8D0004468C3690D6823F0807323F4E64343EAB8
:10A8E00005238D6822F4005242EA05320A4DA8423F
:10A8F00007D005F5C055A84203D005F58065A842EC
:10A9000004D14D6924F4804444EA85144460C36151
:10A910004B680364026230BD002C0140036A23F4DB
:10A9200080330362026A30B54468436D0D6823F4D6
:10A93000803323F070032B438D6822F4003242EA07
:10A9400005420B4DA84207D005F5C055A84203D0DB
:10A9500005F58065A84204D14D6924F4803444EAA9
:10A960000524446043654B688365026230BD00BFC7
:10A97000002C0140036A23F480130362026A30B59D
:10A980004468436D0D6823F0807323F4E04343EA89
:10A9900005238D6822F4001242EA05520A4DA842AE
:10A9A00007D005F5C055A84203D005F58065A8423B
:10A9B00004D14D6924F4802444EA8524446043652D
:10A9C0004B68C365026230BD002C0140704710B572
:10A9D000846A626A82420BD101232377D2690AB961
:10A9E00084F83E302046F8F7A1FF0023237710BDFE
:10A9F000A36A834208D102222277DB69002BF1D1BE
:10AA0000012384F83F30EDE7E36A834208D1042252
:10AA10002277DB69002BE5D1012384F84030E1E7A0
:10AA2000236B8342DED108222277DB69002BD9D148
:10AA3000012384F84130D5E7704710B5846A636A12
:10AA4000834207D1012323772046FFF7F5FF002338
:10AA5000237710BDA36A834201D10223F3E7E36A9F
:10AA6000834201D10423EEE7236B8342ECD1082318
:10AA7000E9E7704710B5846A636A834209D101230C
:10AA8000237784F83E302046FFF7F3FF0023237737
:10AA900010BDA36A834205D102232377012384F8E2
:10AAA0003F30F0E7E36A83424FF0010304D1042210
:10AAB000227784F84030E6E7226B824203BF082207
:10AAC000227784F8413084F83D30DCE71A4A036885
:10AAD000904210B502D0B0F1804F09D14C6823F0FC
:10AAE0007003904243EA040309D0B0F1804F06D0CE
:10AAF000124A904203D002F58062904203D1CA68A4
:10AB000023F4407313434A6923F080031343036023
:10AB10008B68C3620B688362074B984207D003F5CA
:10AB2000C053984203D003F58063984201D10B696A
:10AB300003630123436110BD002C01400044014028
:10AB400010B5044650B390F83D3003F0FF021BB936
:10AB500080F83C20F9F7EAF80223206884F83D30B9
:10AB6000211DFFF7B3FF012384F84830002084F84B
:10AB70003E3084F83F3084F8403084F8413084F827
:10AB8000423084F8433084F8443084F8453084F807
:10AB9000463084F8473084F83D3010BD0120FCE792
:10ABA00010B5044650B390F83D3003F0FF021BB9D6
:10ABB00080F83C20FFF70AFF0223206884F83D302C
:10ABC000211DFFF783FF012384F84830002084F81B
:10ABD0003E3084F83F3084F8403084F8413084F8C7
:10ABE000423084F8433084F8443084F8453084F8A7
:10ABF000463084F8473084F83D3010BD0120FCE732
:10AC0000036A23F010030362036A426870B5846923
:10AC10000D6824F0807424F4E64444EA05248D6829
:10AC200023F0200343EA05130F4DA8420ED1CD684F
:10AC300023F0800343EA051323F04003D1E90556CE
:10AC400022F44062354342EA850206E0074DA842FD
:10AC5000F4D005F58065A842F0D042604A6884616E
:10AC60008263036270BD00BF002C014000440140BC
:10AC700038B590F83C30012B044673D001200C2AE3
:10AC800084F83C004ED008D8042A2BD0082A39D0AA
:10AC9000BAB1002384F83C3038BD102A52D0142AAF
:10ACA000F7D12068FFF766FE436D0A6943F400633D
:10ACB0004365436D23F480634365436D43EA022398
:10ACC0004EE02068FFF78AFD83690A6943F00803B4
:10ACD0008361836923F00403836183691343836180
:10ACE0000020D6E72068FFF78BFF83690A6943F4E9
:10ACF00000638361836923F480638361836943EA2A
:10AD00000223ECE72068FFF7A7FDC3690A6943F057
:10AD10000803C361C36923F00403C361C369134318
:10AD2000C361DDE72068FFF7CDFDC3690A6943F41D
:10AD30000063C361C36923F48063C361C36943EAE9
:10AD40000223EDE72068FFF7E9FD436D0A6943F050
:10AD500008034365436D23F004034365436D1343C8
:10AD60004365BDE7022097E710B584680A4324F4E1
:10AD70007F4442EA03222243826010BD38B590F836
:10AD80003C30012B04464FF0020000F0958084F81F
:10AD90003D000122206884F83C208568474B2B4009
:10ADA00083600B68602B54D037D8402B6BD019D8F8
:10ADB000202B0DD00AD833F0100109D0012384F8DC
:10ADC0003D30002384F83C30104638BD302BF5D19F
:10ADD000826822F4401222F070021A4342F0070205
:10ADE00082602BE0502BE9D14A68CD68016A036A82
:10ADF00023F001030362836921F00A0123F0F003C9
:10AE000043EA05130A4383610262836823F4401313
:10AE100023F0700343F057030FE0B3F5805F0DD0CC
:10AE2000B3F5005F0CD0702BC8D1CB68D1E90121FC
:10AE3000FFF79AFF836843F0770383600022BDE742
:10AE4000CB68D1E90121FFF78FFF836843F480438A
:10AE5000F3E7036A4D68C96823F01003036282694F
:10AE6000036A22F4704223F0A00343EA051342EA86
:10AE7000013282610362836823F4401323F070037C
:10AE800043F06703D9E74A68CD68016A036A23F093
:10AE900001030362836921F00A0123F0F00343EA0E
:10AEA00005130A4383610262836823F4401323F08D
:10AEB000700343F04703C0E7024685E78800CEFFF2
:10AEC000036A01F01F0110B501248C4023EA04033A
:10AED0000362036A8A401A43026210BD38B50D4608
:10AEE000082D044611461BD005D85DB1042D14D0A1
:10AEF00094F8430008E00C2D15D0102DF8D190F8EF
:10AF0000420001E090F83E00A0F1020CDCF10000EC
:10AF100040EB0C0050B1022076E090F83F00F3E7E0
:10AF200090F84000F0E790F84100EDE7082D1AD0C6
:10AF300007D86DB1042D13D094F84320012A19D0FD
:10AF40000CE00C2D27D0102DF6D194F842000CE027
:10AF500094F83E20501E424242415AB9012053E02B
:10AF600094F83F20F6E794F84000421E50425041CA
:10AF70000028F3D00029F1D0002BEFD0082D4FF09E
:10AF8000020256D00AD885B1042D3ED0042D84F893
:10AF90004320E3D13BE094F84100E6E70C2D5CD080
:10AFA000102DF3D184F84220D8E7606A84F83E205F
:10AFB0003A4AC2623A4A02633A4A426322683432E7
:10AFC000FDF7C0F90028C9D12268D36843F40073A3
:10AFD0002068D36029460122FFF772FF324A90426F
:10AFE00050D0324B98424DD003F58063984249D0FF
:10AFF000B0F1804F4DD182682D4B1340062B02D00B
:10B00000B3F5803F45D1002038BD84F83F20A06AC9
:10B01000224AC262224A0263224A426322683832CA
:10B02000FDF790F9002899D12268D36843F4806332
:10B03000CEE7E06A84F84020184AC262184A0263E8
:10B04000184A426322683C32FDF77CF9002885D11A
:10B050002268D36843F40063BAE7206B84F8412088
:10B060000E4AC2620E4A02630E4A426322684032AE
:10B07000FDF768F900287FF471AF2268D36843F4C4
:10B080008053A5E7436C904243F400434364B2D03D
:10B09000AEE7036843F001030360B4E7CFA90008FB
:10B0A0003BAA000875AA0008002C0140004401409A
:10B0B00007000100FFF712BF082938B504460D4606
:10B0C0004FD004D861B1042944D0012038BD0C29E7
:10B0D000FBD10268006BD36823F48053D36005E092
:10B0E0000268406AD36823F40073D360FDF7A3F9C4
:10B0F000206800222946FFF7E3FE2A4B984207D03A
:10B1000003F5C053984203D003F5806398420DD1F4
:10B11000026A41F211131A4208D1026A40F2444312
:10B120001A4202BF436C23F400434364026A41F2B3
:10B1300011131A4208D1026A40F244431A4202BF74
:10B14000036823F00103036001238DB984F83E30C6
:10B150000020BBE70268806AD36823F48063D36071
:10B16000C4E70268C06AD36823F40063D360BDE714
:10B170000C2D13D007D8042D0AD0082D0BD0012395
:10B1800084F84330E4E7102DF9D184F84230DFE74A
:10B1900084F83F30DCE784F84030D9E784F8413068
:10B1A000D6E700BF002C0140FFF786BF70B590F8CE
:10B1B0003C30012B02464FF0020020D082F83D00C7
:10B1C0000F4D106843688468A84202BF4E6823F49C
:10B1D000700333430E6823F070033343A842436087
:10B1E00002D0B0F1804F04D1896824F080030B4372
:10B1F00083600123002082F83D3082F83C0070BD5E
:10B20000002C014010B590F83C30012B02463BD099
:10B21000CB6888681D4C23F440730343486823F4CB
:10B2200080630343086823F400630343086923F43D
:10B2300080530343486923F400530343086B23F40A
:10B2400080430343886923F4702343EA0043106872
:10B25000A04214D1CC6923F0805323438C6A23F499
:10B26000700343EA04530C6A23F0807323434C6A4F
:10B27000C96A23F00073234323F000530B43436454
:10B28000002082F83C0010BD0220FCE7002C0140A9
:10B29000026852E8003F23F0C00342E80031026830
:10B2A0000029F5D102F1080353E8003F23F400031D
:10B2B00002F1080C4CE800310029F3D12023C0F83A
:10B2C0008830704710B5026852E8003F23F490734D
:10B2D00042E8003102680029F5D10F4C02F1080361
:10B2E00053E8003F234002F1080C4CE800310029EC
:10B2F000F4D1C36E012B07D152E8003F23F01003B5
:10B3000042E800310029F7D12023C0F88C30002317
:10B31000C366436710BD00BFFEFFFFEFF8B50446EC
:10B320001346D4F88850202D32D1F1B1EAB1E06F44
:10B33000A4F85620A4F8542000262122C4F89060D6
:10B340002165C4F88820226888B1124FC762124F65
:10B350000763124F2832C0E90D76FCF7F3FF30B1D6
:10B360001023C4F89030C4F888500120F8BD236839
:10B3700040221A62226802F1080353E8003F43F0BA
:10B38000800302F1080141E800300028F3D1EDE725
:10B390000220EBE7A1B30008E9B30008F5B3000809
:10B3A00008B50346806A1B681B6813F0200317D199
:10B3B000A0F85630026802F1080353E8003F23F07A
:10B3C0008003083242E8003102680029F2D152E8D5
:10B3D000003F43F0400342E800310029F7D108BDA7
:10B3E000F8F796FFFBE7704708B5806AFFF7FBFFA9
:10B3F00008BD7047806A38B50468D0F88830D0F846
:10B400008C50A268120606D5212B04D10023A0F887
:10B410005630FFF73DFFA3685B0606D5222D04D109
:10B420000023A0F85E30FFF74DFFD0F8903043F0D6
:10B430001003C0F89030FFF7DCFF38BD08B5806A14
:10B440000023A0F85E30A0F85630FFF7D2FF08BD09
:10B45000704700000368D9691A682DE9F04140F689
:10B460000F0631429D68044610D18E0640F1978048
:10B4700002F0200605F080573E4300F09080436FB5
:10B48000002B00F08580BDE8F0411847AB4EAC487A
:10B490002E401040304300F08280CF0709D5D00500
:10B4A00007D501201862D4F8900040F00100C4F8DC
:10B4B00090008F0709D5E80707D502201862D4F855
:10B4C000900040F00400C4F890004F0709D5E80749
:10B4D00007D504201862D4F8900040F00200C4F8A8
:10B4E00090000F070BD502F02000304307D0082052
:10B4F0001862D4F8900040F00800C4F890000E05DF
:10B500000AD5500108D54FF400601862D4F8903085
:10B5100043F02003C4F89030D4F89030002B37D09B
:10B520008B0609D502F0200205F080552A4303D08E
:10B53000636F0BB1204698472668D4F89020B36813
:10B5400002F0280203F0400353EA0205204621D00E
:10B55000FFF7B8FEB3685F0617D5226802F108034B
:10B5600053E8003F23F04003083242E8003100294D
:10B57000F3D1D4F8800040B1724B8363FCF75BFFDA
:10B5800030B1D4F88000836B7DE72046FFF731FFB0
:10B59000BDE8F081FFF72DFFC4F89050F8E7E06EAA
:10B5A000012840F08980CE0640F18680D00640F127
:10B5B000838010221A629A6851064BD5D4F88020F5
:10B5C00011684A6892B2002AE2D0B4F85C00904256
:10B5D000DED9A4F85E200A6892062FD453E8002F23
:10B5E00022F4807243E800210029F7D103F1080218
:10B5F00052E8002F22F0010203F1080040E8002188
:10B600000029F3D103F1080252E8002F22F0400292
:10B6100003F1080040E800210029F3D12022C4F8FA
:10B620008C20E16653E8002F22F0100243E800214D
:10B630000029F7D1D4F88000FCF7C8FE0223236765
:10B64000B4F85E30B4F85C10C91A89B22046FFF72E
:10B65000FFFE9DE7B4F85E20B4F85E00B4F85C101D
:10B6600080B292B2002893D0891A89B200298FD073
:10B6700053E8002F22F4907243E800200028F7D10D
:10B68000314D03F1080252E8002F2A4003F1080669
:10B6900046E800200028F4D12022C4F88C206067FE
:10B6A000E06653E8002F22F0100243E80020002853
:10B6B000F7D102232367C9E7CF0209D56E0207D568
:10B6C0004FF4801220461A62BDE8F04100F0A0BDA0
:10B6D00008060BD502F0800005F40005284305D0CC
:10B6E000A36F002B3FF454AF2046CCE64F0611D594
:10B6F00056060FD553E8002F22F0400243E8002100
:10B700000029F7D12023C4F88830A1672046F8F734
:10B71000FFFD3DE70D0206D5500004D52046BDE8EB
:10B72000F04100F077BDCB017FF532AF002ABFF6C4
:10B730002FAF2046BDE8F04100F06BBD01000010C6
:10B74000200100043DB40008FEFFFFEFD0F88C207C
:10B75000B0F86010222A08B5036855D15B6A826D83
:10B760000B401370836D01338365B0F85E30013B8D
:10B770009BB2A0F85E30B0F85E309BB2002B42D195
:10B78000026852E8003F23F4907342E800310368F6
:10B790000029F5D103F1080252E8002F22F001023E
:10B7A00003F1080C4CE800210029F3D12022C0F855
:10B7B0008C20184A41679342016705D1C26E012A65
:10B7C0000ED0F8F7B3FD1EE05A681102F6D553E823
:10B7D000002F22F0806243E800210029F7D1EDE735
:10B7E0000022C26653E8002F22F0100243E8002135
:10B7F0000029F7D1DA69B0F85C10D20644BF1022F4
:10B800001A62FFF725FE08BD9A6942F008029A61A4
:10B81000F9E700BF00800040D0F88C20B0F860103D
:10B82000222A08B5036852D15A6A1140826D22F863
:10B83000021B8265B0F85E20013A92B2A0F85E2049
:10B84000B0F85E2092B2002A40D153E8002F22F4D3
:10B85000907243E800210029F7D103F1080252E871
:10B86000002F22F0010203F1080C4CE8002100290E
:10B87000F3D12022C0F88C20174A41679342016718
:10B8800005D1C26E012A0ED0F8F750FD1EE05A68AD
:10B890001102F6D553E8002F22F0806243E8002120
:10B8A0000029F7D1EDE70022C26653E8002F22F00D
:10B8B000100243E800210029F7D1DA69B0F85C10E2
:10B8C000D20644BF10221A62FFF7C2FD08BD9A6972
:10B8D00042F008029A61F9E7008000402DE9F84F34
:10B8E0000368B0F86060D3F81CB01F689D68D0F89A
:10B8F0008C20222A044640F0B980B0F8683043B169
:10B90000DFF87491DFF874A14FF000081BF0200FEE
:10B9100020D1B4F85E309BB2D3B1B4F868209A421B
:10B9200016D9226802F1080353E8003F23F0805340
:10B93000083242E8003122680029F2D1504B636797
:10B9400052E8003F43F0200342E800310029F7D1DC
:10B95000BDE8F88F2368A26D5B6A33401370A36D56
:10B960000133A365B4F85E30013B9BB2A4F85E30AE
:10B970002368D3F81CB01BF0070F2ED01BF0010F6B
:10B9800009D0F90507D501221A62D4F8902042F0B7
:10B990000102C4F890201BF0020F09D0EA0707D576
:10B9A00002221A62D4F8902042F00402C4F89020D7
:10B9B0001BF0040F09D0E80707D504221A62D4F857
:10B9C000903043F00203C4F89030D4F8903023B1A3
:10B9D0002046FFF70EFDC4F89080B4F85E309BB2AD
:10B9E000002B93D1226852E8003F23F4807342E891
:10B9F000003123680029F5D103F1080252E8002F35
:10BA000002EA090203F1080040E800210029F3D10D
:10BA100020225345C4F88C20616721670AD05A68F8
:10BA2000110207D553E8002F22F0806243E800217D
:10BA30000029F7D1E26E012A14D10022E26653E810
:10BA4000002F22F0100243E800210029F7D1DA6923
:10BA5000B4F85C10D20644BF10221A622046FFF7E9
:10BA6000F7FC53E72046F8F761FC4FE79A6942F08C
:10BA700008029A616CE700BFFEFFFFEF0080004004
:10BA80004DB700082DE9F84F0368B0F86060D3F8AF
:10BA90001CB01F689D68D0F88C20222A044640F014
:10BAA000B780B0F8683043B1DFF87091DFF870A16B
:10BAB0004FF000081BF0200F20D1B4F85E309BB28D
:10BAC000D3B1B4F868209A4216D9226802F108036B
:10BAD00053E8003F23F08053083242E800312268E7
:10BAE0000029F2D14F4B636752E8003F43F0200337
:10BAF00042E800310029F7D1BDE8F88F2368A26D34
:10BB0000596A314022F8021BA265B4F85E20013A5E
:10BB100092B2A4F85E20D3F81CB01BF0070F2ED011
:10BB20001BF0010F09D0F90507D501221A62D4F8DC
:10BB3000902042F00102C4F890201BF0020F09D0BF
:10BB4000EA0707D502221A62D4F8902042F00402D4
:10BB5000C4F890201BF0040F09D0E80707D5042291
:10BB60001A62D4F8903043F00203C4F89030D4F84D
:10BB7000903023B12046FFF73CFCC4F89080B4F825
:10BB80005E309BB2002B95D1226852E8003F23F42F
:10BB9000807342E8003123680029F5D103F10802DF
:10BBA00052E8002F02EA090203F1080040E80021F0
:10BBB0000029F3D120225345C4F88C206167216706
:10BBC0000AD05A68110207D553E8002F22F080628C
:10BBD00043E800210029F7D1E26E012A14D10022A6
:10BBE000E26653E8002F22F0100243E8002100290A
:10BBF000F7D1DA69B4F85C10D20644BF10221A6299
:10BC00002046FFF725FC55E72046F8F78FFB51E764
:10BC10009A6942F008029A616EE700BFFEFFFFEFEB
:10BC20000080004019B8000838B50446036821694F
:10BC3000A2681D68C0690A4361690A4377490243E3
:10BC400029400A431A605A68E16822F440520A43C4
:10BC50005A60734AA16993421CBF226A11439A68D1
:10BC600022F06E4222F430620A439A60DA6A616A14
:10BC700022F00F020A43DA626A4A934219D14FF066
:10BC8000B043694AD3F8883003F0030343F44033E8
:10BC9000934200F0B480B3F1031F24D0013A9342E1
:10BCA00040F0B580B0F5004F40F08F80FCF780FF8A
:10BCB0006EE05E4A93421CD14FF0B0435C49D3F82A
:10BCC000883003F00C0343F440228A4200F097804E
:10BCD00006D8002B7CD0574B9A42E3D0012026E0B7
:10BCE000B2F10C1FFAD1B0F5004F53D04FF4004021
:10BCF00075E04B4A9342F1D14FF0B043D3F888300E
:10BD000003F44063B3F5006F18D006D85BB1B3F508
:10BD1000806FE3D1FCF74CFF07E0B3F5406FDDD156
:10BD20004FF400400BE0FDF73BFB40B900204FF023
:10BD30000113A3660023C4E91D3338BD3E4865687E
:10BD40003E4B626A05EB450133F81220B0FBF2F37B
:10BD50009942C3D8B3EB053FC0D800231946F6F784
:10BD6000A3FB090241EA10616B080002C0182A46D1
:10BD70004FF0000341F10001F6F796FB304BA0F5C0
:10BD800040729A42AAD82368D860CFE7FDF708FB33
:10BD90000028CBD06168294B626A33F81220B0FBCF
:10BDA000F2F24B0803EB42034FF6EF72B3FBF1F3F1
:10BDB000A3F11001914291D823F00F02216892B2B1
:10BDC000C3F342031343CB60B0E7FCF7F1FE04E09A
:10BDD000B0F5004FDAD0FDF7E3FA0028A6D063688B
:10BDE000616A164A32F81120B0FBF2F000EB530002
:10BDF000B0FBF3F04FF6EF73A0F11002C1E7B0F51E
:10BE0000004F0D48EBD1C5E7FDF7DAFAC0E7B0F512
:10BE1000004FF9D0FDF7D4FADFE700BFF369FFCF99
:10BE20000080004000380140020003000044004050
:10BE300008000C0004000C000024F40058820308E1
:10BE4000FFFC0F00836ADA0710B506D50168C46AE3
:10BE50004A6822F4003222434A609C0706D50168F2
:10BE6000046B4A6822F4803222434A60590706D59F
:10BE70000168446B4A6822F4802222434A601A0710
:10BE800006D50168846B4A6822F4004222434A6066
:10BE9000DC0606D50168C46B8A6822F4805222430E
:10BEA0008A60990606D50168046C8A6822F40052FB
:10BEB00022438A605A060FD50168446C4A6822F40E
:10BEC00080122243B4F5801F4A6005D14A68846C11
:10BED00022F4C00222434A601B0606D50268C16CE8
:10BEE000536823F400230B43536010BD2DE9F8433E
:10BEF000DDF8209005460F46164698462A68D36915
:10BF000037EA03030CBF01230023B34201D0002012
:10BF100029E0B9F1FF3FF2D0F7F730FEA0EB0800BF
:10BF200048452C6802D8B9F1000F1ED154E8003FF3
:10BF300023F4D07344E80032002AF7D104F1080357
:10BF400053E8003F23F0010304F1080141E8003207
:10BF5000002AF3D12023C5F88830C5F88C3000239F
:10BF600085F884300320BDE8F88323685A07C5D5D7
:10BF7000E3691B05C2D54FF40063236254E8003F18
:10BF800023F4D07344E80032002AF7D104F1080307
:10BF900053E8003F23F0010304F1080141E80032B7
:10BFA000002AF3D12023C5F88830C5F88C30C5F8B5
:10BFB0009030D4E773B504460026C0F89060F7F7D8
:10BFC000DDFD23681B681A07054619D423681B6822
:10BFD0005B070AD56FF07E43009300222B464FF497
:10BFE00080012046FFF782FFB0B900202023C4F86B
:10BFF000883084F88400C4F88C30E06620670CE058
:10C000006FF07E430093324603464FF40011204602
:10C01000FFF76CFF0028D9D0032002B070BD10B527
:10C02000044650B3D0F888301BB980F88430F8F754
:10C030007DF822682423C4F88830136823F00103B4
:10C0400013602046FFF7F0FD012816D0A36A13B154
:10C050002046FFF7F7FE23685A6822F490425A60A0
:10C060009A6822F02A029A601A6842F00102204679
:10C070001A60BDE81040FFF79DBF012010BD000011
:10C0800030B581658168A0F85C200023B1F5805F40
:10C09000A0F85E20436735D10369002B40F2FF13FF
:10C0A00018BFFF23A0F860300023C0F8903022238F
:10C0B000C0F88C30016801F1080353E8003F43F0F9
:10C0C0000103083141E800340368002CF2D1456EC9
:10C0D00084680169B5F1005F32D1B0F868509542CB
:10C0E0002ED8B4F5805F244A03D1244C002908BF20
:10C0F00022464267B1B153E8002F42F4807243E810
:10C100000021F7E729B90369002B14BF7F23FF2320
:10C11000C8E7B1F1805FC5D10369002B14BF3F238D
:10C120007F23BFE703F1080252E8002F42F080525C
:10C1300003F1080040E800210029F3D1002030BDC0
:10C14000B4F5805F0E4A03D10E4C002908BF224689
:10C15000426741B153E8002F42F4907243E8002156
:10C160000029F7D1EAE753E8002F42F0200243E824
:10C1700000210029F7D1E1E7DDB8000885BA000801
:10C180004DB7000819B80008D0F88C30202B30B417
:10C1900015D1B9B1B2B100230468C3660A4B9C4201
:10C1A0000AD063681B0207D554E8003F43F0806360
:10C1B00044E80035002DF7D130BCFFF761BF022005
:10C1C00030BC70470120FBE700800040436E30B573
:10C1D0002BB90123A0F86A30A0F8683030BD03689D
:10C1E000094D9A689968094C490FC2F342626B5C29
:10C1F000615CDB00B3FBF1F3A0F86A30AB5CA25CDE
:10C20000DB00B3FBF2F3E7E77882030870820308F0
:10C210007047704770471FB504AB03E9060090F8FC
:10C220008430012B04463AD0012380F88430242343
:10C23000C0F8883003681A6822F001021A609A6810
:10C2400022F440120A439A6071B95A68BDF80C0092
:10C250009DF80E1022F0100202435A605A6822F034
:10C260007F4242EA01625A601A6842F001021A6093
:10C27000F7F784FC6FF07E42034600924FF4800192
:10C2800000222046FFF732FE38B92023C4F8883058
:10C29000002384F8843004B010BD0320F8E70220A6
:10C2A000F9E790F88430012B0FD0012380F8843017
:10C2B000016851E8002F42F0020241E80023002B00
:10C2C000F6D180F88430184670470220704710B5C8
:10C2D00090F88430012B044617D02423C0F888300E
:10C2E00003681A68196821F00101196042F00052D0
:10C2F0004FF0005141661A60FFF768FF2023C0F835
:10C300008830002084F8840010BD0220FCE770B55E
:10C3100090F88430012B044617D005682423C0F818
:10C3200088302E682B6823F001032B60AB6823F064
:10C3300060431943A960FFF749FF20232E60C0F82E
:10C340008830002084F8840070BD0220FCE770B5BE
:10C3500090F88430012B044617D005682423C0F8D8
:10C3600088302E682B6823F001032B60AB6823F024
:10C3700060631943A960FFF729FF20232E60C0F8EE
:10C380008830002084F8840070BD0220FCE70000A3
:10C3900038B5084D052455F8043B2BB9013C14F081
:10C3A000FF04F8D1204638BDDB6898470028F5D057
:10C3B000F9E700BF58230020034BD870034B1B68DC
:10C3C0001B6C03B118477047402300203C2300201A
:10C3D000034B1874034B1B685B6C03B11847704721
:10C3E000402300203C230020F0B5314D314B95F91E
:10C3F0000420314E91B00C46012795F905108DF8B7
:10C40000047002288DF809208DF80A1010D18DF8DB
:10C410000800D8711C7203F075FB337803B114B1B6
:10C4200001A804F0A5F8254B059A1A6011B0F0BDDB
:10C4300059714FF480711A71D9801C7233788DF85C
:10C44000087053BB1F2306A88DF81C208DF81830E8
:10C4500003F036FD20238DF8183006A82B798DF8CF
:10C460001C3003F02DFD22238DF8183006A86B79BF
:10C470008DF81C3003F024FD21238DF8183006A818
:10C480006B798DF81C3003F01BFD29238DF81830D3
:10C4900006A80B4B079303F013FD03F033FB0123B6
:10C4A00006A88DF818308DF81C3003F009FDB4E7AC
:10C4B00040230020E00300201C2200201023002045
:10C4C000000400017FB5092301A88DF8043004F0B1
:10C4D0004FF80038044B059A1A6018BF01204042FB
:10C4E00007B05DF804FB00BF1023002070B50446C0
:10C4F0000B46144962784A700020A2780A720870CC
:10C500001A884A729A788A72DB780B746368CB60F7
:10C510000D4B1B68DA6A2AB1237803F0FB030A2B60
:10C5200000D09047094E002556F8043B1BB15B6ACA
:10C530000BB1204698470135EBB2052B6DB2F3D114
:10C5400070BD00BFB00300203C2300205823002012
:10C5500070B5044611480123037063784370A378D3
:10C560008372E368C360E3780376236943762379B3
:10C5700043720B4B1B689B6A03B19847094E002519
:10C5800056F8043B1BB19B690BB120469847013517
:10C59000EBB2052B6DB2F3D170BD00BFC403002018
:10C5A0003C23002058230020014B1868704700BF2F
:10C5B0001023002000B58BB0012368468DF80030B1
:10C5C00003F058FB38B99DF80400003818BF01206B
:10C5D0000BB05DF804FB0020FAE7000008B502F09C
:10C5E00049FC40B9FFF7E6FF012806D0054B197A50
:10C5F000D879FFF7F9FE012008BDBDE80840FFF734
:10C60000C7BE00BFE00300202DE9F04186B005461B
:10C610000E46174602F02EFC002873D102F042FCB1
:10C62000044640B9FFF7C6FF01280AD03D4B197AEE
:10C63000D879FFF7D9FE6FF00204204606B0BDE8B6
:10C64000F081DFF8E48088F80860003E18BF01261A
:10C650008DF80460354E687833798DF8123069466C
:10C6600003F0A6FA00283FD08DF804400394ADF8FB
:10C6700010406FF0060495E803002D4B83E803009B
:10C68000337988F80A30394601A804F075F8294B47
:10C69000059A1A6011283FD801A353F820F000BF73
:10C6A0000BC7000805C7000819C7000819C700080C
:10C6B00019C7000819C7000819C7000837C60008BD
:10C6C00019C7000819C7000819C70008FFC60008E5
:10C6D00019C7000819C7000805C7000805C70008E2
:10C6E00005C700081FC700082B788DF808306B7845
:10C6F000ADF810306B6803934FF0FF34BBE76FF079
:10C7000005049AE76FF0010497E70B4B00221A70BB
:10C71000E31D18BF144690E74FF0FF348DE76FF02C
:10C7200004048AE7E0030020C40300204023002023
:10C73000D4030020102300200F23002037B502F07F
:10C74000BBFB134D052455F8043B4BB11A693AB1B4
:10C750009B682BB1984718B155F8043C1B69984762
:10C76000013C14F0FF04EED1FFF712FE68B9094D49
:10C770002B7853B1084BADF80040D978019422468C
:10C780006846FFF741FF00B92C7003B030BD00BF11
:10C79000582300200F2300204023002030B58BB009
:10C7A000044602F067FB0546002835D1FFF702FF7B
:10C7B000012834D168468DF8005003F05BFA40BB85
:10C7C0009DF80430A34204D0012C22D0022C12D0B8
:10C7D00014B100200BB030BD002BFAD068468DF8A4
:10C7E000044003F06DFBA0B90E4B1B681B6B002BC4
:10C7F000EFD09847EDE763B968468DF8044003F041
:10C800005FFB30B9074B1B681B6B002BE1D0204648
:10C81000EFE74FF0FF30DDE76FF00100DAE76FF090
:10C820000200D7E73C23002010B504468AB018B9AF
:10C830004FF0FF300AB010BD002368468DF800307D
:10C8400003F018FA0028F3D19DF804302370F1E7C3
:10C850007FB500220B4620498DF8072001220A707F
:10C8600042784A700446002A33D102790A721A8843
:10C870004A729A788A72DB780B740369CB60C3784A
:10C88000164D8DF80830037B8DF8093083680393CB
:10C890002B68DB6A0BB102A898472B689B6B13B11E
:10C8A000227E02B198470E4E052556F8043B1BB177
:10C8B000DB690BB120469847013D15F0FF05F4D127
:10C8C0000DF10700FFF7B0FF637913B1054B0122AB
:10C8D0001A7004B070BD00BFB00300203C230020DC
:10C8E000582300200F23002010B504468AB018B941
:10C8F0004FF0FF300AB010BD202368468DF800309D
:10C9000003F0B8F90028F3D1024A9DF904302370EE
:10C910001371EFE74023002000B58BB02323019073
:10C9200068468DF8003003F0CBFA003818BF0120BC
:10C9300040420BB05DF804FB70B5654C01468EB00B
:10C940001822204606F0BCFF624B00221A70FAF74C
:10C950007FFE23784068012202FA03F1014004D1EE
:10C960005D4B084608F098FFFEE75C495C481A46B4
:10C9700002F00AFF18B14FF0FF300EB070BD272350
:10C9800004A88DF8103003F09BFA564E564D00283F
:10C9900070D1012333702B68DB690BB100209847FD
:10C9A000272304A88DF8103003F064F9059B93F851
:10C9B0004820227093F8182193F81A316270A370FE
:10C9C000464BD3E9020106F06BFE05460028D2D1A2
:10C9D000464E062304A88DF8103003F04BF9059B52
:10C9E000736104A803F06CFA022304A88DF81030D8
:10C9F000059603F03FF90836032304A88DF810309C
:10CA0000059603F037F90F2606F010FF012304A85E
:10CA10008DF814308DF8106003F052FA10230DEBEE
:10CA200003008DF810308DF8145003F049FA0423F8
:10CA30008DF8103004A8A3788DF8143003F040FA74
:10CA40003A238DF8103004A86369059303F038FA8F
:10CA500002A920788DF8086004F0CCFF003818BFD8
:10CA60000120E0711420FFF757FFE07904F046F849
:10CA7000284682E728238DF810302B681B6943B1C4
:10CA800004A803F0F7F82B6805981B6940F2C4511D
:10CA90009847272304A88DF8103003F011FA50B9F5
:10CAA000012304A88DF8103003F0E4F89DF8143049
:10CAB000002B7FF46EAF3378002B7FF46CAF052230
:10CAC00004A88DF81020059303F0FAF978E700BF69
:10CAD000402300200F23002080820308142300201D
:10CAE0002C2300201C2200203C2300207C2300203B
:10CAF00037B500230D4601930446D0B900F07CFD04
:10CB00000190019BD3B10F4A42F824300E4A9A6239
:10CB10000E4A1268916B1963916C596392690C49C2
:10CB2000D9625A6128465B680A49F2229847002078
:10CB300006E001A900F076FD0028E2D04FF0FF30BA
:10CB400003B030BD58230020E9C300083C23002077
:10CB5000C5C400081D220020194B07B51860194BE9
:10CB6000194A1A60194A5A60194A9A60194ADA60D1
:10CB7000194B02681A6042685A6082689A60C268FB
:10CB8000DA60164A1A6182695A61154BC26B5A60A3
:10CB9000144A019119609A601946134ADA6000201C
:10CBA000FFF7A6FF48B901A800F02AFD003818BF1A
:10CBB0000120404203B05DF804FB4FF0FF30F9E77D
:10CBC0003C2300202C23002051C5000851C8000838
:10CBD00091CC0008EDC4000814230020A519010819
:10CBE0006C230020B9C30008D1C3000849B118B1B3
:10CBF000012804D000207047034B0B60FAE7034B79
:10CC0000FBE74FF0FF307047000400010100010214
:10CC100008B503F08FFF002814BF6FF0010000205B
:10CC200008BD08B502F096FF002814BF6FF00100A0
:10CC3000002008BD20B1044BDB7903700020704751
:10CC40004FF0FF30704700BF4023002008B5034B72
:10CC5000D87103F053FF002008BD00BF402300201F
:10CC600010B504468AB018B94FF0FF300AB010BDB5
:10CC7000212368468DF8003002F0FCFF0028F3D134
:10CC8000024A9DF9043023705371EFE740230020DE
:10CC90002DE9F0412F4D304F00232B7043786B70FE
:10CCA0003B689B6A8AB004460BB128469847DFF878
:10CCB000AC80002658F8043B1BB11B6A0BB1204620
:10CCC00098470136F3B2052B76B2F3D12378052BC2
:10CCD0002FD00B2B35D0012B25D1214C06236846B4
:10CCE0008DF8003002F0C6FF0199E07906F01EFDD4
:10CCF00010B91C4B019A5A611B48FFF7F5FD1B4800
:10CD0000FFF7AEFF6B788BB9A371194B5878FFF71B
:10CD100045FD3B685B6A0BB1114898476B7813B9C6
:10CD2000E07906F095FD0AB0BDE8F081FF23A3711C
:10CD3000EFE7104B01225A74227A9A74627ADA74FD
:10CD4000F1E76378002BEED00AB0BDE8F041FFF7C1
:10CD5000B9BB00BFC40300203C230020582300209F
:10CD6000E00300207C230020E4030020E5030020F2
:10CD700040230020B003002030B58BB0FFF751FFF7
:10CD80000446F0B904F016FE831C1DD0F8B9134D0B
:10CD90002B685B69DBB1272368468DF8003002F011
:10CDA00069FF2B6801985B694FF4B961984704F0FB
:10CDB00013FE78B92CB9094B1B68DB690BB1012054
:10CDC000984720460BB030BD6FF00704EFE74FF0F7
:10CDD000FF34ECE74FF0FF34F3E700BF3C230020C3
:10CDE000014B1878704700BFAC230020014B5878E6
:10CDF000704700BFAC230020064B074810B5012246
:10CE00005A7309F085F9054B5B6913B1BDE8104011
:10CE1000184710BDAC23002094230020EC03002011
:10CE200013B50A4C79B1A27001230022616023700E
:10CE30000748084B00924FF0FF3109F0BDF800237E
:10CE4000637002B010BD2170F9E700BFAC23002071
:10CE500094230020F9CD00082DE9FF47C378CA2BA1
:10CE6000804600F0BE8004B0BDE8F087D8F80830F6
:10CE70005A5D6E1CF6B2032A0FD8DFE802F0022ECC
:10CE80006CAB7A6800231355611CA31CDBB2C9B2DA
:10CE9000012050540334D054E4B2354698F80C3095
:10CEA000AB42E3D8002CDED0CA238DF80830504BBB
:10CEB0008DF809405B6803930DF10700FFF7BAFE98
:10CEC0000020FFF7C3FE0122002102A8FFF79CFB10
:10CED0009DF80700FFF7BAFEC5E700227A7398F8BD
:10CEE00018204AB96A1DD2B2397A9A5C01F00F0152
:10CEF00002F00F02914202D0AE1DF6B2CDE7AA1C9D
:10CF0000D2B29E5D9A5C06EB0226EA1CD2B20DF10B
:10CF1000080A9A5C06EB02462A1DD2B250469B5C78
:10CF200006EB036608F022FF029B334402939AE863
:10CF3000030008F0F3FE3B7AC3F30302013262F30D
:10CF400003033B722B4B1B6B002BD5D00136022EFB
:10CF5000D2D89847D0E7EE1C0235EDB21E215B5DBA
:10CF6000002003F00F0380259D4006F08DFC7A68B9
:10CF70000223135504EB030A631CDBB20021D154D6
:10CF8000054402A808F0F2FE029B7A684B4504F1C2
:10CF9000030188BFA3EB09035FFA8AFAC9B2180A32
:10CFA00002F80A305054611D201DC9B2C0B24FEAC8
:10CFB000134C1B0E02F800C053544FF47A716943AE
:10CFC0000D4809F0DFF806340B48F6B2E4B209F078
:10CFD0009FF862E79B5D023503F007037B73EEB2B7
:10CFE0005BE70024024FDFF81490254656E700BFA8
:10CFF000AC230020EC03002094230020803DD512B8
:10D0000010B5114C637A8AB0E3B104238DF8003077
:10D010006846A37A8DF8043002F052FF18238DF889
:10D0200000306846E37A8DF8043002F049FF20238F
:10D030008DF800306846237B8DF8043002F040FF05
:10D04000002363720AB010BDAC2300200048704773
:10D05000EC03002030B58FB0FFF7C0FA002861D193
:10D06000324C657A4DBB042304A88DF8103002F0D1
:10D0700001FE9DF81430A37204A88DF8145002F03C
:10D080001FFF182304A88DF8103002F0F3FD9DF85F
:10D090001430E37204A801238DF8143002F010FF5D
:10D0A000202304A88DF8103002F0E4FD9DF8143020
:10D0B00023731F4BDB6A03B1984702A808F056FEA2
:10D0C000029A1C4B1C4913448B4288BF1B4B61685E
:10D0D00088BF9B181A0A4B708A701A0C1B0E0B71B2
:10D0E000237ACA7001256FF304134B710D702372FC
:10D0F0000DF1070040F2CA63ADF81030059165727A
:10D10000FFF798FD0020FFF7A1FD2A46002104A8A3
:10D11000FFF77AFA04469DF80700FFF797FD2046CF
:10D120000FB030BD4FF0FF34F9E700BFAC23002053
:10D13000EC03002080C22AED803DD512008555DA2F
:10D1400010B5054C637B2BB1FFF784FF10B9637BEF
:10D15000013B637310BD00BFAC230020014B187866
:10D16000704700BFD8230020014B5878704700BF9C
:10D17000D823002070470000044B9A7A0AB101229C
:10D180005A70034B5B6903B118477047D8230020DE
:10D190002404002073B5224C6378002B33D008F0B0
:10D1A00025FF66680546FFF7FFF90644AE4214D234
:10D1B000A37A93B1E0228DF800208DF80130217A16
:10D1C000E368019301226846FFF71EFA08B10730B1
:10D1D00010D100236370A372656094F83430EBB112
:10D1E000002384F834300F4B5B6BBBB102B0BDE859
:10D1F0007040184740F2DC510B4808F0C3FF0A4862
:10D2000008F086FFE8E794F83520002AE5D094F886
:10D21000360084F83530FFF7C1FADEE702B070BDA2
:10D22000D823002024040020BC23002037B5104D53
:10D23000104CC8B1C1B16272012300222860E160C4
:10D2400023700D480D4B00924FF0FF3108F0B4FEF3
:10D2500000250B4825822022294606F045FB6570F3
:10D26000A574A58603B030BD00232B602370EFE7C3
:10D27000D4230020D8230020BC23002079D100082B
:10D28000EC2300202DE9F0478E4C23788CB0002B46
:10D2900056D0C2780AB9837B13B1238A0133238223
:10D2A000437B002B4CD0E02A4AD10023A37287682D
:10D2B00097F80080B8F1220F27D8B8F1220F30D8A4
:10D2C000DFE818F04100FB0052005A0061006E00D8
:10D2D00075008E009D00B400C7002F002F002F00A6
:10D2E0002F002F002F002F002F002F002F002F00C6
:10D2F0002F002F002F002F002F002F002F002F00B6
:10D300002F002F00C900D000D400B8F17E0F00F02C
:10D31000CC80B8F17F0F00F0DF80B8F17D0F00F016
:10D32000AB80A57A002D00F05B81674C637A3BB936
:10D330004FF47A71204608F025FF204608F0E8FEF9
:10D340000CB0BDE8F087E36801220021A2721970D9
:10D35000A37AE1689818A0720620C854A37AE168FD
:10D360009818A072CA54DCE7584B9B6A002BD8D09F
:10D37000012102209847D4E77B7884F836300123D6
:10D3800084F83530CDE704238DF804307B78003BFA
:10D3900018BF012301A88DF8083002F091FDC0E705
:10D3A0007878003818BF012003F0A8FBB9E7484E91
:10D3B0000FCE01AD0FC50FCE0FC596E8070085E86B
:10D3C00007007B780A2BACD8424A12685268002AC0
:10D3D000A7D00CA901EB830353F82C0C9047A0E7CE
:10D3E0007878431E012B9CD83A4B01381B6818BF34
:10D3F000012020729B68002B93D0984791E7E26848
:10D4000001230821A3721170627A057BA17AAA42D6
:10D4100028BF2A46934284D285685A1CEB5CE56893
:10D4200001334E1CA6726B54D3B2EDE7E3680122C0
:10D43000A27209221A70A37AE268218A581CA0728B
:10D44000D154A27A238AE1681B0A501CA0728B5423
:10D4500067E7238265E705238DF8043001A803F010
:10D4600087F85EE7194BDB6A98475AE7194B7878DB
:10D470001B686075DB68BEE7037B072B7FF451AF49
:10D4800006238DF80430B7F80130ADF808307B7909
:10D490003A791B0443EA0223FA7813436422534384
:10D4A0000393BB798DF81030D8E73B2201A88DF8A3
:10D4B00004208DF8083002F003FD012384F8343095
:10D4C0002FE700BFD8230020BC2300202404002025
:10D4D000D42C0308D42300202A2301A88DF804307B
:10D4E00002F0C8FB94F80A90E6689DF808009DF8E1
:10D4F00009509DF80A709DF80BC09DF80D309DF8FD
:10D500000E209DF80F109DF80CE009F1010A84F837
:10D510000AA006F80980354E94F80A903668D4F8C7
:10D520000C8009F1010A84F80AA096F803A008F813
:10D5300009A094F80A90D4F80C8009F1010A84F843
:10D540000AA096F802A008F809A094F80A90D4F866
:10D550000C8009F1010A84F80AA096F801A008F8E5
:10D5600009A094F80A9009F1010A84F80AA096F833
:10D570000080E66806F8098094F80A80E66808F1F9
:10D58000010984F80A9006F808C094F80AC0E66811
:10D590000CF1010884F80A8006F80C70A77AE66896
:10D5A00007F1010C84F80AC0F555A57AE6686F1CEE
:10D5B000A7727055A07AE568461CA6722954A17A14
:10D5C000E0684D1CA5724254A27AE168501CA0721A
:10D5D0008B54A37AE268591CA17202F803E0A0E61A
:10D5E000034808F047FD6570AAE600BFD423002079
:10D5F000BC2300207047000000487047240400202E
:10D60000002108B50120FFF773FA014638B902205E
:10D61000FFF76EFA003818BF0120404208BD4FF0F6
:10D62000FF30FBE710B50C4661B1012803D002289A
:10D6300005D0002010BDFFF709FD2060F9E700F0DC
:10D640001FFCFAE74FF0FF30F4E70000014B1878B9
:10D65000704700BF94040020014B5878704700BF0A
:10D6600094040020F7B500208DF80700EFF3108236
:10D6700072B62A4FBB78FD7882F31088012B08D050
:10D68000022B04D1264B93F82030012B3CD103B060
:10D69000F0BD234E0DF10700FFF7C6F8382303FB5A
:10D6A000056393F82C00012806D19DF80730022B62
:10D6B00008D10023BB70EAE7022803D19DF80730A8
:10D6C000012BF5E7FFF76AF805EB4504E400B0B974
:10D6D000144BB8701C44382303FB05664FF47A7171
:10D6E00096F82830994096F82C30012B00D1C901CA
:10D6F000204608F047FD204608F00AFDC7E70A4B20
:10D700001C444FF47A71F3E7FFF748F80028D0D0B3
:10D71000044C05EB450504EBC504F2E79404002036
:10D7200040240020102400202824002037B50F4C6E
:10D73000D1B100250123A160227123702A460C4B30
:10D740000C4800954FF0FF3108F036FC0A4B0B48AF
:10D7500000952A464FF0FF3108F02EFC084A0023BE
:10D760006370137003B030BD2170F7E7940400209C
:10D77000B9D700082824002085D7000810240020ED
:10D780004024002010B5084808F074FC074B002224
:10D7900083F82020064B02225A80064B5B6913B1A6
:10D7A000BDE81040184710BD102400204024002080
:10D7B000940400205C04002010B5084808F05AFCCE
:10D7C000074A012382F82030064A5380064B5B69E2
:10D7D00013B1BDE81040184710BD00BF2824002039
:10D7E00040240020940400205C0400202DE9F04F28
:10D7F000C378C82B8FB0824600F029830FB0BDE8F4
:10D80000F08FDAF80820D05C591CC9B2052816D868
:10D81000DFE810F00600AA00F000AE01E1018B0283
:10D82000BA680023601C1355C0B2A31CDBB24FF0D2
:10D83000020C02F800C001200334D054E4B20B46BD
:10D840009AF80C209A42DCD8002CD7D0C8238DF847
:10D850001430B74B8DF815409B6806930DF11300FB
:10D86000FFF7E8F90020FFF7F1F90122002105A8F0
:10D87000FEF7CAFE9DF81300FFF7E8F9002DBDD1B1
:10D88000AC4CAD4F637803F003032A46294600935E
:10D890000220AA4B08F000F82646636800932A4647
:10D8A0002946A74B022007F0F7FF16F8083F009320
:10D8B0002A462946A34B022007F0EEFF012516F861
:10D8C000013F009300223B4611460220013507F03C
:10D8D000E3FF102DF3D1002211469B4B022007F0ED
:10D8E000DBFFA369009300221146984B022007F04A
:10D8F000D3FFE369009300221146954B022007F005
:10D90000CBFF636A009300221146924B022007F07E
:10D91000C3FF94F82820012393400022114600936E
:10D9200002208D4B07F0B8FF94F82C300022012B19
:10D93000236B00931146894B4FF0020040F08D821B
:10D9400007F0AAFF94F9343000930022844B11466B
:10D95000022007F0A1FFE38E0093824B00221146C4
:10D96000022007F099FF49E7BD6812F801C00122C3
:10D970002A55023300220234DBB2E4B21146964645
:10D980000CF0010C96F80080BEF1000F07D01201D8
:10D9900002F0700211436970054619464FE7B8F16D
:10D9A000000FF4D0BCF1000F21D005F804E004F121
:10D9B000010E5FFA8EFE716805F80E1004F1020E7A
:10D9C00071685FFA8EFE090A05F80E1004F1030E65
:10D9D0005FFA8EFEB6F8068005F80E80211DC9B2EA
:10D9E00096F807E005F801E00534E4B2614601323B
:10D9F0008646C7E7555C382105F0030501FB056144
:10DA000003F1020B5FFA8BFB4D70002D40F08E800E
:10DA1000D81C12F80B107160C0B203F1050C105C39
:10DA200001EB0021181DC0B27160105C5FFA8CFC24
:10DA300001EB0041716012F80CC0981D01EB0C69FC
:10DA400003F11601DFF820C1C6F80490C0B2C9B2D4
:10DA500086460130C0B212F80EE00CF801EF8842A1
:10DA6000F6D1115CB16103F11700C0B203F11E0BD6
:10DA7000105C01EB002103F11800C0B2B161105C31
:10DA800001EB004103F11900C0B2B161105C01EB80
:10DA9000006803F11A01C9B2C6F8188003F11B002F
:10DAA000515CF161C0B25FFA8BFB105C01EB0021AD
:10DAB00003F11C00C0B2F161105C1D3301EB0041A9
:10DAC000DBB2F161D35C0DF1170001EB036321229E
:10DAD0000021F361039321F001FE40F20112ADF841
:10DAE00014207278039B0A93C2F301028DF816206A
:10DAF00005A81E4ACDF818900792CDF8248002F0B0
:10DB000065FC012390B93370B96802230B55621C80
:10DB10001C44382303FB0563D2B25B78C3F30103D3
:10DB200043EA80008854E4B2594688E60120EBE7D6
:10DB300094040020402400201F830308E48203088B
:10DB4000F78203080C8303083A7D03082583030842
:10DB5000388303084B8303085E8303087383030839
:10DB6000868303089C830308472400204824002060
:10DB7000555C382005F00305023300FB05FB5FFA16
:10DB800083F906EB0B034FF00008184610224146BC
:10DB9000083083F80180C3F80480039305F0A4FEE5
:10DBA000039BC3E90688BB68032204F101081A55E8
:10DBB00028465FFA88F802F051FC40B145F00403B2
:10DBC000BA68023402F80830E4B2494637E606F88B
:10DBD0000B002B46F4E74FF0000B8DF813B0555CAB
:10DBE00003F1020815F003055FFA88F840F096800B
:10DBF000DFF874B24FF002098BF82C90D81C12F8A1
:10DC00000810CBF82410C0B203F10B08105C01EB34
:10DC10000021181DC0B2CBF82410105C01EB0041AC
:10DC2000581DC0B2CBF82410105C01EB00618F4886
:10DC30000844991DC9B2CBF82400515C01F00F01D2
:10DC40008BF82810D91DC9B203F10800515CCBF83C
:10DC50003010C0B25FFA88F8105C41EA002103F18D
:10DC60000900C0B2CBF83010105C0A3341EA004121
:10DC700064204143DBB2CBF83010D35C8BF83430F6
:10DC80000DF113020BF12C01284602F013FC0028C1
:10DC900049D105A808F06AF8DBF82420059BA2EB1F
:10DCA000030BBBF1000F31DD4FF47A7101FB0BF177
:10DCB0006F48039108F066FA6D4808F029FA039955
:10DCC00000916C4B29462A46484607F0E5FD0121A4
:10DCD000BA6804231355601CC0B29DF813C002F843
:10DCE00000C0A31CDBB271B102F803B0E31CDBB2CD
:10DCF0004FEA2B21D154631D0434E4B24FEA2B4B7D
:10DD000002F804B0DBB21C46414698E59DF813309A
:10DD100043F010038DF813302946D9E710238DF80E
:10DD200013305946D4E7AB46F6E74FF0000B8DF8B9
:10DD300013B0555C03F1020815F003055FFA88F88B
:10DD40007ED1DFF824B14FF001098BF82C90D81C5C
:10DD500012F80810CBF82410C0B203F10B08105CC5
:10DD600001EB0021181DC0B2CBF82410105C01EBB0
:10DD70000041581DC0B2CBF82410105C01EB0061CB
:10DD80003A480844991DC9B2CBF82400505CC0F34E
:10DD90000210ABF83600515C01F00F018BF828102F
:10DDA000D91DC9B203F10800515CCBF83010C0B2E4
:10DDB0005FFA88F8105C41EA002103F10900C0B263
:10DDC000CBF83010105C0A3341EA00416420414333
:10DDD000DBB2CBF83010D35C8BF834300DF113028A
:10DDE0000BF12C01284602F065FB70BB05A807F07B
:10DDF000BDFFDBF82420059BA2EB030BBBF1000F5A
:10DE000016DD4FF47A7101FB0BF11948039108F00C
:10DE1000B9F9174808F07CF903990091154B294688
:10DE20002A46022007F038FD4946BA68052351E723
:10DE30009DF8133043F010038DF813302946F4E7B2
:10DE400010238DF813305946EFE7AB46F6E7002470
:10DE5000094F054EFF252346F2E407F01DFD94F916
:10DE600034300093054B79E540240020803DD512E5
:10DE700028240020C9820308940400208683030814
:10DE8000004870475C040020044B054A93F81831A1
:10DE9000022B18BF062382F890347047E42A002032
:10DEA000A8300020034BD3F8483313B15B6903B1AA
:10DEB00018477047A8300020034A137843F0040342
:10DEC0001370FFF7EFBF00BF8C2400201FB50A4B73
:10DED0008DF8090093F87C208DF80A2093F88C20A7
:10DEE00093F848000D3202A98DF8082003F082FD56
:10DEF000C0B205B05DF804FBE42A002008B507486D
:10DF000008F0B8F8064B93F81A2412B1012283F8EE
:10DF10001924BDE80840FFF7C5BF00BFA8340020A2
:10DF2000A830002010B50C4CD4F8403343F08003E7
:10DF3000C4F8403394F81A3413B10020FFF7DEFF21
:10DF400094F8913423F0120343F0120384F89134CF
:10DF5000BDE81040FFF798BFA83000202DE9F04140
:10DF6000DFF8AC8098F81831022B06460D4602D037
:10DF7000284BDB6A984702F078FE044628B102205D
:10DF800002F069FE002002F06BFE98F81831012BB8
:10DF900017D102F06CFE074630B1002002F05CFEA3
:10DFA000002002F05EFE3C4602F063FE48B1002015
:10DFB00002F053FE002002F055FEBDE8F041FFF7ED
:10DFC00063BF002CF9D1144C94F8902494F81A34BF
:10DFD000BAB90BB184F84164304602F0EBFFD8F8CF
:10DFE0002C0008F00DF8D4F8B4339842E5D30B4870
:10DFF00008F040F894F8913443F0100384F8913419
:10E00000DBE70BB184F84154284602F0D3FFF1E777
:10E01000E42A0020DC8A0308A830002040340020D5
:10E02000074A10B5137843F002031370FFF73AFF65
:10E03000BDE81040034B01220021022007F02CBC58
:10E040008C240020AF830308074A10B5137843F0EF
:10E0500008031370FFF726FFBDE81040034B0122B1
:10E060000021022007F018BC8C240020BF83030885
:10E070002DE9F0410F4616461D46804607F0B6FFD3
:10E080000B4A0C4C1378278123F0110343F0110342
:10E09000C4E90008137066812573FFF703FFBDE82C
:10E0A000F041054B01220021022007F0F5BB00BF23
:10E0B0008C24002078240020CF83030813B507F0B8
:10E0C00095FF0D4B6C461860204607F04FFE94E814
:10E0D00003000A4A0A4B83E80300137843F0200345
:10E0E0001370FFF7DFFE074B01220021022002B070
:10E0F000BDE8104007F0D0BB882400208C2400200D
:10E10000E0330020DC8303082DE9F04192B006469D
:10E1100002F0ABFD002840F05881AD4D95F8183164
:10E12000012B09D02B6BAB4C93B194F80431BBB1EC
:10E13000042B6FD0032003E002F099FD18B10F20EB
:10E1400012B0BDE8F08102F094FD0028EAD0F6E7B5
:10E15000B5F82031D4F81C24013B53432B63E4E78A
:10E160009D4803F07EFB002840F0128194F80C31AA
:10E1700023802B6B0C930DF1180895F839308DF82E
:10E180003830404695F81C318DF83A3007F014FECF
:10E19000D5F82831009302AF98E80600D5F824316D
:10E1A000384607F09FFD97E803000FAB83E80300B4
:10E1B000EB6A0D9300238DF844302388ADF8463088
:10E1C00095F8303101228DF839201BB98DF84420A3
:10E1D0008DF83930814B0093814B95F84800A3F1BD
:10E1E00079020CA903F07BFCC0B10B28A8D1D4F8AC
:10E1F000941499B1002EA3D0D4F84033794843F059
:10E200002003C4F8403307F0BDFF764807F080FFD5
:10E21000002095E7704803F058FBA4E795F8487094
:10E2200095F9693095F9392095F87D106E4E38468C
:10E2300003F062FC009641B2EB6C95F85020384632
:10E24000183603F0FDFB0096EB6C95F8502095F91D
:10E25000701095F8480003F0F3FBD4F8C413AB6DCD
:10E26000D4F8DC230B44C4F8B033EB6D1344C4F88A
:10E27000B43394F80431042B07D02B6E0B44C4F84C
:10E28000B0336B6E1344C4F8B4330023089395F88D
:10E290003031002B40D100238DF8133095F8393000
:10E2A0008DF8213095F838308DF82230D5F880304F
:10E2B0000993D5F884300A932388ADF82C3095F86B
:10E2C000303194F81B648DF82E3095F84800474B98
:10E2D0008DF820600DF1130208A903F0C5FB01239E
:10E2E00084F8413495F8393084F842349DF813307D
:10E2F00084F84334D4F81C34C4F85064C4F8483467
:10E30000C4F8583402F0B7FCC8B1D4F81C0402F0C9
:10E31000C4FCA0B1102013E708A802F07BFD60B98F
:10E3200095F9390094F837629DF82070FFF7CEFD1B
:10E330003E44B042AFD2082002E7132000E795F830
:10E340001831012B01D102F0AAFC02F097FC002346
:10E35000059394F8043195F9395094F81B649BB1F6
:10E36000042B7FF4E7AE05A802F088FF58BB94F8B1
:10E37000183413B1059B013B0593174B05983246A2
:10E38000E9B202F0E1FF02E0134802F0B1FF08B188
:10E390001120D5E6D4F8403394F80C11218043F0D5
:10E3A0000203C4F8403394F8183411480133DBB247
:10E3B00084F8183484F845340E4B00259B6AC4F861
:10E3C0009854984724E71220BAE60E20B8E600BF1A
:10E3D000E42A0020A8300020B0310020142B0020B7
:10E3E0003C3500201034002060340020C43400206C
:10E3F000AA300020DC8A030873B5134D134E009633
:10E40000EB6C95F8502095F9781095F8480003F0DA
:10E4100017FB95F83031337595F8480040F2012329
:10E4200006F13C023146738203F016FB50B196F8B8
:10E430003C3086F88230064B00205B6B9847F37CBB
:10E4400086F8A83002B070BDE42A00209034002085
:10E45000DC8A0308F8B5324C94F81831012B0546D4
:10E460000ED0022B4ED0002B57D138B9D4E91B0166
:10E4700004F1740383E803000020F8BD012806D1ED
:10E4800002F0FEFB0028F8D184F81851F5E70228C5
:10E4900043D1244E84F8180106F5747CBCE80F00C3
:10E4A00006F57A770FC79CE8030094F8E92094F802
:10E4B000003187E8030086F8FB53D2B1022B18D154
:10E4C000D4F804316367C6F8EC3394F87D3094F8DF
:10E4D000082186F8F83394F88C3084F8782086F890
:10E4E000F93396F81B2486F8E82340F20133A6F8A6
:10E4F000FA33002386F81A340B4BDB6A9847FFF790
:10E500007BFFB9E748B9074B84F81801062283F866
:10E510009024054BDB6A9847AEE70320ADE700BFC8
:10E52000E42A0020A8300020DC8A0308F0B5504C13
:10E53000504EB4F8DC202287D4E92D0194F8B120A4
:10E5400084F8692004F16C0282E80300D4E92F0109
:10E5500004F1740282E80300B4F8C420A4F87C201B
:10E5600091B0D4F8CC20D4F8C810C4F88420002589
:10E57000D4F8D020C4F888200123A4F82031C4F8AE
:10E58000801084F83051A56284F81B5184F83A5009
:10E5900084F81D5184F81E51C4F83451C6F89854BB
:10E5A000A6F8185486F81A54A4F838518DF8183083
:10E5B00004F50973039304F50A7394F8480004936F
:10E5C00003A92D4B84F84551C4E94F55A4F8465191
:10E5D000059303F01DFAE36EC6F8D43394F87D304A
:10E5E00086F8E03394F88C3086F8E1334FF480738A
:10E5F000A6F8E23386F8D05394F8303186F8E43345
:10E6000006F574770FCF06F57A740FC497E8030008
:10E6100040F2012384E80300A6F8FA33D6F8483321
:10E6200086F81B54CDE901551BB15A685B6901920C
:10E630000293124B0793A3F148020892A3F114022C
:10E6400009920F4A0B9229330A93A2F19C030C936F
:10E65000A2F198030D93131D0E9301A902F14C032F
:10E6600007A802F599620F9302F0F4FA11B0F0BD19
:10E67000E42A0020A830002090240020103500203B
:10E68000C82B0020F8B50D4F0D4E0C4607F0F2FCDC
:10E690003B6B98470B4A96F84800214603F0DCF99B
:10E6A00050B1094D706D95F8243485F86A347B6B50
:10E6B0009847E37C85F89034F8BD00BFDC8A0308F6
:10E6C000E42A0020CC340020A83000200F4890F825
:10E6D0001B3480F8B8330E4B93F8692080F8BB23C5
:10E6E00093F87D2080F8C82393F88C2080F8C92304
:10E6F00093F8303180F8CC330022A0F8CA2300F51B
:10E700006E7100F56070FFF7BDBF00BFA83000203C
:10E71000E42A0020114890F89034EBB190F81B34B3
:10E7200080F8D0330E4BDA6EC0F8D42393F87D20F6
:10E7300080F8E02393F88C2080F8E12393F83031BF
:10E7400080F8E4334FF48072A0F8E22300F574718E
:10E7500000F56670FFF796BF704700BFA830002035
:10E76000E42A002070B5344C2421204605F0BEF880
:10E77000636A984218BF60624FF01C012F4814BFB3
:10E780000125002505F0B2F8636C984218BF60645B
:10E790004FF480712A4818BF45F0020505F0A6F82D
:10E7A000D4F84831984218BFC4F848014FF0D4015A
:10E7B000244818BF45F0040505F098F8D4F8203235
:10E7C000984218BFC4F820024FF000011E4818BF3D
:10E7D00045F0080505F08AF8D4F82432984218BFAD
:10E7E000C4F824024FF46071184818BF45F01005B2
:10E7F00005F07CF8D4F8A835984218BFC4F8A805ED
:10E800004FF01401124818BF45F0200505F06EF8CE
:10E81000D4F8C03598420F4B18BFC4F8C005D3F8E0
:10E82000483318BF45F040052BB11B691BB1284682
:10E83000BDE87040184770BDE42A00200C2B002072
:10E840002C2B0020302C0020082D00200C2D002027
:10E8500090300020A83000202DE9F04F8FB04FF00D
:10E860000009012B06460F4690468DF80D90ADF835
:10E87000109002D84C46BC4202D30FB0BDE8F08FD6
:10E88000305D02F007FB2044B842F6DC335D651CC6
:10E89000023BEDB2112BF0D801A252F823F000BFD9
:10E8A000E9E8000813E9000811EA000839EA00085D
:10E8B000B7EA0008DDEA000843EB00086BEB00084C
:10E8C000F1EB00087BE800087BE8000845EC000855
:10E8D0007BE800087BE80008EDEC000815ED000877
:10E8E0004DED000881ED0008052002F07BFB70B1C2
:10E8F0000521002002F03CFB725DBA4BE51C02349E
:10E90000E4B283F85C24325D83F85D24EDB22C46DA
:10E91000B1E700238DF80E308DF80F308DF81430EC
:10E920008DF81830B9F1000F6DD1AF4C4FF00509DB
:10E9300094F87C208DF831206B1E94F839208DF8E6
:10E940003320334494F838200B938DF8342094F816
:10E950001A3194F868208DF83520D4F82C218DF8E0
:10E9600032300A9273B37B1C5B1BDBB28DF8303004
:10E9700006AB019305AB009394F848000DF10F032B
:10E980000DF10E020AA903F07BF88DF80D0000F0DE
:10E990000700072813D194F939209DF90E3084F827
:10E9A00039309A429DF80F3084F83830B8BF0122D0
:10E9B0009DF81430B8BF84F81D2184F868304FF0FA
:10E9C000000A09E00523D1E701220DF10D01032022
:10E9D00002F078F90AF1010A5FFA8AF29DF818301C
:10E9E000B3FBF9F19142EFD82B44DDB26B1EDBB2E1
:10E9F0009F420BD9F25C032A9AD0AF4288BF1D46D2
:10EA00004FF0010983E70534E5B2F9E71D46F7E762
:10EA1000735D754903F00F03012281F81B31023445
:10EA200002FA03F3A1F82031E4B2002204A9042081
:10EA300002F048F925466AE707238DF80D30735D2B
:10EA4000C3F3021203F00F038DF82830E31CDBB28E
:10EA50008DF82920F25C231DDBB2651DF35C0234C6
:10EA6000E4B21B0443EA0223325D5F4C1343642289
:10EA7000534394F848000B930AA903F010F800F0F0
:10EA80000703072BEDB28DF80D000CD19DF828304F
:10EA900084F8703084F878300B9BE36663679DF8E8
:10EAA000293084F869308DF81000012204A905206E
:10EAB00002F008F92BE74B4BD3F8483363B11B68DE
:10EAC00053B1984708F03F038DF810008DF81130CE
:10EAD000022204A90620EBE7FF20F3E703238DF8C9
:10EAE0000D30735D8DF81C300AAB0693E31CDBB26E
:10EAF000A51DF25C231DDBB206A9F35C1B0443EAEF
:10EB00000223A21CD2B20534B25C134364225343E5
:10EB1000E4B20A9300230B93335D8DF83030324B0F
:10EB200093F8480002F0C1FFC3B20028EDB28DF89F
:10EB30000D30FFF6ECAE8DF81030012204A907204D
:10EB4000B6E7735D03F00F03012B4FF47A7238BF01
:10EB500001235343244A0234936503F57A73D36542
:10EB6000E4B2002204A9082062E7735D1E4DC3F3DE
:10EB700040128DF8152095F84800C3F3001205A93E
:10EB800003F00F038DF814208DF8163002F093FF78
:10EB900002340130E4B23FF44DAFBDF81430134AF3
:10EBA000A5F87C309DF816309DF814A0D05CF3F7E2
:10EBB00001FA0223C5F880000AA995F848008DF8EB
:10EBC00028308DF82AA002F015FF95F9393006900B
:10EBD00040B29842B8BF184685F83900002204A90F
:10EBE000092025E7A8300020E42A0020E983030853
:10EBF00003238DF80D30735D8DF82830E31CDBB2F4
:10EC0000651DF25C231DDBB20234F35CE4B21B042D
:10EC100043EA0223325D1343642253430B93644B54
:10EC20000AA993F8480002F04CFFC3B20028EDB2E5
:10EC30008DF80D30FFF66BAE8DF81030012204A96F
:10EC40000A2035E7092002F0CDF9DFF868B1002885
:10EC500049D00921002002F08BF90023ADF81E30C5
:10EC6000A31CDBB2F25CE31CDBB216F803A0735DFD
:10EC70004FEA0A4A4AEA022A4AEA030A231DDBB299
:10EC8000A51D0534F35CE4B24AEA036A335D4FF430
:10EC90007A7253430AAC1B122046ADF81C3007F0C1
:10ECA00065F8454B53440693DBF83C3300930DF174
:10ECB000180A9AE80600DBF8383308A807F012F8BB
:10ECC000099B009394E80600089B504606F0EFFF6E
:10ECD0009AE8030007F022F801F0DCFF0123EDB20F
:10ECE0008BF8383413E68BF8380410E60C2002F069
:10ECF00079F900283FF40BAE0C21002002F038F91E
:10ED00002C4B93F89034043B012B7FF600AE01F0BE
:10ED1000BDFFFCE5A31CDBB2725DF15CE31CDBB262
:10ED2000651DF35C0434E4B21B04305D43EA012347
:10ED300013436421594300F00F0001F0A8FFEDB226
:10ED40008DF81000012204A91120B1E60D2002F077
:10ED500049F900283FF4DBAD0D21002002F008F94D
:10ED6000A31CDBB2154AF05C735D1268251D0334E9
:10ED7000E4B243EA0020315DEDB201F08AFFC6E55E
:10ED8000725DA31C251D0334DBB2E4B2F15C335D7C
:10ED90001B0443EA012313436420584301F07BFF23
:10EDA000EDB28DF81000012204A9132080E600BF07
:10EDB000E42A0020A8300020803DD51278240020CD
:10EDC0000E4B93F89124920703D593F88F24012AD0
:10EDD00008D90B4991F81A2122B18A6A501C18BF30
:10EDE00001328A620022A3F8182483F81A24D3F887
:10EDF000402322F00202C3F840237047A8300020CD
:10EE0000E42A002070B5184C1848194D07F032F963
:10EE1000D4F84033D4F89804D5F8906023F0200358
:10EE2000C4F8403338B107F0EBF8864203D2002330
:10EE300085F83A3070BD0120FFF766F90028F9D057
:10EE40000B28F7D095F8393084F84234092094F82B
:10EE5000183484F8453484F8410402F0ABF8BDE876
:10EE60007040FFF7ADBF00BFA83000201034002075
:10EE7000E42A0020094BD3F84023012A0AD008498C
:10EE80000978C90708D43AB993F89204013818BF31
:10EE9000012070470020704701207047A8300020F3
:10EEA0008C240020034BD3F84003431E58425841A2
:10EEB000704700BFA83000202DE9F04FA9B0EFF354
:10EEC000108272B6DFF8F0B20021DBF80030CBF828
:10EED000001082F31088B94C002B00F0E180DAB208
:10EEE0009B06039264D5B64D95F81831022B02D0DB
:10EEF000B44BDB6A9847EFF3108872B6B24F07F055
:10EF000075F83E68D4F8B013361A3144AF4807F0AC
:10EF100039F9AE4807F0FCF8D4F8B413AC483144E2
:10EF200007F030F9AA4807F0F3F888F3108894F84E
:10EF30001A34002B00F06B81152312A995F84800B4
:10EF40008DF8483002F056FDD4F8B4130F90014408
:10EF5000A04807F017F99F4807F0DAF83B6894F8E3
:10EF60001B24EB620DAF38468DF870201D9306F020
:10EF700023FFD5F82831009306AE97E80600D5F8B0
:10EF80002431304606F0AEFE96E803001FAB83E85E
:10EF90000300D4F81C341E9395F8303195F84800DE
:10EFA000003B18BF01231CA98DF8713002F02BFD26
:10EFB000039BDF0648D5824DDFF81CA2D5F8E4207C
:10EFC00004929BF80020BAF90A809AF90C90A4F8F0
:10EFD0008C84002363F300020A9384F84434A4F879
:10EFE000223484F82534C4F82834A4F82C3484F866
:10EFF0002E34C4F8303484F82034C4F8343484F81F
:10F000003834C4F83C346F4B8BF8002094F89024CB
:10F01000DB6A84F88E9484F88F24DAF80470BAF8E6
:10F020000860984794F88F3413B9694807F022F8BC
:10F030003146384601F017FE8346002800F0EA808A
:10F04000A4F87E8484F88094039B19071AD55C4B3E
:10F0500093F81831022B02D05A4BDB6A98470220F2
:10F06000FEF712FF84F8410401F0A4FF94F81A346B
:10F0700013B1012384F8193494F8913443F0100348
:10F0800084F89134039B5A0703D506210520FEF727
:10F0900065FF039B9B0703D504210320FEF75EFF5A
:10F0A00001F000FE94F89124D7065FD5002384F880
:10F0B0009234D4F840331E0644BF23F08203C4F8D0
:10F0C000403312F0050F00F0FB820B2001F08AFFA5
:10F0D000002800F0F58294F89134DD0700F1F08209
:10F0E000580740F10783D4F8403323F00203C4F8F3
:10F0F0004033D4F8402382BB94F8915415F00101B9
:10F100001EBF2B4662F3000384F8913494F89134C7
:10F110005E0744BF6FF3820384F89134012384F8BF
:10F12000923421B1D4F844332C481B6898476D07BA
:10F130000BD52B4801F062FF01F090FF28B194F845
:10F14000913443F0040384F8913401F098FD94F86D
:10F1500091346FF3041384F89134012384F89234CA
:10F1600094F8913443F0200384F8913494F8913466
:10F1700018070AD56FF3C3031A4984F89134D4F8F9
:10F180004433A1F12400DB68984794F8913499073F
:10F190000AD56FF34103134984F89134D4F844330A
:10F1A000A1F16C005B68984794F89034022B1BD156
:10F1B000FFF722F918E000BF8C240020A8300020BF
:10F1C000E42A0020DC8A0308882400202834002058
:10F1D00040340020A834002078240020E8340020A7
:10F1E000FC3400203435002094F891349A0640F124
:10F1F000C4826FF3451384F89134D4F84033002B64
:10F2000040F0BB8229B0BDE8F04FFFF7ABBA84F8FD
:10F210004134A3E695F81831012B0CD101F027FDFC
:10F22000804668B1584601F017FD584601F019FDB7
:10F23000042384F88F347EB9012384F821344FE10C
:10F2400001F017FD0028F6D0404601F006FD4046CB
:10F2500001F008FD0523ECE73B7805935B09013BD2
:10F26000062B00F21782DFE813F007001502950065
:10F270001502920015020602102EDDD995F83031E4
:10F280001297F6B28DF84C60002BD5D11CA804F073
:10F290003FFA12AA1CA9FF2002F072F99DF858301B
:10F2A000C3F3030307468DF82C3095F8480095F812
:10F2B0007D308DF82D3007220BA902F0AEFB002F18
:10F2C0005DD100285BD09DF853309DF852201599F0
:10F2D000C5F8E4101B0443EA02239DF851200220E4
:10F2E0001343C5F8E03004F021FA9DF8583095F842
:10F2F000480085F82E71C3F30212C3F3030385F8A7
:10F30000703085F878309DF8593085F86920012BE8
:10F3100038BF01234FF47A725343AB651344EB6556
:10F320000DF15A034FF001081093113E94F81B346D
:10F330008DF83C300FA985F868808DF8446002F0A4
:10F3400074FB0223404685F8303101F04BFE18B1C2
:10F350004146384601F00CFE94F88F34012B00F240
:10F36000A78194F81A34002B40F09A8194F89134D4
:10F3700043F0100384F89134FEF786FD64E6012023
:10F3800001F030FE0028E7D001210720E2E7012349
:10F3900084F8203495F87D308DF82E3094F824349C
:10F3A0008DF82D3095F88C3095F848000D330BA969
:10F3B0008DF82C3002F01EFBA6F10D031BB2099054
:10F3C00023EAE37300B283423FF736AF0B2E7FF69A
:10F3D00033AFBA4B25931CA8FF231C978DF874609C
:10F3E0008DF8983002F0E2F9074600287FF424AF48
:10F3F00095F81831012B13D101F039FC002872D097
:10F40000384601F029FC384601F02BFC04239DF816
:10F410007C101E9884F88F34C1F3001101F041FC78
:10F420009DF87C301E99C4F8341413F00F0203D0F9
:10F430009DF89000002862D19DF89800002861D0C6
:10F44000002A7FF4F9AE9DF89020002A14BF4FF0F7
:10F4500003084FF0020800220A92D5F8EC2095F834
:10F46000E900914251D100284FD0D5F80C1195F800
:10F47000EAB009680A9195F81811022902D103210E
:10F4800084F88F14B8F1030F7FF4D6AE13F0600F39
:10F490007FF4D2AE0492012795F82E31BBF1000F14
:10F4A00036D0BBF1010F13D1012B33D16FF0090618
:10F4B00046FA08F606F00106C6F10206F6B2BDF8F5
:10F4C0007E100AAA304601F0E5FE38B3072823D0A3
:10F4D000012384F821340A9BC4F83034C4F86C3416
:10F4E000FEF720FDB0E501F0C4FB002898D03846B7
:10F4F00001F0B3FB384601F0B5FB052387E74FF079
:10F500000008A8E74FF00108A5E74FF0010BC3E79B
:10F510000426D4E70326D2E70823DAE71CAB0093DE
:10F5200004990A9B3246584601F076FF20B1022822
:10F5300014BF0B230A2380E60A9BC4F83034C4F8B6
:10F540006C349DF87C3084F82104C3F3401384F8B4
:10F550002E3484F8443494F88F3484F82274012BC8
:10F560009EBF0122A86285F81E21012FC4F828043D
:10F5700084F82C0484F8410438D1022284F8202431
:10F5800095F83A20002A4AD19DF87C20D60646D428
:10F59000012B94F840149DF87C2005D8012901D155
:10F5A000900601D501F020FCB8F1020F94F88F34D9
:10F5B00043D0B8F1030F0AD09DF87C10B8F1010FC9
:10F5C0004A4601F00F0120A83BD0FFF745F99DF80E
:10F5D000903084F82334259BC4F828349DF8983063
:10F5E00084F82C34012384F82D3430E0059A02F09D
:10F5F000E002A02A1BD195F82E11012285F83A20AD
:10F6000009B927996963012B84F8202407D9D5F813
:10F610009020C4F83C24DAF80020C4F8982495F827
:10F620001821002AB4D1012284F82524B0E7002251
:10F6300085F83A2084F82024A6E79DF898102598AC
:10F640004A46FFF709F99DF8903084F823349DF875
:10F650009020E02A08D195F81F312BB984F8232493
:10F66000C4F82834A4F82C3494F8913443F00203FD
:10F6700084F8913470E6114D013EB2B2791C2846EF
:10F6800004F01EF90323A4F82034C4F8285484F8A5
:10F690002C64E9E7012384F82134FEF743FC5BE6A0
:10F6A00094F84434002B3FF461AE0020FEF726FCB2
:10F6B00094F88F34022B3FF45FAE57E6E03200201F
:10F6C00094F89134590715D5012001F08BFC60B1F5
:10F6D000012001F05FFC08B984F81804D4F8403325
:10F6E00023F00203C4F8403304E0062001F07AFC62
:10F6F0000028F3D194F89134DA077FF5FAAC94F846
:10F7000040240AB1032A18D11D4A94F8181492F81B
:10F710006820914205D29B0723D594F88F34012BA2
:10F720001FD8184806F0A6FCD4F8403323F0200375
:10F73000C4F84033FFF744FBDBE4012A11D194F80D
:10F740001924002A3FF4D5AC0D4A94F8181492F805
:10F7500068209142E5D29F0703D594F84434002BEA
:10F76000DFD194F8913400206FF3041384F89134BE
:10F7700084F81904FFF746FBBBE429B0BDE8F08F1D
:10F78000E42A0020103400202DE9F04F89468DB086
:10F7900090460746002800F08F81002900F08C81F8
:10F7A0000368002B00F088814368002B00F08481FF
:10F7B0008368002B00F08081C368002B00F07C81FF
:10F7C000104602F013F9002800F07881BD4CBE4DC0
:10F7D000384601F083FB40F2C4520021204604F079
:10F7E00083F840F21C520021284604F07DF8B74B04
:10F7F000C4F82C3104F50973089304F50A73002644
:10F800004046099308A9B24B84F848800A9384F8CB
:10F81000186184F88C608DF82C6002F0F9F80F23E1
:10F8200006A994F848008DF8183002F0E3F8801B20
:10F8300018BF01204FF00A0B84F81C0106A994F8A8
:10F8400048008DF818B002F0D5F84FF0060A84F899
:10F85000DC0006A994F848008DF818A002F0CAF858
:10F86000102384F8DD0006A994F848008DF81830BC
:10F8700002F0C0F81123C4F89C0006A994F84800CF
:10F880008DF8183002F0B6F81223C4F8A00006A9CB
:10F8900094F848008DF8183002F0ACF81323C4F83F
:10F8A000A40006A994F848008DF8183002F0A2F8D8
:10F8B0001423C4F8A80006A994F848008DF818305D
:10F8C00002F098F81623C4F8AC0006A994F8480092
:10F8D0008DF8183002F08EF8172384F8B10006A9CD
:10F8E00094F848008DF8183002F084F818230DEBD6
:10F8F0000301C4F8B400C4F8BC0094F848008DF8C3
:10F90000183002F077F8C0B21D2384F8B80084F8EC
:10F91000C00006A994F848008DF8183002F06AF883
:10F920001E2384F8C40006A994F848008DF8183006
:10F9300002F060F81F2384F8C50006A994F8480077
:10F940008DF8183002F056F82023C4F8C80006A934
:10F9500094F848008DF8183002F04CF80B23C4F8E6
:10F96000CC0006A994F848008DF8183002F042F84F
:10F970000C2306A9A4F8D00094F848008DF818309C
:10F9800002F038F8D4F89C306365D4F8A030A36551
:10F99000D4F8A430E365D4F8A83023664FF001080A
:10F9A000D4F8AC300590A4F8D200636684F8B08037
:10F9B000C4F894B084F898A0C4F84CB084F850A06F
:10F9C00084F8688084F81F81C5F84893FEF7AEFD7F
:10F9D000C5F84473C4E90B663E4B84F8198185F879
:10F9E0009164C5F8408332464FF0FF31009605F52B
:10F9F0005A7006F0E1FA384B009632464FF0FF316C
:10FA000005F5607006F0D8FA344B009632464FF098
:10FA1000FF3105F5667006F0CFFA02AF304B009665
:10FA200032464FF0FF3105F5806006F0C5FA3846E2
:10FA300006F0C2F997E8030004F5927383E8030027
:10FA4000284B294F1E60294BC5F84C33284BC5F86D
:10FA50005433284BC5F85C33274BC5F85033274B3C
:10FA6000C5F8583305F553703B68984704F5A67000
:10FA700003F06AFC20B1112630460DB0BDE8F08FCE
:10FA8000204601F0D7FB0028F5D101F00DF9B8B9F7
:10FA90001B4801F021FC06460028ECD17B69984701
:10FAA00003F0ECFEBB6D94F819019847FB6A984788
:10FAB000012385F89234DFE70326DDE70926DBE73B
:10FAC0001326D9E7E42A0020A83000200004000112
:10FAD0009024002005EE0008CDE6000815E7000898
:10FAE000FDDE00088C240020DC8A0308BDE000084D
:10FAF00071E00008B9DE000849E0000821E00008D4
:10FB0000CC2B002008B5034B0020C3F84003FEF7C0
:10FB1000BBF908BDA830002010B5FFF7ABF90A4CBF
:10FB200060B90A4B93F81831022B02D1084BDB6AFB
:10FB300098470123C4F84033002010BDD4F8400397
:10FB4000013818BF0120F8E7A8300020E42A00207F
:10FB5000DC8A030838B5124C204606F08BFA04F113
:10FB6000180006F087FA04F1300006F083FA04F179
:10FB7000980006F07FFA01F081F80A4B0025DB6A55
:10FB8000984744F8285CFEF7EDFD0749074840F226
:10FB9000C45203F095FE012344F8283C284638BDA2
:10FBA00010340020DC8A0308E42A002020250020ED
:10FBB00070B52E4B8AB0054693F8DD008DF809002C
:10FBC00093F8DC008DF80A0029489A6A90F8180426
:10FBD000039200268DF80B0004960C46002940D0B5
:10FBE0000692D3F8882007921A8F93F81A118DF88D
:10FBF000151052BAADF8202093F87C2093F84830C5
:10FC00008DF8243003AB8DF822008DF8232000936B
:10FC10000DF10A020DF10B030DF1090105A88DF894
:10FC2000146000F0A9FF9DF90900FEF74FF960701C
:10FC300004A801F0EFF8B0B9049A0F2A0DD8637840
:10FC40009A420AD81544AB42A3EB02012CBF002014
:10FC500001202170C0000AB070BD0023237008206D
:10FC6000F9E70320F7E71320F5E700BFE42A0020B7
:10FC7000A83000201FB50446002800F0108103784A
:10FC8000412B00F20781DFE813F0420049004D00EC
:10FC90005100550059005E000501050105010501EF
:10FCA0000501050105010501650069006D00780089
:10FCB0007F00820085008A0088008C0090009300FD
:10FCC000960099009C009F00AE00B200BA00B600FA
:10FCD000BE00C100C500CE00CA00CC000501D200A4
:10FCE00005010501050105010501050105010501E4
:10FCF0000501050105010501050105010501DA0000
:10FD0000DE00E200E700EB00EF00F300FC00664BD2
:10FD100093F818312371002004B010BD624B93F8A2
:10FD20003031F7E7406803F0ADFCF4E7406803F0DA
:10FD3000EFFCF0E75C4B93F81A31EBE75A4BD3F842
:10FD4000E0306360E7E7584B011D93F8300103F0A2
:10FD5000F7FCE0E7544B93F81931DBE7524B93F88B
:10FD60008C30D7E71C238DF808304F4B02A993F84D
:10FD7000480001F03FFE6060CDE74C4B043493E84F
:10FD8000030084E80300C6E7494B0434F7E7494B16
:10FD90000434F4E7484B0434F1E71A23E3E719236A
:10FDA000E1E7414B93F86830B4E73F4B5B6DC8E740
:10FDB0003D4B9B6DC5E73C4BDB6DC2E73A4B1B6E81
:10FDC000BFE7394B5B6EBCE702238DF80830364B3A
:10FDD00002A993F87C2093F848008DF80A2001F0DE
:10FDE00009FE207197E7304B93F8DD3092E72E4BF8
:10FDF00093F839308EE72C4B93F8DC308AE72A4BA6
:10FE000093F8383086E7284BDB6C9AE7264B93F85B
:10FE100050307FE7244BD3F8843063607BE7224B7C
:10FE20008FE7264B8DE7204BD3F8CC30F5E71E4B00
:10FE3000D3F82C31436001F06BFEA0606BE71A4BE6
:10FE4000D3F890307DE7184B93F81F3162E7164BDB
:10FE5000B3F88830A3805EE7134BB3F88A30F9E734
:10FE6000114BB3F8D030F5E70F4BB3F8D230F1E7D0
:10FE70000D4B93F848200AB1062A12D1B3F8A035E9
:10FE8000E8E7094B93F848200AB1062A09D1D3F8CC
:10FE9000A43556E704B0BDE8104000F0F3BE0320DF
:10FEA0003AE7182038E700BFE42A0020502B002052
:10FEB000982B0020582B0020A02B0020202500206C
:10FEC0007FB5044610B9032004B070BDA34DD5F82A
:10FED00040339A0700F16F820278412A00F268826B
:10FEE000DFE812F04200470055005B005F0064004D
:10FEF00069007600810087008D00930099009F00C3
:10FF0000A500AB00B5006602BA00DC00EF001601E8
:10FF10003801290142014B014F01530157015B0197
:10FF200066025F01710199018701AB01B101B8015E
:10FF3000BD01C2016602280266026602660266020E
:10FF40006602660266026602660266026602660271
:10FF50006602660266026602340239023E0243020B
:10FF600048024D0252025C020079FEF773FA30B18A
:10FF7000AAE70379022BA6D0794A82F8303195F8A6
:10FF8000913443F0200385F8913400209CE74068C9
:10FF900003F06AFB0028F2D095E7406803F0A8FB65
:10FFA000F8E76F4B027983F81A21E8E76C4B426857
:10FFB000C3F8E020E3E76A4E416896F8300103F0A9
:10FFC000B5FB00287FF47FAF6368C6F8E430D6E75E
:10FFD000416800293FF477AF002001F0B1FA002812
:10FFE000CDD0112070E7416800293FF46CAF0120AB
:10FFF000F3E7416800293FF466AF0820EDE7416868
:020000040801F1
:1000000000293FF460AF0920E7E7416800293FF489
:100010005AAF0C20E1E7416800293FF454AF0D20AE
:10002000DBE7416800293FF44EAF0E20D5E7416879
:1000300000293FF448AF0F20CFE74A4C484B0079E6
:1000400083F81901A36D9847E36A984797E7444BF3
:10005000027983F88C2092E7414E037A8DF80430C0
:1000600096F8480096F87D308DF80530072201A9F2
:1000700001F0D3FC00283FF426AF636896F84800EF
:100080000193002201A901F0C8FC00283FF41BAF36
:100090006C36D4E9010186E8030070E7304E037A3C
:1000A0008DF8043096F8480096F87D308DF80530CC
:1000B000072201A901F0B1FC00283FF404AFB436D7
:1000C000E7E7274E037A8DF8043096F8480096F853
:1000D0007D308DF80530072201A901F09EFC002833
:1000E0003FF4F1AED4E9010106F1740383E80300A3
:1000F00096F81831022B7FF442AF96F83031002B7E
:100100003FF43DAF174BDB6A9847FEF775F936E7CA
:10011000134E037A8DF8043096F8480096F87D3037
:100120008DF80530072201A901F077FC00283FF483
:10013000CAAEBC36ADE74368029301238DF80C309C
:10014000074B02A993F8480001F074FC00287FF4E3
:1001500016AFB8E6436802930023EFE7A83000200B
:10016000E42A0020DC8A030803795A1E0E2A3FF68F
:10017000AAAE934A82F8683001E7914B42685A650B
:10018000FDE68F4B42689A65F9E68D4B4268DA6569
:10019000F5E68B4B42681A66F1E6894B42685A666F
:1001A000EDE6874C037994F848008DF80430062278
:1001B00001A901F032FC00283FF485AE9DF804301F
:1001C00084F8DD30DBE67E4C03798DF8043094F85A
:1001D000480094F87C308DF80630052201A901F022
:1001E0001CFC00283FF46FAE9DF8043084F83930D1
:1001F000C5E6734C037994F848008DF804300A2260
:1002000001A901F00AFC00283FF45DAE9DF804301E
:1002100084F8DC30B3E66A4C037994F848008DF832
:100220000430092201A901F0F8FB00283FF44BAE8D
:100230009DF8043084F83830A1E6614B4268C3F879
:100240009420DA649BE65E4B027983F8982083F869
:10025000502094E65A4B4268C3F884208FE6584BEE
:100260004268C3F8CC208AE6012B40F0A480554CAC
:100270002421204603F03AFB636A984201D01720FC
:1002800022E61C2104F1280003F030FB636C984245
:10029000F5D14FF4807104F1480003F027FBD4F846
:1002A00048319842EBD1D42104F5A67003F01EFB2F
:1002B000D4F820329842E2D1002104F5097003F00D
:1002C00015FBD4F824329842D9D14FF4607104F56B
:1002D0000A7003F00BFBD4F8A8359842CFD1142153
:1002E00004F2AC5003F002FBD4F8C0359842C6D1FA
:1002F000334E2146304640F2C45203F0E1FA204624
:1003000040F2C452002103F0EFFA95F81B3485F84F
:10031000E833736FC5F8EC3396F87D3085F8F83321
:1003200040F20123A5F8FA33274B96F819019B6D8B
:10033000984724E68379012B3FF6C5AD204B4268F0
:100340004068C3F82C2100F091FF48E61C4B42683E
:10035000C3F8902013E61A4B027983F81F210EE6AA
:10036000174B8288A3F8882009E6154B8288A3F8EA
:100370008A2004E6124B8288A3F8D020FFE5104BB8
:100380008288A3F8D220FAE50D4B93F848200AB1F1
:10039000062A12D1A288A3F8A025F0E5084B93F80D
:1003A00048200AB1062A08D16268C3F8A425E6E508
:1003B00000F06AFCDBE5012086E5182084E500BF3B
:1003C000E42A002020250020DC8A0308DFF880C012
:1003D000F8B5DCF840339B07064635D48778002F04
:1003E00034D105460FCD1B4C0FC40FCD0FC42B6865
:1003F00023609CF89134B16843F020038CF8913469
:100400003378BBB10D2001F09BF810B111273846AD
:10041000F8BD7168B07801F031F90028F6D1B278F2
:100420000D4B302101FB02334FF0FF32D3F80C317A
:100430001A60ECE70E2001F083F80028E6D1F1689D
:100440000F2001F07DF8E8E70127E0E71627DEE757
:10045000A8300020CC2B0020E42A0020F0B5134F58
:10046000D7F840339B078BB006461AD4D8B9104C46
:1004700094F8E930BBB10146242201A801AD03F094
:1004800033FA0FCDE8340FC40FCD0FC42B682360AF
:1004900097F8913443F0200387F8913430460BB03D
:1004A000F0BD0126FAE71626F8E700BFA8300020C5
:1004B000E42A002000F00303F7B51C33294F137022
:1004C0001546D7F8402392070C4647D40A78013ADC
:1004D000012A03D90325284603B0F0BD00283FD1E7
:1004E000214E96F8E920002A3AD003F00F032B7032
:1004F00091F908308DF8043096F8480096F87D3070
:100500008DF80530072201A901F087FA18B12B7880
:1005100023F004032B70636896F8480001930022CF
:1005200001A901F07AFA18B12B7823F008032B7097
:100530002D78002DCED194E807000C4B83E80700FE
:1005400097F8912442F0200287F891242278012A1A
:10055000C1D1A3F1180000F0A3FBBCE70125BAE765
:100560001625B8E7A8300020E42A0020E42B00205C
:100570002DE9F04387B00023ADF80030064600288F
:1005800000F0EE800361FEF775FC20B101242046E7
:1005900007B0BDE8F08300F067FD0028F6D100F059
:1005A0005DFD014618B96F48142203F09DF96E4DA8
:1005B00095F89134012243F0040385F8552485F819
:1005C000913433788DF804300021013B8DF80520FB
:1005D000ADF806100C2B00F2BB80DFE803F007B982
:1005E000B9B97982B9B990B9AD9AA900D5F8407373
:1005F00017F02007CAD196F80480B8F1020F46D14F
:10060000DFF868815A4CFDF791FF96F9051098F8CC
:1006100048003A4601F05BFA88F83900B37988F867
:100620003830384607238DF80530FDF713FFFF23D8
:1006300004F58670A5F80C31C5F8084185F80471F9
:1006400003F066F804F58A7003F01CF83846FDF7ED
:100650005BFD0446002839D096F9051098F848004B
:10066000012201F034FA88F83900D5F89434336166
:10067000002C71D000F0F2FC002888D195F891345C
:1006800085F81A0460F3820385F891347FE7B8F1A6
:10069000010F4FF00204E8D1DFF8D0908DF814403C
:1006A00099F8480089F81D7102A901F0B1F9337970
:1006B00089F830318DF805708DF80680FDF7F2FB72
:1006C00095F8913443F0100385F891340024CCE779
:1006D00000226946022000F0F5FA0028F6D0132423
:1006E000C3E7244BB288DB6B96F90C10B0689847CF
:1006F000D5F8403343F00203C5F84033E6E702A9DA
:100700000D2000F055FB0028E0D0002269460D20A6
:10071000E1E7164B93F81831D3B9347904F00700A8
:1007200000F0ABFA8DF80040012269461020D2E7B4
:10073000002269461220CEE78DF8072000F08EFADD
:10074000044638B900F087FA204600F089FABDE780
:1007500002248AE7012488E701A800F0D3FB16E70A
:10076000032414E7FC340020A8300020E42A0020F1
:10077000AA300020DC8A03082DE9F04F99B08046AA
:10078000059118B9032019B0BDE8F08F002303616B
:10079000FEF770FB0446002840F0A58046460FCEC9
:1007A0000EAD0FC51422524898F800A0B8F80C708E
:1007B00098F90EB04F4E214603F096F84E4B0122A9
:1007C00083F8412496F83021022A25460BD196F869
:1007D0001821022A07D196F81E2122B9BAF1010F79
:1007E00038BF4FF0010ABAF1010F2BD0BAF1030F55
:1007F0002AD0BAF1000F33D102229DF83C30DDF847
:100800004090029362F34715012496F87C108DF80E
:10081000321002220CA996F848008DF8302001F021
:10082000E9F896F81A3196F830C196F81D1140B2E1
:10083000002B63D0BCF1010F57D1002955D1002CFA
:1008400061D153E00422D8E70023DDF83C90BDF8E5
:1008500040709DF942B0029365F01F050124D4E772
:100860004FF0000BD946CDF808B0CEE74FF00100AD
:1008700084F81A04D2E005F29A420BA900F0D6FAE5
:10088000002800F015811320049B33871A4B0022A7
:1008900083F81A2423E105F29A452A460BA900F0B1
:1008A000C5FA0028EFD10B9B84F82801C4F82C511D
:1008B00084F83031FCE0B9F1000F00F0F980002A33
:1008C00000F0F6804946E01C02F0FAFF94F8373257
:1008D00001332380ECE01220D6E70220D4E7072082
:1008E000D4E71320D2E701204DE7FCB90220F6E05F
:1008F000E8340020E42A0020A8300020002CF5D0A5
:100900005845B8BF584696F87C308DF8200005222F
:1009100096F848008DF8223008A901F07EF80028EA
:100920003FF430AF9DF8203086F839306F4A704B75
:10093000D2F89804D3F8904038B105F061FB6C4BC5
:1009400084423CBF002283F83A20198F1A8F93F813
:1009500030010491996A099152BA0028BFD093F8E6
:100960001B0100B9186393F81801ADF8582001383D
:1009700093F87C2093F81A411491D0F1000BD3F82E
:1009800088108DF85B204BEB000B93F8482093F810
:100990003A0093F868308DF85A3009AB0093554B04
:1009A00003904FF001008DF84C0015918DF85C20FC
:1009B000A3F12F01A3F1300213A88DF84D4000F0F0
:1009C000DBF8039B4FEA0B1B4BEA431B00264BEA69
:1009D000801B4BEAC413B145444C039308BF374610
:1009E0003A46494604F59C70CDE90A669B46268046
:1009F00084F81A6402F064FFE9B2A570C5F34215E9
:100A0000FAB2042D3A4E039B84F837223FF42EAFFE
:100A1000072D3FF450AF022D7FF45FAF364D84F8C1
:100A20000D110420029984F80401FF2084F80C01C0
:100A300084F8281184F81431D6F8E410C4F8085169
:100A400005F59B730AA8C4F8101184F83021C4F886
:100A50002C3100F013FC00287FF43DAF0A9BA4F872
:100A600044040BA8A4F81631C4F84C3400F0D2F9B1
:100A700000287FF408AF0B9BD3B196F93900FDF73E
:100A800025FA94F83732002B3FF405AF0B9B0F2B60
:100A90003FF6F1AE05F58B720BA90F2000F0C6F9F9
:100AA00000287FF4F0AE0B9B63F3030B84F814B1C2
:100AB0000598FDF729FB00287FF4E6AE099B86F830
:100AC0003A00B36200F082F900287FF40AAF94F88C
:100AD000913484F840A443F0010384F89134034B2B
:100AE000D3F89434C8F810304DE600BFA830002089
:100AF000E42A00204C2B0020AA30002037B50B4DF3
:100B00008DF8040004460F2295F8480001A900F072
:100B100084FF40B1064A85F81C4192F8913443F0B5
:100B2000200382F8913403B030BD00BFE42A0020D6
:100B3000A830002010B5FEF7EFFF044688B90A4838
:100B400005F098FA094805F095FA094805F092FA77
:100B500000F094F8FDF7EAFC064BDB6A9847204664
:100B600010BD0124FBE700BF103400202834002012
:100B700040340020DC8A03082DE9F04F8BB0477821
:100B80000093149B90F90C8090F90D6090F80EB0D2
:100B90008A464168196004469146002F58D00223C6
:100BA0008DF8103004A9C37B007C8DF8123000F062
:100BB00021FFB4F808C0618943B260689845454692
:100BC0006144B8BF1D46604534BF002701278842F5
:100BD00009D30A218DF81010207C019304A900F09C
:100BE00009FF019B46B2B4F808C0608961680CEB4C
:100BF000400E714519D3A1EB0C01B1FBF0FC00FBD9
:100C00001C1191B9984503DC2378CBB94FF0010B47
:100C100021238DF81030207CE37B8DF8115004A93E
:100C20008DF8123000F0E6FE45B2009B8AF80050C5
:100C3000384689F8006083F800B00BB0BDE8F08F4B
:100C40000223207C8DF8243006A900F0E1FEDDE7C8
:100C50004546EAE770477047704770470020704785
:100C60007047704770470020704700207047002091
:100C700070470020704700207047704770477047EA
:100C80000220704702207047022070477047002002
:100C900070477047704700207047002070477047CA
:100CA000704770477047000010B5054C4FF4037251
:100CB0002046002102F018FE0020C4E9000010BD0B
:100CC000C43500202DE9F8438146904600293CD0E8
:100CD0001F4C2023224604F1100012F8017F6FBB45
:100CE0008242FAD11B4E3368013403B93460736811
:100CF00003B11C6000252560C4F8088074601FFAE9
:100D000088F284F80490601D02F0DAFDB9F1110F49
:100D10004FF0000398BF104D6373D6F8083298BFA8
:100D200025FA09F503F1010398BF05F001054344D5
:100D30002573C6F808323846BDE8F883013B13F046
:100D4000FF030446C6D10227F5E70127F3E700BFFA
:100D5000CB350020C43500202007020010B518B3A1
:100D6000124A1368984204D103681360002305E017
:100D70000B46002BFAD019688842F9D15168884295
:100D800008BF53600BB101681960D2F8083281685E
:100D9000013B00245B1A04602146C2F8083210228D
:100DA00002F0A2FD204610BD0120FCE7C435002062
:100DB000054B1B6813B11A798242FAD1002B0B60E4
:100DC0000CBF032000207047C435002010B5054B30
:100DD000186800B910BD037B04680BB9FFF7BEFFAC
:100DE0002046F6E7C435002038B5084B084C186893
:100DF00000B938BD03790568112B05D824FA03F32F
:100E0000DB0701D5FFF7AAFF2846F1E7C43500202C
:100E10002007020028B1044BD3F8083203600020F9
:100E200070470120704700BFC43500202DE9F04114
:100E300007460E46154642B339B3154B1C680023CE
:100E40002CB93046FFF7E6FF0020BDE8F081A2682C
:100E5000F91A0132914215D32279EA54581C228999
:100E60005FFA80F8611D55FA80F002F029FDA36851
:100E7000246898445FFA88F3E2E720462568FFF784
:100E80006DFF2C46002CF8D1DBE70120DDE700BF29
:100E9000C43500200238C0B211289ABF014B185C3B
:100EA00000207047F983030830B50B4B93F82020DE
:100EB0000446084672B100211C330578A54208D0CB
:100EC00001319842CDB214BF04301038AA42F4D890
:100ED000002030BD1046FCE7D037002010B5084C8C
:100EE00000232060142204F10C00FF2184F820303C
:100EF000C4E9010002F0F8FC012384F8213010BDA0
:100F0000D037002010B50E4A92F82010042915D8C9
:100F1000936804781C7044785C70C478807898700A
:100F20000131DC7082F8201002F11C018B4214BFE9
:100F3000043302F10C039360012010BD0020FCE794
:100F4000D0370020094B93F8200068B15A6803F1AC
:100F50001C018A4200F1FF3014BF043203F10C027D
:100F600083F820005A600120704700BFD03700206E
:100F700010B5074B93F820200446084632B1596853
:100F8000FFF792FF10B101234470837010BD00BFC2
:100F9000D037002008B5064B93F820202AB15968B5
:100FA000FFF782FF08B1407808BD0120FCE700BFD1
:100FB000D037002030B50A4A92F82010536882F8E2
:100FC000210061B1916801241C32DD78587005B9A7
:100FD0009C70934214BF0433103B9942F5D130BD4D
:100FE000D037002008B5044B5968FFF75DFF003883
:100FF00018BF012008BD00BFD0370020F7B504227C
:10100000154E044600210DEB020096F8207002F008
:101010006BFC0025EBB29F4201D803B0F0BD7368B2
:10102000197821705A786270987838B13368204600
:101030009B689847FFF786FF0135EBE7DB788DF873
:1010400004108DF805208DF80730FFF77BFF01A80D
:10105000FFF758FFF0E700BFD0370020014B93F8AF
:1010600020007047D0370020034B93F8200004285D
:1010700094BF002001207047D03700201FB5002406
:10108000CDE90244C41F8DF800408DF801100C0A10
:10109000ADF80420090C120C8DF803108DF8062011
:1010A0008DF8073002461B0A012168468DF8024080
:1010B0008DF8083002F073FA002818BF0E2004B033
:1010C00010BD2DE9F04188B090460D460F9A0746B5
:1010D000002847D000240121CDE904448DF81010E8
:1010E0009DF838108DF81510ADF81630190CCDE9B3
:1010F00000441B0ECDE902448DF81930ADF81A20DA
:10110000130C120E07948DF818108DF81C308DF802
:101110001D20E3B21E01002DF6B203DC002008B052
:10112000BDE8F081013310218DF81F3042466B4637
:101130000DEB010002F0C9F90346A8B9102D2846AD
:101140003E44A8BF10206946327811F801CB013324
:1011500082EA0C02984206F8012BF5DC103D2DB214
:101160000134D6E70920DAE70E20D8E70138032852
:1011700015D8DFE800F002080C100A4B1B681B6949
:101180000B6000207047074B1B685B69F8E7054B55
:101190001B689B69F4E7034B1B68DB69F0E70520DC
:1011A000704700BFF43700202DE9F041C4B00C4671
:1011B0004A9E17461D468046B8B3B1F5807F36D8A3
:1011C0004FF488720021684602F08EFB4923009399
:1011D0004FF48073ADF804302B0C8DF80830330CCD
:1011E000ADF80650ADF80A608DF80C3022460023A9
:1011F000414604A82D0E360E8DF80E308DF809509C
:101200008DF80D608DF80F4002F05AFB04F11001CB
:101210004B9A3B4689B2684602F041F910B1012869
:1012200018BF0E2044B0BDE8F0810920FAE70D2078
:10123000F8E7000010B590B10A4C28220021206088
:1012400002F052FB2368084A1A6000204FF0FF3278
:10125000C3E90302C3E90522C3E9072210BD082040
:10126000FCE700BFF437002000010101024B1B68BE
:1012700018600020704700BFF437002030B1044BE5
:101280001B68DB680133036000207047092070474A
:10129000F437002013B500230C460193CAB101A90D
:1012A000FFF764FF18B9019B591C02D1146002B00A
:1012B00010BD99B2611A002901DD5C18F6E702D170
:1012C00013600720F3E71B0C1B0403F580331C4459
:1012D000ECE70920EBE7000028B1044B1B681C3346
:1012E0004362002070470920704700BFF437002098
:1012F0001FB5044600B3002303A8039302F0A6F928
:10130000104ABDF80C30126820469380E38200F04A
:10131000A8FA98B904F11803009321680123132255
:1013200002F0B2F860B9204600F09BFA003818BF0E
:101330000120000104B010BD0920FBE71020F9E7EF
:101340000E20F7E7F4370020F0B5054687B01C46BD
:1013500013B9092007B0F0BD2E4E3368DB68834215
:1013600055D894F82020002A0CBF08220922834275
:1013700005D3204600F0A9FA68B11020EAE700235F
:1013800001900093A36894F82810606AFFF799FE13
:101390000028EED0DEE723792168B4F808C0A768FA
:1013A000043B9AB20029D4D0B2F5807F2DD8ADF895
:1013B0000EC08DF817304FEA174C04F12C033F0E86
:1013C0008DF8117000932F0C08234FF0490EADF8E3
:1013D0000C008DF814708DF816002F0E0DEB030025
:1013E000CDF808E08DF810C0ADF812508DF81570EA
:1013F00002F04AF808B10E20ACE7204600F065FA8A
:101400000028BAD13368DD60A4E70D20A2E70620EA
:10141000A0E700BFF43700202DE9FF410A9D804678
:101420000F4616461C46002D5AD0002303A910462D
:101430000393FFF79BFE18B1062004B0BDE8F081CE
:10144000039B9C4201D80133F6D1284600F0AEF947
:10145000002847D1264B1A78424503D01A794245D5
:1014600042D10120AA68BA4240D103EB8002EB6A64
:1014700092F801802979CDE90043043992782868EF
:101480003B4689B2FFF790FE0028D6D195F8203070
:101490000194002B4FF00103009314BF4246082231
:1014A00095F82810686A3B46FFF70BFE0028C4D168
:1014B000013E032EC1D8DFE806F002070B0F0D4BEB
:1014C0001B681C611C62B8E70A4B1B685C61F9E78A
:1014D000084B1B689C61F5E7064B1B68DC61ACE7B9
:1014E0000920AAE70F20A8E70B20A6E70220A4E71F
:1014F000A0040020F43700201FB50B294FF0000393
:10150000CDE90033CDE902330A4607D00C2914D0C7
:101510000A2910D00A2005B05DF804FB012802D189
:1015200020238DF800300021684602F038F80028AA
:1015300018BF0E20EFE73023F3E70B21F4E700009C
:1015400038B5054602F026F8044610B10E242046B0
:1015500038BD002DFBD1094B1B680B219878FFF794
:10156000CBFF0028F2D10C21FFF7C6FF0028EDD1F8
:101570000A21FFF7C1FF0028E9D0E7E7F437002090
:101580002DE9F04380468FB00C461746002A6BD0F9
:10159000002969D0002529461D2206A805951EF0C0
:1015A0009DF88DF81350344D2B680DF114099E8869
:1015B000CDF804900DF1130302933B7900933B683F
:1015C00032462146404602F006F800284ED13868DF
:1015D0003A79494602F074F9384600F099F8002843
:1015E00046D13C7AFA79BB79240444EA02241C43AC
:1015F0002B689A6894423DD99C609DF813000B219A
:10160000FFF77AFF034658BB0C21FFF775FF03462F
:1016100030BB0A21FFF770FF034608BB7B7ABA7A1A
:10162000FF7A3F0447EA02271F433A4633462146E2
:101630000920FFF723FD034690B933463A46214679
:101640000820FFF71BFD034650B92A689DF81310C8
:1016500091700021D1604FF0FF31C2E90411916116
:1016600018460FB0BDE8F0830923F9E70E23F7E72A
:101670000F23F5E70323F3E7F437002070B588B0B4
:1016800000293FD0214C2378834231D023798342F3
:101690003AD101220023CDE90133CDE9053304EB32
:1016A0008204039307930123C1F30720CDB28DF881
:1016B0000030C1F30743090E8DF802008DF80410C5
:1016C00002268DF812008DF814106278E1788DF8FA
:1016D000015068468DF803308DF810608DF8115078
:1016E0008DF8133001F05BFF20B10E2008B070BD03
:1016F0000022CFE7A278E17804A801F050FF00288B
:10170000F4D0F2E70920F1E70B20EFE7A004002076
:1017100010B50446002845D00168002942D011F8D0
:10172000013B43710322063002F0CAF8204603222F
:1017300050F8091B043102F0C3F82168CB79E3604B
:101740000A7A43EA0223E3604A7A43EA0243E36007
:101750008A7A43EA0263E360CB7A23740B7B637477
:101760002379212B1AD110220D3104F1120002F03D
:10177000A7F81D222168501C8B5C6362085C43EA59
:101780000023901C6362085C033243EA00436362F7
:101790008A5C43EA02636362002010BD112B03DC04
:1017A0000D22E7E70220F8E70120F6E710B504462E
:1017B000002854D00168002951D00B7843714B7830
:1017C00083608A7843EA02238360CA7843EA02434B
:1017D00083600A7943EA026383604B7903738B79F0
:1017E000C381CA7943EA0223027BC38102F00F025C
:1017F0000831103002F064F8237B002203F00F035D
:1018000084F8202084F82820227903F10800111A96
:1018100004290DDD21680933043AD21A085C84F8E2
:101820002000D2B2606A84F82820194402F048F8F7
:10183000237922681A44002012F8043CE36212F86B
:10184000031C43EA0123E36212F8021C43EA01434A
:10185000E36212F8012C43EA0263E36210BD022046
:10186000FCE710B5044660B3036853B30279162A47
:1018700029D942791A700146082251F8060B013025
:1018800002F028F82146082251F80E0B093002F028
:1018900021F82368E28A5A74E38A22681B0A937447
:1018A0002368A269DA74A36922681B0A1375236886
:1018B000628B5A752368E27E9A7517232371002084
:1018C00010BD0120FCE70220FAE738B504460028E5
:1018D00063D00168002960D0037B90F8282003F0D2
:1018E0000F03002A57D10833207904321344984259
:1018F00055D363790B702368A2685A70A368226875
:101900001B0A937023686289DA702368E27A1A717D
:101910002368227B5A712368E2899A71E3892268DD
:101920001B0A2146D371227B51F8100B02F00F02E3
:10193000083001F0C5FF237B94F8282003F00F0343
:1019400003F108052AB1226894F82010515503F1DB
:101950000905206894F82820616A284401F0B0FF46
:1019600094F828302268E16A2B44D1545A1CE16A69
:10197000206892B2090A81549A1C2168E08D92B2C3
:101980008854DA1C216894F82F0092B204338854EA
:101990002371002038BD0933A6E70120FAE70220B1
:1019A000F8E70000024B1A8810431880704700BF08
:1019B000F837002008B5074B1B883BB1FEF7ACF8A1
:1019C000002814BF6FF00200002008BD6FF0010076
:1019D000FBE700BFF837002010B5034B00241C8044
:1019E000FEF790F8204610BDF8370020B0FA80F0DE
:1019F0004009704782B018B9084602B000F0CAB872
:101A0000002002B0704710B9084600F079B970475D
:101A100010B9084600F090B97047034608461146D1
:101A20000BB900F0DDB90020704710B9084600F08E
:101A300039BD704710B9084600F0FEB90020704764
:101A400010B40446084611461A46019B14B910BC4E
:101A500000F00CBA10BC70470346084611460BB99B
:101A600000F036BA0020704710B40446084611460C
:101A70001A4614B910BC00F0A3BA002010BC70477D
:101A800030B40546084611461A46DDE902341DB950
:101A9000029430BC00F022BB002030BC704710B96B
:101AA000084600F0D3BB0020704710B9084600F08C
:101AB00037BD0020704710B9084600F0E2BB002097
:101AC000704710B9084600F0DFBB0020704703469E
:101AD000084611460BB900F0F9BB0020704710B45E
:101AE0000446084611461A46019B14B910BC00F082
:101AF000EFBB092010BC704710B4044608461146DD
:101B00001A4614B910BC00F02DBDC8B210BC704705
:101B10000048704701000102064B10B51B6A0446DD
:101B2000984730B10448054B204498428CBF0020B0
:101B3000012010BDDC8A0308403576C9405DC6002F
:101B4000F0B5114B85B00C4610491F56054601F003
:101B500017F80F4BE4B25E6A072D4FF00103CDE991
:101B6000024301460AD105220023CDE900234FF4A8
:101B70007A727A431846B04705B0F0BD08220020BB
:101B8000CDE900203A46F5E7C4840308A48403089D
:101B9000DC8A03081FB5002300930378013B372B31
:101BA00021D8DFE803F01C242020201E2020202044
:101BB0004143454E2055585B5E6164206C1E6E7338
:101BC000787A7D207F83262020202020202020203E
:101BD0002020202085878C2020858C208E92C37821
:101BE0000BB102230093009805B05DF804FB8378E5
:101BF000F6E743788DF8043007238DF805308378B5
:101C0000003B18BF01235B008DF8063010238DF8D0
